:100000000C944C160C947D160C947D160C947D1655
:100010000C947D160C947D160C947D160C947D1614
:100020000C947D160C947D160C947D160C947D1604
:100030000C947D160C9458590C947D160C947D16D6
:100040000C947D160C9450C40C947D160C947D1663
:100050000C947D160C947D160C9483760C940E599A
:100060000C947D160C94C14B0C947D160C947D164B
:100070000C947D160C947D160C947D160C947D16B4
:100080000C947D160C947D160C947D160C947D16A4
:100090000C947D160C947D160C947D160C947D1694
:1000A0000C947D160C947D160C947D160C947D1684
:1000B0000C947D160C947D160C947D160C947D1674
:1000C0000C947D160C947D160C947D160C947D1664
:1000D0000C947D160C947D160C9473580C94345823
:1000E0000C947D168D31AA31DB31F8310D32363268
:1000F000A3320933B233FA370838013828382C389C
:100100004638A13C5B38A738CE38F5381E397439EB
:1001100085399639A739B839C939A13CAC3BA13CDE
:10012000B73B273C2D3C4D3C37B83AB829B82DB8E1
:1001300033B871B83EB842B848B84CB850B856B8A1
:100140005AB85EB871B864B868B86CB8D4BDD9BDD7
:10015000DEBDE8BDF2BD6BBEFCBD04BE0CBE16BE6E
:1001600020BE2ABE39BE43BE6BBE4DBE57BE61BE69
:10017000084AD73B3BCE016E84BCBFFDC12F3D6C0E
:1001800074319ABD56833DDA3D00C77F11BED9E474
:10019000BB4C3E916BAAAABE000000803F05A84C54
:1001A000CDB2D44EB93836A9020C50B99186880820
:1001B0003CA6AAAA2ABE000000803F004E414E493C
:1001C0004E495459494E46CDCCCC3D0AD7233C1715
:1001D000B7D13877CC2B329595E6241FB14F0A0062
:1001E0000020410000C84200401C4620BCBE4CCA52
:1001F0001B0E5AAEC59D74434F4D4D554E4943415C
:1002000054494F4E0044525952554E004552524F98
:10021000525300494E464F004543484F0047322F46
:1002200047332062616420706172616D657465722C
:10023000730A00206F6620004D424C20473239205F
:10024000706F696E74200059206F7574206F66207E
:1002500072616E67652028312D35292E0A005820DD
:100260006F7574206F662072616E67652028312D6E
:1002700035292E0A004D6573682070726F62696EB1
:100280006720646F6E652E0A005374617274206D6E
:100290006573682070726F62696E67207769746831
:1002A0002022473239205331222066697273742E1E
:1002B0000A004732380A47323920533200537461FA
:1002C00074653A20004D65736820626564206C6532
:1002D00076656C696E6720686173206E6F2064615B
:1002E00074612E0A0053206F7574206F662072614E
:1002F0006E67652028302D35292E0A004D657368FC
:1003000020706F696E742063616E6E6F7420626519
:10031000207265736F6C7665640A00456E642066B2
:10032000696C65206C6973740A00426567696E20A8
:1003300066696C65206C6973740A00286E6F2066AC
:10034000696C6529005344207072696E74696E6728
:10035000206279746520004E6F74205344207072BF
:10036000696E74696E670A0043757272656E7420F7
:1003700066696C653A20002569730025696D202542
:100380006973002569682025696D2025697300253A
:100390006964202569682025696D20256973002519
:1003A000697920256964202569682025696D2025E3
:1003B0006973005072696E742074696D653A20002B
:1003C0006F6E2E0A006F66662E0A00473236204492
:1003D000656275672000180213020C020502F7011E
:1003E0006F66660044454255473A004B494C4C45C0
:1003F000442E20004D3131332053006F6B002C20F0
:10040000002C2000544845524D414C5F50524F54EF
:10041000454354494F4E004155544F5245504F5259
:10042000545F53445F53544154555300454D455216
:1004300047454E43595F5041525345520043415343
:10044000455F4C494748545F4252494748544E45DE
:10045000535300544F47474C455F4C49474854530A
:1004600000534F4654574152455F504F5745520035
:100470004255494C445F50455243454E54004C450B
:1004800056454C494E475F44415441005A5F5052D3
:100490004F4245004155544F4C4556454C00505233
:1004A000494E545F4A4F420050524F4752455353B2
:1004B000004155544F5245504F52545F54454D5092
:1004C00000564F4C554D45545249430045455052F6
:1004D0004F4D0053455249414C5F584F4E5F584F66
:1004E0004646004649524D574152455F4E414D45A3
:1004F0003A4D61726C696E20312E312E39202847B9
:1005000069746875622920534F555243455F434FC4
:1005100044455F55524C3A68747470733A2F2F6794
:1005200069746875622E636F6D2F4D61726C696EB0
:100530004669726D776172652F4D61726C696E20CC
:1005400050524F544F434F4C5F56455253494F4EB4
:100550003A312E30204D414348494E455F54595061
:10056000453A3344205072696E7465722045585480
:1005700052554445525F434F554E543A31205555DC
:1005800049443A63656465326132662D34316132C3
:100590002D343734382D396231322D633535633699
:1005A000326633363766660A002F2F20002054004B
:1005B000205200416363656C65726174696F6E3AC5
:1005C0002050005741524E494E4721204C6F772012
:1005D0005A204A65726B206D6179206C65616420D8
:1005E000746F20756E77616E7465642070617573C9
:1005F00065732E0A00546F6F206661722066726FF9
:100600006D207265666572656E636520706F696ED8
:10061000740A0020466C6F773A20000001363726B6
:10062000032BFFFFFF3C3D382AFFFFFFFF2E303E2C
:1006300012FFFFFFFFFFFFFF0809FF2C071A1C181E
:10064000FFFFFF08440A2C4324221E20643A0020A6
:10065000693A0020703A00496E76616C69642065E1
:10066000787472756465720A0043290A0061626CCD
:10067000656420286D696E2074656D702000436F7D
:100680006C6420657874727564657320617265208E
:100690000020643A0020693A0020703A004E6F2032
:1006A00063617365206C696768740A004545505240
:1006B0004F4D204F4B0A00205A004475616C204575
:1006C0006E6473746F702041646A7573746D656EC7
:1006D0007420286D6D293A20003F4B2076616C759F
:1006E00065206F7574206F662072616E67652028C3
:1006F000302D3130292E0A00416476616E63652009
:100700004B3D004163746976652045787472756469
:1007100065723A2000496E76616C69642065787470
:1007200072756465720A0043616E6E6F7420656E47
:10073000746572207375626469723A2000473931BA
:100740000A4731205A2D302E310A47393000537074
:10075000656369616C204D656E753A205A20446F5F
:10076000776E20302E310A004739310A4731205A3E
:100770002D302E30320A473930005370656369617D
:100780006C204D656E753A205A20446F776E20308C
:100790002E30320A004739310A4731205A2B302E89
:1007A00030320A473930005370656369616C204DFF
:1007B000656E753A205A20557020302E30320A006E
:1007C0004739310A4731205A2B302E310A47393008
:1007D000005370656369616C204D656E753A205AEF
:1007E00020557020302E310A004732392053320014
:1007F0005370656369616C204D656E753A204E6576
:100800007874204D65736820506F696E740A0047D4
:100810003239205331005370656369616C204D6536
:100820006E753A205374617274204D657368204C64
:100830006576656C696E670A004D31343020533639
:1008400030005370656369616C204D656E753A20A8
:1008500050726568656174204265640A004D3530E8
:1008600032005370656369616C204D656E753A2086
:100870004C6F61642046572044656661756C7473E3
:100880000A004D353030005370656369616C204D4E
:10089000656E753A205361766520454550524F4D3F
:1008A0000A004D33303320452D312053363020435C
:1008B00036205531005370656369616C204D656E5B
:1008C000753A204175746F2054756E6520486F74B9
:1008D000626564205069640A004D3130362053321D
:1008E00030340A4D333033204530205332313020FC
:1008F0004336205531005370656369616C204D6546
:100900006E753A204175746F2054756E6520486F7E
:1009100074656E64205049440A003C5370656369F5
:10092000616C5F4D656E753E003C53706563696137
:100930006C5F4D656E753E002F002F002F002F2E2F
:100940002E0A002F2E2E002F2E2E003C5370656392
:1009500069616C5F4D656E753E0A003C537065635E
:1009600069616C204D656E753E003C53706563692E
:10097000616C204D656E753E003C4C6F6164204695
:10098000572044656661756C74733E003C4C6F6122
:10099000642046572044656661756C74733E003C64
:1009A0004175746F2054756E6520486F746265647C
:1009B000205049443E003C4175746F2054756E656B
:1009C00020486F74626564205049443E003C417584
:1009D000746F2054756E6520486F74656E64205086
:1009E00049443E003C4175746F2054756E65204843
:1009F0006F74656E64205049443E003C45786974CC
:100A00003E003C457869743E003C53617665204564
:100A10004550524F4D3E003C536176652045455050
:100A2000524F4D3E003C4E657874204D65736820F2
:100A3000506F696E743E003C4E657874204D65734E
:100A40006820506F696E743E003C5374617274206C
:100A50004D657368204C6576656C696E673E003C39
:100A60005374617274204D657368204C6576656CB3
:100A7000696E673E003C507265686561742062650E
:100A8000643E003C50726568656174206265643E36
:100A9000003C5A20446F776E20302E313E003C5A85
:100AA00020446F776E20302E313E003C5A20446F38
:100AB000776E20302E30323E003C5A20446F776EE5
:100AC00020302E30323E003C5A20557020302E30DF
:100AD000323E003C5A20557020302E30323E003CD1
:100AE0005A20557020302E313E003C5A205570203F
:100AF000302E313E0056313136004A333320004D1E
:100B00003530300A4D3432302053310A4731205AC3
:100B1000313020463234300A4731205830205930A5
:100B2000204636303030004A3232004A32320047F6
:100B300031205A3520463234300A47312058313975
:100B400030205932302046363030300A4731205A72
:100B5000302046323430004731205A352046323476
:100B6000300A473120583139302059313930204648
:100B7000363030300A4731205A3020463234300087
:100B80004731205A3520463234300A473120583117
:100B90003930205932302046363030300A47312043
:100BA0005A302046323430004739310A4731205A12
:100BB000313020463234300A4739300A4732380A59
:100BC0004732390A473120583230205932302046D6
:100BD000363030300A4731205A3020463234300027
:100BE0004A3032004A3132004731205A3130004F0A
:100BF0004B004731205A313000473930004731200F
:100C00004525694635303000473120452D302E319D
:100C10004625690047312045302E31462569004779
:100C200031205A2569462569004731205A2D302E3A
:100C300031462569004731205A302E31462569005A
:100C400047312059256946256900473120592D3003
:100C50002E314625690047312059302E314625690D
:100C60000047312058256946256900473120582D15
:100C7000302E314625690047312058302E31462527
:100C800069004739310047323800473238205A006E
:100C90004732382059004732382058004132305608
:100CA00020004731205A3130004A3034004A323176
:100CB000004A3230004B494C4C45442E20004A300B
:100CC0003400454E4400464E20004A303200393947
:100CD000393A393939004D00480041375620004132
:100CE0003656202D2D2D004A303200413656200038
:100CF0005A3A2000593A2000583A2000413556000F
:100D000041345620004133562000413256200041E4
:100D10003156200041305620004D3834004A3136DB
:100D2000004A3138004739310A4731205A313020E2
:100D3000463234300A473930004A3134004A3030C4
:100D4000004A3031004A31300024F4D43050C38E90
:100D500020C2A24017828B7011127A910D816CD93A
:100D60000AA861E108C7586607615143061E4B5D3A
:100D700005C145A7041A411104093D980371393191
:100D8000034036DB0265339102D4305402802E1DBD
:100D900002632CEE01752AC501B028A0011027813D
:100DA000018F2564012B244B01E0223401AC211F6B
:100DB000018D200D01801FFC00841EED00971DDFBA
:100DC00000B81CD200E61BC600201BBC00641AB28F
:100DD00000B219A8000A19A0006A189900D1179149
:100DE0000040178B00B516840031167E00B31579CC
:100DF000003A157300C7146F0058146A00EE1366AA
:100E0000008813630025135E00C7125B006C125745
:100E10000015125400C111510070114F0021114BE7
:100E200000D61049008D10470046104400021042C1
:100E300000C00F4000800F3E00420F3C00060F3BF9
:100E400000CB0E3800930E37005C0E3500270E34B1
:100E500000F30D3200C10D3100900D3000600D2EF9
:100E600000320D2D00050D2C00D90C2B00AE0C29E5
:100E700000850C29005C0C2700350C27000E0C2681
:100E800000E80B2400C40B2400A00B23007D0B23DF
:100E9000005A0B2100390B2100180B2000F80A1F03
:100EA00000D90A1E00BB0A1E009D0A1D00800A1DF3
:100EB00000630A1C00470A1B002C0A1B00110A1AB7
:100EC00000F7091A00DD091900C4091900AB091956
:100ED00000920917007B091800630917004C0916D6
:100EE0000036091600200916000A091500F5081534
:100EF00000E0081400CC081400B8081400A408147A
:100F000000900813007D0812006B081300580812A7
:100F100000460812003408110023081100120811BD
:100F20000001081100F0071000E0071000D00710C2
:100F300000C0071000B0070F00A107100091070EB6
:100F40000083070F0074070F0065070E0057070E98
:100F50000049070E003B070D002E070E0020070D6D
:100F60000013070D0006070D00F9060C00ED060D35
:100F700000E0060C00D4060C00C8060C00BC060CF1
:100F800000B0060C00A4060B0099060C008D060BA1
:100F90000082060B0077060B006C060B0061060A48
:100FA0000057060B004C060A0042060A0038060AE3
:100FB000002E060A0024060A001A060A0010060976
:100FC0000007060A00FD050900F4050900EB050904
:100FD00000E2050900D9050900D0050900C7050987
:100FE00000BE050900B5050800AD050800A5050906
:100FF000009C050800940508008C0508008405087D
:10100000007C050800740508006C050700650508EC
:10101000005D050700560508004E05070047050757
:10102000004005080038050700310507002A0507BC
:1010300000230507001C050600160507000F05071D
:10104000000805060002050700FB040600F504077A
:1010500000EE040600E8040600E2040700DB0406D4
:1010600000D5040600CF040600C9040600C3040628
:1010700000BD040600B7040600B1040500AC040678
:1010800000A6040600A00405009B040600950405C4
:1010900000900406008A040500850405008004060B
:1010A000007A04050075040500700405006B040552
:1010B0000066040500610405005C04050057040592
:1010C00000520405004D04050048040500430405D2
:1010D000003E0404003A0405003504050030040411
:1010E000002C04050027040400230405001E04044A
:1010F000001A04040016040500110404000D040481
:1011000000090405000404040000040400FC0304B6
:1011100000F8030400F4030400F0030400EC0304EB
:1011200000E8030400E4030400E0030400DC03041B
:1011300000D8030400D4030400D0030400CC03044B
:1011400000C8030300C503030024F404D9201BC412
:101150000C5C0E9804C4095F0265077101F405F97F
:1011600000FB04B30048048700C10369005803551D
:101170000003034500BE023A008402310053022AF4
:10118000002902250004022000E4011C00C8011906
:1011900000AF0117009801140084011300710110C1
:1011A000006101100051010E0043010D0036010BDA
:1011B000002B010B0020010B00150109000C010997
:1011C0000003010800FB000800F3000800EB000723
:1011D00000E4000600DE000600D8000600D200068B
:1011E00000CC000500C7000500C2000500BD0004DA
:1011F00000B9000400B5000400B1000400AD000413
:1012000000A9000400A5000300A20003009F000441
:10121000009B000300980003009500020093000368
:1012200000900003008D0002008B00030088000284
:10123000008600020084000300810002007F00029B
:10124000007D0002007B00020079000200770001AF
:1012500000760002007400020072000100710002BA
:10126000006F0002006D0001006C0002006A0001C6
:1012700000690002006700010066000100650001CE
:1012800000640002006200010061000100600001D2
:10129000005F0002005D0001005C0001005B0001D6
:1012A000005A0001005900010058000100570001D8
:1012B00000560001005500010054000100530000D9
:1012C00000530001005200010051000100500001D4
:1012D000004F0001004E0000004E0001004D0001D3
:1012E000004C0001004B0000004B0001004A0001CF
:1012F00000490001004800000048000100470001CB
:1013000000460000004600010045000000450001C5
:1013100000440001004300000043000100420000BF
:1013200000420001004100000041000100400001B6
:10133000003F0000003F0001003E0000003E0001B1
:10134000003D0000003D0001003C0000003C0000AA
:10135000003C0001003B0000003B0001003A00009F
:10136000003A000100390000003900010038000097
:10137000003800000038000100370000003700018D
:101380000036000000360000003600010035000085
:10139000003500000035000100340000003400007A
:1013A000003400010033000000330000003300016E
:1013B0000032000000320000003200010031000065
:1013C000003100000031000100300000003000005A
:1013D00000300001002F0000002F0000002F00004F
:1013E000002F0001002E0000002E0000002E000142
:1013F000002D0000002D0000002D0000002D000138
:10140000002C0000002C0000002C0000002C00012B
:10141000002B0000002B0000002B0000002B00011F
:10142000002A0000002A0000002A0000002A000113
:101430000029000000290000002900000029000008
:1014400000290001002800000028000000280000FA
:1014500000280000002800010027000000270000ED
:1014600000270000002700000027000100260000E0
:1014700000260000002600000026000000260001D3
:1014800000250000002500000025000000250000C8
:1014900000250000002500010024000000240000B9
:1014A00000240000002400000024000100230000AC
:1014B00000230000002300000023000000230000A0
:1014C0000023000000230001002200000022000091
:1014D0000022000000220000002200000022000183
:1014E0000021000000210000002100000021000078
:1014F0000021000000210000002100010020000068
:10150000002000000020000000200000002000005B
:10151000002000000020000000200001001F00004B
:10152000001F0000001F0000001F0000001F00003F
:10153000001F0000001F0001001E0000001E000030
:10154000001E0000001E000000232C0000B8220036
:1015500000561800003A0F0000B8080000B104005F
:1015600000710200003E010000696E206D6F76651B
:101570005F746F282920666565645F76616C7565A8
:1015800020666F722058593A002C2065793D002959
:10159000202D3E202865783D002C2073793D0020C9
:1015A000436F6E6E656374696E6720776974682037
:1015B000766572746963616C206C696E652028734E
:1015C000783D002C2065793D0029202D3E2028659E
:1015D000783D002C2073793D0020436F6E6E65636B
:1015E00074696E67207769746820686F72697A6FB2
:1015F0006E74616C206C696E65202873783D003FC5
:1016000053706563696669656420582C5920636F5F
:101610006F7264696E617465206F7574206F6620E7
:10162000626F756E64732E0A003F285229657065DB
:1016300061742076616C7565206E6F7420706C61CA
:10164000757369626C653B206D75737420626520EB
:101650006174206C6561737420312E0A003F28523A
:10166000296570656174206D7573742062652073DF
:101670007065636966696564207768656E206E6F62
:1016800074207573696E6720616E204C43442E0A86
:10169000003F537065636966696564206E6F7A7A8E
:1016A0006C652074656D7065726174757265206E0D
:1016B0006F7420706C61757369626C652E0A003FEF
:1016C0005370656369666965642066696C616D6500
:1016D0006E742073697A65206E6F7420706C61750A
:1016E0007369626C652E0A003F53706563696669B1
:1016F0006564207072696D65206C656E6774682022
:101700006E6F7420706C61757369626C652E0A006F
:101710003F5072696D65206C656E677468206D75E9
:1017200073742062652073706563696669656420FF
:101730007768656E206E6F74207573696E672061BF
:101740006E204C43442E0A003F53706563696669FE
:101750006564206E6F7A7A6C652073697A65206E95
:101760006F7420706C61757369626C652E0A003F3E
:10177000537065636966696564205265747261635C
:1017800074696F6E204D756C7469706C6965722038
:101790006E6F7420706C61757369626C652E0A00DF
:1017A0003F52657472616374696F6E204D756C741D
:1017B00069706C696572206D757374206265207341
:1017C00070656369666965642E0A003F53706563DE
:1017D0006966696564206C6179657220686569670E
:1017E0006874206E6F7420706C61757369626C65CB
:1017F0002E0A003F537065636966696564206265FF
:10180000642074656D7065726174757265206E6FA9
:101810007420706C61757369626C65202834302D9A
:1018200031343043292E0A0047323620636F6D6D04
:10183000616E6420737461727465642E20576169EF
:1018400074696E6720666F722068656174657228BE
:1018500073292E0A00024A3135004A3132004A31DA
:1018600037002020506C616E6E6572427566666549
:101870007242797465733A20002046726565204D86
:10188000656D6F72793A2000436F6D70696C6564A5
:101890003A204A616E20203420323031390A00204B
:1018A0007C20417574686F723A202864617669649F
:1018B00072616D69726F2C20666F7220416E796360
:1018C00075626963206933204D656761290A0032BA
:1018D0003031392D30312D303200204C617374207D
:1018E000557064617465643A2000312E312E390AD6
:1018F000004D61726C696E0020536F66747761727F
:10190000652052657365740A0020576174636864CA
:101910006F672052657365740A002042726F776E9C
:10192000206F75742052657365740A0020457874C1
:1019300065726E616C2052657365740A00506F7732
:10194000657255700A0073746172740A004D323406
:10195000004D3233202573006175746F25692E6741
:10196000006572726F722077726974696E67207495
:101970006F2066696C650A00205A3A0020593A00C7
:1019800020583A00656E6473746F707320686974D0
:101990003A2000446F6E6520736176696E67206639
:1019A000696C652E0A004D32390020746F6F206C0F
:1019B0006F6E6720657874727573696F6E207072D0
:1019C0006576656E7465640A0020636F6C642065DB
:1019D0007874727573696F6E2070726576656E7457
:1019E00065640A00454550524F4D2064617461732F
:1019F000697A65206572726F722E0A00290A0020CA
:101A000062797465733B206372632000536574745C
:101A1000696E67732053746F726564202800290A09
:101A2000002062797465733B206372632000207329
:101A3000746F7265642073657474696E6773207265
:101A40006574726965766564202800202863616C7E
:101A500063756C6174656429210A0020213D2000B2
:101A6000454550524F4D20435243206D69736D617F
:101A7000746368202D202873746F726564292000B8
:101A80002053697A653A2000496E6465783A2000EF
:101A9000204D61726C696E3D563535290A00284526
:101AA0004550524F4D3D00454550524F4D207665B3
:101AB0007273696F6E206D69736D61746368200065
:101AC0001000C90210012C0140012201700118010F
:101AD000B0010E01F00104015002FA00B002F00062
:101AE0003003E600D003DC009004D2007005C8008B
:101AF000A006BE000008B400B009AA00D00BA000E8
:101B0000600E960060118C0000158200201978008C
:101B1000C01D6E00A0226400B0275A00902C500017
:101B200000314600E0343C0010383200903A280082
:101B3000603C1E00A03D1400803E0A00203F0000D3
:101B40002CFFFFFFFFFF0001010101016265640A34
:101B5000002C2073797374656D2073746F707065D9
:101B60006421204865617465725F49443A200042EF
:101B700065642068656174696E67206661696C657B
:101B8000640048656174696E67206661696C6564AC
:101B90000045312048656174696E67206661696C33
:101BA00065640048656174696E67206661696C658B
:101BB000640070012C0190012701B0012201C001D5
:101BC0001D01F00118011002130130020E01600224
:101BD000090190020401C002FF000003FA00400363
:101BE000F5008003F000D003EB002004E600700451
:101BF000E100E004DC004005D700C005D20040064B
:101C0000CD00D006C8008007C3003008BE00F00831
:101C1000B900C009B400B00AAF00B00BAA00D00CE4
:101C2000A500000EA000500F9B00C010960050129F
:101C3000910000148C00C0158700B0178200B01905
:101C40007D00D01B7800001E730040206E009022A3
:101C50006900F024640040275F0090295A00E02BBF
:101C60005500102E500020304B0010324600E0335B
:101C7000410090353C001037370070383200A039F1
:101C80002D00B03A2800A03B2300603C1E00103D10
:101C90001900903D1400103E0F00703E0A00C03E37
:101CA0000500003F0000403FFBFF803FF6FFC03FC4
:101CB000F1FF453120544845524D414C2052554E7C
:101CC000415741590042454420544845524D414CEA
:101CD0002052554E4157415900546865726D616CF0
:101CE0002052756E61776179004531204572723AF4
:101CF000204D415854454D50004572723A204D4197
:101D00005854454D5020424544004D415854454D8E
:101D100050207472696767657265640045312045BB
:101D200072723A204D494E54454D50004572723AF8
:101D3000204D494E54454D5020424544004D494E9A
:101D400054454D5020747269676765726564004D33
:101D5000383420582059205A204500202F00204296
:101D6000403A0020403A006F70656E206661696CF1
:101D700065642C2046696C653A200043616E6E6F85
:101D800074206F70656E2073756264697220004AFA
:101D90003035004A3233004739310A4731205A2D55
:101DA000313020463234300A473930005344206302
:101DB000617264206F6B0A006F70656E526F6F7492
:101DC000206661696C65640A00766F6C756D652EBE
:101DD000696E6974206661696C65640A0045727297
:101DE0006F723A00534420696E6974206661696CB1
:101DF0000A006563686F3A00656E7175657565699F
:101E00006E672022004B494C4C45442E20005072F6
:101E1000696E7465722073746F7070656420647588
:101E20006520746F206572726F72732E2046697818
:101E300020746865206572726F7220616E6420750F
:101E40007365204D39393920746F20726573746160
:101E500072742E202854656D706572617475726598
:101E60002069732072657365742E20536574206930
:101E7000742061667465722072657374617274692E
:101E80006E67290A004E6F20436865636B73756D3A
:101E90002077697468206C696E65206E756D626567
:101EA000722C204C617374204C696E653A20004E90
:101EB0006F20436865636B73756D20776974682064
:101EC0006C696E65206E756D6265722C204C617355
:101ED00074204C696E653A2000636865636B7375A6
:101EE0006D206D69736D617463682C204C6173742F
:101EF000204C696E653A20004C696E65204E756D08
:101F0000626572206973206E6F74204C6173742057
:101F10004C696E65204E756D6265722B312C204CBC
:101F2000617374204C696E653A20004D3131300088
:101F30004D33310053442072656164206572726FC5
:101F4000720A00446F6E65207072696E74696E6704
:101F50002066696C650A00205A3A0020593A002030
:101F6000436F756E7420583A0020453A00205A3A63
:101F70000020593A00583A003A004361703A002074
:101F80005A00205900580020204D61783A20002046
:101F90005A00205900580020204D696E3A20004F09
:101FA0006E20004F666600536F667420656E647322
:101FB000746F70733A20004B642000236465666977
:101FC0006E652044454641554C545F004B692000E6
:101FD00023646566696E652044454641554C545FEF
:101FE000004B70200023646566696E652044454699
:101FF00041554C545F00504944204175746F7475CD
:102000006E652066696E6973686564212050757419
:1020100020746865206C617374204B702C204B69B0
:1020200020616E64204B6420636F6E7374616E7404
:10203000732066726F6D2062656C6F7720696E74B5
:102040006F20436F6E66696775726174696F6E2E7B
:10205000680A00504944204175746F74756E65209C
:102060006661696C6564212074696D656F75740AB9
:1020700000453120544845524D414C2052554E4167
:102080005741590042454420544845524D414C2047
:1020900052554E4157415900546865726D616C202C
:1020A00052756E61776179004531204865617469C8
:1020B0006E67206661696C656400426564206865CE
:1020C0006174696E67206661696C6564004865616A
:1020D00074696E67206661696C65640050494420CC
:1020E0004175746F74756E65206661696C656421F5
:1020F0002054656D706572617475726520746F6FC0
:1021000020686967680A00204B643A2000204B6908
:102110003A2000204B703A20000A20436C61737310
:10212000696320504944200A002054753A20002059
:102130004B753A2000206D61783A2000206D696E61
:102140003A200020643A200020626961733A20003E
:10215000504944204175746F74756E6520666169DD
:102160006C656421204261642065787472756465D1
:1021700072206E756D6265720A0050494420417587
:10218000746F74756E652073746172740A004F66A3
:10219000660A0046616465204865696768742000C6
:1021A000426564204C6576656C696E672000466107
:1021B000696C656420746F20656E61626C65204295
:1021C0006564204C6576656C696E670A004D6573C1
:1021D0006820426564204C6576656C20646174619A
:1021E0003A0A004D65736820706F696E74206361F0
:1021F0006E6E6F74206265207265736F6C766564B5
:102200000A004D34323120696E636F7272656374F7
:1022100020706172616D65746572207573616765A8
:102220000A007C3C3E5E2B3D3F2F5B5D3B2C2A220F
:102230005C00627573793A2070617573656420661D
:102240006F7220696E7075740A00627573793A2036
:1022500070617573656420666F7220757365720AAC
:1022600000627573793A2070726F63657373696E7B
:10227000670A004A3135004B494C4C45442E20003A
:102280004B494C4C20636175736564206279204B27
:10229000494C4C20627574746F6E2F70696E0A0021
:1022A0004B494C4C45442E20004B494C4C2063611B
:1022B0007573656420627920746F6F206D75636833
:1022C00020696E6163746976652074696D65202D7F
:1022D0002063757272656E7420636F6D6D616E64DC
:1022E0003A20004A3131005072696E74657220687C
:1022F000616C7465642E206B696C6C2829206361A5
:102300006C6C6564210A000000A0C00000000000A1
:102310000000005761726E696E673A20486F6D6900
:102320006E672042756D702044697669736F722004
:102330003C20310A000202040000A0400000A0403E
:10234000000000400000614300005C4300004D437A
:10235000FFFFFF20496E76616C69642065787472B6
:102360007564657220000000A0C00000000000003D
:10237000000000005C4300005C4300004D43486FD8
:102380006D696E67206661696C656400206E6F74AC
:1023900020656E74657265642E0A0046696C65205E
:1023A00064656C657465643A0044656C6574696F56
:1023B0006E206661696C65642C2046696C653A2004
:1023C0000050726F7465637465642050696E0A0012
:1023D0004A3036004A3034004A30370020573A003D
:1023E0004A3038004A30390020573A0054524947A1
:1023F0004745524544006F70656E003A20007A32BE
:102400005F6D696E007A5F6D696E00795F6D696EF0
:1024100000785F6D696E005265706F7274696E67E7
:1024200020656E6473746F70207374617475730AC1
:10243000000A4D6561737572656420706F696E7412
:10244000733A0A005A206F66667365743A20004E2C
:10245000756D20582C593A20352C350A00000000A3
:1024600001000000010000800055555500000040AB
:102470000033333300AAAA2A004992240000002026
:1024800000C7711C0099991900D1451700555515C1
:10249000003BB1130024491200111111000000107B
:1024A000000F0F0F00E3380E0043790D00CCCC0C69
:1024B00000C3300C00E8A20B0064210B00AAAA0A9A
:1024C00000703D0A009DD80900427B090092240952
:1024D00000DCD308008888080010420800000008CB
:1024E00000F0C107008787070075500700711C07BF
:1024F000003EEB0600A1BC06006990060066660679
:1025000000703E06006118060017F4050074D1053E
:10251000005BB00500B290050062720500555505DC
:102520000078390500B81E0500050505004EEC04CD
:102530000087D40400A1BD040090A70400499204C0
:1025400000C17D0400EE690400C756040044440441
:10255000005C320400082104004110040000000463
:10256000003FF00300F8E0030026D20300C3C303DA
:1025700000CCB503003AA803000A9B0300388E0381
:1025800000C08103009F750300D0690300505E0303
:10259000001D53030034480300913D03003333030F
:1025A0000016290300381F030097150300300C03A1
:1025B00000030303000BFA020049F10200BAE8022B
:1025C000005CE002002DD802002DD0020059C802A4
:1025D00000B0C0020031B90200DAB10200AAAA02BA
:1025E00000A0A30200BC9C0200FA9502005C8F02CE
:1025F00000DF88020082820200457C02002776020A
:102600000027700200436A02007C640200D05E0270
:10261000003F590200C85302000000210024002797
:10262000002A002D003000330001010000040107E2
:10263000010A0100002200250028002B002E003195
:1026400000340002010000050108010B0100002018
:10265000002300260029002C002F0032000001007A
:10266000000301060109010505050507050808081D
:1026700008020202020A0A08080404040401010113
:10268000010101010103030303030303030407071B
:10269000070C0C0C0C0C0C0C0C02020202060606B9
:1026A00006060606060B0B0B0B0B0B0B0B010210A1
:1026B000202008081020401020408002010201085C
:1026C000040201010204081020408080402010080C
:1026D0000402018004020180402010080402010865
:1026E00004020101020408102040800102040810C5
:1026F00020408000000A0B02090C0D0E080703049D
:1027000001000000000000000000000000000000C8
:1027100000000000000000000000000000000012A7
:102720001110000000000000000000000000000088
:10273000000000000000000000556E6B6E6F776EA9
:1027400020636F6D6D616E643A20220020666972AD
:1027500073740A005A0059005800486F6D652000D4
:102760000000484200004842000080400000000095
:1027700048617264636F6465642044656661756C6A
:10278000742053657474696E6773204C6F6164655F
:10279000640A00B80B0000D00700003C00000010E5
:1027A0002700000000FA430000FA430000C0400088
:1027B0000070420000A0420000A0420000C8433365
:1027C00033B94220286D6D290020204D393030204A
:1027D0004B004C696E65617220416476616E636581
:1027E0003A0A0020440020490020204D3330342094
:1027F000500020440020490020204D33303120502B
:10280000005049442073657474696E67733A0A0016
:10281000205A0020204D36363600456E6473746FA2
:10282000702061646A7573746D656E743A0A002075
:102830005A002059002020473239205333205800B5
:10284000205A0020204D3432302053004D657368EB
:1028500020426564204C6576656C696E673A0A00B3
:10286000205A0020590020204D3230362058004890
:102870006F6D65206F66667365743A0A00204500C7
:10288000205A0020590020580020540020530020D6
:10289000204D32303520510020453C6D61785F6518
:1028A0005F6A65726B3E0020583C6D61785F785FAF
:1028B0006A65726B3E20593C6D61785F795F6A652D
:1028C000726B3E205A3C6D61785F7A5F6A65726B0D
:1028D0003E00416476616E6365643A20513C6D69E7
:1028E0006E5F7365676D656E745F74696D655F7546
:1028F000733E20533C6D696E5F66656564726174FA
:10290000653E20543C6D696E5F74726176656C5FE4
:1029100066656564726174653E0020540020520053
:1029200020204D323034205000416363656C657265
:102930006174696F6E2028756E6974732F73322904
:102940003A20503C7072696E745F616363656C3EDF
:1029500020523C726574726163745F616363656C7D
:102960003E20543C74726176656C5F616363656C94
:102970003E0A00204500205A0020590020204D32F8
:1029800030312058004D6178696D756D2041636369
:10299000656C65726174696F6E2028756E697473F9
:1029A0002F7332293A0A00204500205A002059008E
:1029B00020204D3230332058004D6178696D756D9F
:1029C000206665656472617465732028756E69742C
:1029D000732F73293A0A00204500205A002059001D
:1029E00020204D3932205800537465707320706573
:1029F0007220756E69743A0A0020204D3230302002
:102A000044300A0020204D323030204400204469F8
:102A10007361626C65640A0046696C616D656E7411
:102A20002073657474696E67733A002020473231F1
:102A3000202020203B00FFFDFCFAF8F6F4F2F0EE37
:102A4000ECEAE9E7E5E3E1E0DEDCDAD9D7D5D4D298
:102A5000D0CFCDCBCAC8C7C5C3C2C0BFBDBCBAB931
:102A6000B7B6B4B3B2B0AFADACAAA9A8A6A5A4A29C
:102A7000A1A09E9D9C9A99989795949392908F8EE1
:102A80008D8B8A8988878684838281807F7E7D7B07
:102A90007A797877767574737271706F6E6D6C6B0E
:102AA0006A696867666564636261605F5E5D5C5BFE
:102AB0005A5958585756555453525150504F4E4DDD
:102AC0004C4B4A4A494847464645444342424140A6
:102AD0003F3E3E3D3C3B3B3A39383837363535345E
:102AE0003332323130302F2E2E2D2C2B2B2A292908
:102AF00028272726252524232322212120201F1EA5
:102B00001E1D1C1C1B1B1A19191818171616151533
:102B100014131312121111100F0F0E0E0D0D0C0CB9
:102B20000B0A0A0909080807070606050504040335
:102B3000030202010000526573656E643A20006F63
:102B40006B0020746F6F206C6F6E672065787472F5
:102B50007573696F6E2070726576656E7465640A50
:102B60000020636F6C6420657874727573696F6E92
:102B70002070726576656E7465640A004572726FC6
:102B8000722077726974696E6720746F20454550B2
:102B9000524F4D210A0057726974696E6720746F35
:102BA0002066696C653A20006F70656E2066616909
:102BB0006C65642C2046696C653A20006F70656E08
:102BC000206661696C65642C2046696C653A20005A
:102BD00046696C652073656C65637465640A0020E2
:102BE00053697A653A200046696C65206F70656E9E
:102BF00065643A20002066696C653A2000646F695C
:102C00006E67006672657368004E6F772000454EF0
:102C10004420535542524F5554494E450A002220F4
:102C2000706F73002220706172656E743A220053D7
:102C30005542524F5554494E452043414C4C207407
:102C400061726765743A22004B494C4C45442E2012
:102C500000747279696E6720746F2063616C6C20F8
:102C60007375622D67636F64652066696C65732098
:102C70007769746820746F6F206D616E79206C6560
:102C800076656C732E204D4158206C6576656C20FE
:102C900069733A00C7DF7DE111241FBECFEFD1E297
:102CA000DEBFCDBF00E00CBF14E0A0E0B2E0E4EB7B
:102CB000FCED01E00BBF02C007900D92A831B107F7
:102CC000D9F728E1A8E1B4E001C01D92A13DB20707
:102CD000E1F716E1CBE4D6E100E006C02197010957
:102CE000802FFE010E94B2EDCA34D10780E00807B0
:102CF000A9F70E9427DA0C9449EE0C9400002F9259
:102D00003F924F925F926F927F928F929F92AF927B
:102D1000BF92CF92DF92EF92FF920F931F93CF93C8
:102D2000DF93CDB7DEB7CA58D1090FB6F894DEBF2E
:102D30000FBECDBF21E02093431080911E188D342B
:102D400011F40C947D21843511F40C94A52E873454
:102D500011F00C94F12E80911C1890911D188A315D
:102D6000910509F4BEC79CF4843091053CF482308F
:102D70009105B4F597FF2DC00C947921843091050D
:102D800009F4D2C1059709F40EC20C9479218A3254
:102D9000910511F40C9470204CF48C31910509F4D8
:102DA000A4C74D9709F4A6C70C9479218B359105DA
:102DB00011F40C94FB208C35910511F40C94FF2038
:102DC0008A35910511F00C94792110922B040C9402
:102DD000F32E8091270281110C94F82E0C94F32E7F
:102DE00020912702222311F40C94F32E11E0029774
:102DF00009F010E00E94ADAA19821A821B821C827F
:102E00001D821E821F82188682E50E949B4C8823A9
:102E100009F43AC10E941B4C4B015C0120E030E0F8
:102E2000A9010E946AE6882309F444C1C0903604CF
:102E3000D0903704E0903804F0903904CCAADDAA91
:102E4000EEAAFFAAC0903A04D0903B04E0903C0464
:102E5000F0903D04C8AED9AEEAAEFBAEC0902811EA
:102E6000D0902911E0902A11F0902B11CCAEDDAE5C
:102E7000EEAEFFAEC0902C11D0902D11E0902E112F
:102E8000F0902F112496CCAEDDAEEEAEFFAE2497BF
:102E90002CAD3DAD4EAD5FAD6CA97DA98EA99FA9AE
:102EA0000E946AE681110BC0A701960168AD79AD59
:102EB0008AAD9BAD0E946AE6882309F4FBC020E03E
:102EC00030E0A901C501B4010E946AE6881F882785
:102ED000881F181739F0C12CD12C80E8E82E8FEB11
:102EE000F82E06C0C12CD12C00E8E02E0FE3F02E06
:102EF0002C96CCAEDDAEEEAEFFAE2C972CA93DA944
:102F00004EA95FA96CAD7DAD8EAD9FAD0E94B5EAB7
:102F100028966CAF7DAF8EAF9FAF289728AD39ADA7
:102F20004AAD5BAD24966CAD7DAD8EAD9FAD249763
:102F30000E94B5EA6B017C0128962CAD3DAD4EADEB
:102F40005FAD2897CA01B9010E94CFE62B013C0171
:102F5000A7019601C701B6010E94CFE69B01AC0113
:102F6000C301B2010E94B6EA0E9421ED2B013C018F
:102F700020E030E040E05FE30E94CFE660966CAF77
:102F80007DAF8EAF9FAF6097A5019401C501B401DD
:102F90000E94CFE64B015C0160962CAD3DAD4EAD7D
:102FA0005FAD6097CA01B9010E94CFE69B01AC01F9
:102FB000C501B4010E94B5EA0E9421ED2C962CAD0A
:102FC0003DAD4EAD5FAD2C970E94CFE64B015C014D
:102FD000C701B6019058A30192010E9492EBA5018E
:102FE00094010E94CFE66B017C012CAD3DAD4EAD4E
:102FF0005FAD6CA97DA98EA99FA90E94B6EA20E0C9
:1030000030E040E05FE30E94CFE69B01AC01C701E6
:10301000B6010E94B6EA2CA93DA94EA95FA90E945B
:10302000B5EA69837A838B839C8324962CAD3DAD6E
:103030004EAD5FAD249768AD79AD8AAD9BAD0E9472
:10304000B6EA20E030E040E05FE30E94CFE66B01AB
:103050007C01A301920128966CAD7DAD8EAD9FAD34
:1030600028970E9492EBA50194010E94CFE69B0154
:10307000AC01C701B6010E94B6EA28AD39AD4AAD30
:103080005BAD0E94B5EA12C089E40E949B4C882384
:1030900031F00E941B4C69837A838B839C838AE482
:1030A0000E949B4C882331F00E941B4C6D837E83D1
:1030B0008F83988720E030E0A90169817A818B8134
:1030C0009C810E946AE681110EC020E030E0A901D7
:1030D0006D817E818F8198850E946AE6811103C08F
:1030E000EDEDFDE10DC0412FBE016F5F7F4F88E226
:1030F00091E10E94CFA40C94F32E0E94CD89F80197
:1031000084918F010F5F1F4F8111F7CFEDE1F2E046
:1031100084918F010F5F1F4F882311F40C94F32EBD
:103120000E94CD89F801F4CF80E50E949B4C882352
:1031300079F08091250490912604009749F04AE0A7
:1031400050E060E070E00E94E9E46B017C0103C0A4
:10315000C12CD12C760183E50E949B4C882361F021
:103160000E941B4C20E030E04AE754E40E94CFE686
:103170000E94FFEB6B017C010E94226A0E940259AF
:10318000C60ED71EE81EF91E0E940259DC01CB01B3
:103190008C199D09AE09BF09B7FD02C00C94F32E2E
:1031A0000E9403A1F1CF80912702882311F40C948F
:1031B000F32E0E94ADAA89E40E949B4C882329F03B
:1031C0000E941B4C2B013C0103C0412C512C3201AD
:1031D0008AE40E949B4C882329F00E941B4C4B01DF
:1031E0005C0103C0812C912C540180E50E949B4C12
:1031F000882329F00E941B4C6B017C0103C0C12C69
:10320000D12C760181E50E949B4C882339F00E94E5
:103210001B4C6CAB7DAB8EAB9FAB04C01CAA1DAA34
:103220001EAA1FAA20914210C657DF4F2883CA58F2
:10323000D0406091020270910302072E000C880BAF
:10324000990B0E9470E6209136023091370240912E
:103250003802509139020E94CFE62AE037ED43E26E
:103260005CE30E94CFE668AB79AB8AAB9BAB409145
:10327000360450913704609138047091390448AF96
:1032800059AF6AAF7BAF9A01AB01C301B2010E9493
:10329000B6EAA1966CAF7DAF8EAF9FAFA19740907D
:1032A0003A0450903B0460903C0470903D04A301AC
:1032B0009201C501B4010E94B6EAA5966CAF7DAF3C
:1032C0008EAF9FAFA5972091281130912911409181
:1032D0002A1150912B11C701B6010E94B6EAA99696
:1032E0006CAF7DAF8EAF9FAFA99720912C1130911D
:1032F0002D1140912E1150912F116CA97DA98EA9ED
:103300009FA90E94B6EAAD966CAF7DAF8EAF9FAF1E
:10331000AD97C8ACD9ACEAACFBACC982DA82EB821F
:10332000FC824D825E826F8278860E9402599B01E8
:10333000AC0128533F4F4F4F5F4FCB57DF4F288390
:1033400039834A835B83C558D040BDEC8B2EBCECDF
:103350009B2EA92CBDE3BB2E25961FAE2597299643
:103360001FAE29972D961FAE2D9761961FAE6197C0
:103370000E94D07B0E9402598B019C01CB57DF4FEA
:10338000C880D980EA80FB80C558D0400C191D093F
:103390002E093F0937FD10C09B01AC0128533F4F58
:1033A0004F4F5F4FCB57DF4F288339834A835B836F
:1033B000C558D0400E9403A125967FAD2597299638
:1033C0006FAD29972D969FAD2D9761968FAD619723
:1033D000272F362F492F582FC501B4010E94B6EA76
:1033E0006CAB78AF8CAF21969FAF219720E030E097
:1033F00040E85FE30E94DCEC181644F41CAA18AE07
:1034000030E83CAF4FE321964FAF219760912811F0
:103410007091291180912A1190912B11E1966CAF36
:103420007DAF8EAF9FAFE1978091360490913704C6
:10343000A0913804B0913904E5968CAF9DAFAEAF42
:10344000BFAFE59721969FAD21979F93ACADAF930A
:10345000B8ADBF93ECA9EF93E196ACACBDACCEACEC
:10346000DFACE197A996ECACFDAC0EAD1FADA99712
:10347000A1962CAD3DAD4EAD5FADA197E5966CAD7F
:103480007DAD8EAD9FADE5970E94B5C50F900F90B5
:103490000F900F9062966FAF629763967FAF6397BE
:1034A00064968FAF649765969FAF6597C0902C1117
:1034B000D0902D11E0902E11F0902F11E996CCAE06
:1034C000DDAEEEAEFFAEE99720913A0430913B04B9
:1034D00040913C0450913D04ED962CAF3DAF4EAF72
:1034E0005FAFED9721963FAD21973F934CAD4F9342
:1034F00058AD5F936CA96F93E996ACACBDACCEAC04
:10350000DFACE997AD96ECACFDAC0EAD1FADAD9761
:10351000A5962CAD3DAD4EAD5FADA597ED966CADCE
:103520007DAD8EAD9FADED970E94B5C50F900F900C
:103530000F900F9066966FAF669767967FAF67970D
:1035400068968FAF689769969FAF699789819A81CE
:10355000AB81BC81C358DF4F88839983AA83BB8327
:10356000CD57D040CD80DE80EF80F884CF57DF4F3D
:10357000C882D982EA82FB82C158D0406A961FAEC7
:103580006A9725967FAD259729966FAD29972D9639
:103590009FAD2D9761968FAD6197272F362F492FBD
:1035A000582FBCA9A8ADFCAD2196EFAD21976B2F8C
:1035B0007A2F8F2F9E2F0E94B5EA2FE632E143E04B
:1035C0005BE30E946AE687FD29C125967FAD2597BA
:1035D00029966FAD29972D969FAD2D9761968FAD4A
:1035E0006197272F362F492F582FBCA9A8ADFCADC6
:1035F0002196EFAD21976B2F7A2F8F2F9E2F0E9450
:10360000B6EA20E030E040E05FE30E94CFE6662EBD
:10361000972E882E792E9F938F937F936F93E196A9
:10362000ACACBDACCEACDFACE197A996ECACFDACDC
:103630000EAD1FADA997A1962CAD3DAD4EAD5FADC2
:10364000A197E5966CAD7DAD8EAD9FADE5970E94DF
:10365000B5C50F900F900F900F906B966FAF6B9753
:103660006C967FAF6C976D968FAF6D97C757DF4F96
:103670009883C958D0407F928F929F926F92E9961B
:10368000ACACBDACCEACDFACE997AD96ECACFDAC70
:103690000EAD1FADAD97A5962CAD3DAD4EAD5FAD5A
:1036A000A597ED966CAD7DAD8EAD9FADED970E946B
:1036B000B5C50F900F900F900F90162F072FB82EB3
:1036C000A92E66962FAD669767963FAD6797689669
:1036D0004FAD689769965FAD6997CF57DF4F6881A7
:1036E00079818A819B81C158D0400E94B6EA20E04E
:1036F00030E040E05FE30E94CFE61B012C016296C0
:103700002FAD629763963FAD639764964FAD649714
:1037100065965FAD6597C358DF4F688179818A816F
:103720009B81CD57D0400E94B6EA20E030E040E0D7
:103730005FE30E94CFE69B01AC016B966FAD6B9788
:103740006C967FAD6C976D968FAD6D97C757DF4FB9
:103750009881C958D0400E94B5EA6B017C0120E0F5
:1037600030E0A9010E94DCEC87FF04C0F7FAF09476
:10377000F7F8F094A2019101612F702F8B2D9A2DF3
:103780000E94B5EA1B012C0120E030E0A9010E9453
:10379000DCEC87FF04C057FA509457F85094A2010C
:1037A0009101C701B6010E94B6EA2DEC3CEC4CEC4D
:1037B0005DE30E946AE618168CF566961FAF669761
:1037C00067960FAF67976896BFAE68976996AFAE7A
:1037D00069976B96DFAC6B976296DFAE62976C96DB
:1037E000EFAC6C976396EFAE63976D96FFAC6D97F9
:1037F0006496FFAE6497C757DF4F2881C958D04001
:1038000065962FAF65976CAA98AE8CAE21967FAE69
:10381000219731E06A963FAF6A97B3CE6A964FAD73
:103820006A97411144C125967FAD259729966FADC2
:1038300029972D969FAD2D9761968FAD6197272F74
:10384000362F492F582FBCA9A8ADFCAD2196EFAD5E
:1038500021976B2F7A2F8F2F9E2F0E94B5EA6B0135
:103860007C012DEC3CEC4CEC5DE30E94DCEC18168A
:103870000CF41DC1A7019601C701B6010E94B6EA6A
:103880002596EFAD25972996BFAD29972D96AFAD1B
:103890002D976196FFAD61972E2F3B2F4A2F5F2FFB
:1038A0000E94B6EA662E972E882E792E20E030E010
:1038B00040E85FE30E94DCEC87FFF9C07F928F92C3
:1038C0009F926F92E196ACACBDACCEACDFACE19711
:1038D000A996ECACFDAC0EAD1FADA997A1962CAD91
:1038E0003DAD4EAD5FADA197E5966CAD7DAD8EADB6
:1038F0009FADE5970E94B5C50F900F900F900F9068
:103900006A966FAF6A976B967FAF6B976C968FAF27
:103910006C976D969FAF6D977F928F929F926F92EB
:10392000E996ACACBDACCEACDFACE997AD96ECACF7
:10393000FDAC0EAD1FADAD97A5962CAD3DAD4EAD1A
:103940005FADA597ED966CAD7DAD8EAD9FADED975E
:103950000E94B5C50F900F900F900F90162F072F54
:10396000B82EA92E262F372F482F592FCF57DF4F8C
:10397000688179818A819B81C158D0400E94B6EAD2
:1039800020E030E040E05FE30E94CFE66B017C0185
:103990006A962FAD6A976B963FAD6B976C964FAD5D
:1039A0006C976D965FAD6D97C358DF4F68817981D5
:1039B0008A819B81CD57D0400E94B6EA20E030E05A
:1039C00040E05FE30E94CFE69B01AC0162966FADE1
:1039D000629763967FAD639764968FAD64976596A3
:1039E0009FAD65970E94B5EA1B012C0120E030E0F5
:1039F000A9010E94DCEC87FF04C057FA509457F8E5
:103A00005094A701960166966FAD669767967FAD55
:103A1000679768968FAD689769969FAD69970E9482
:103A2000B5EA6B017C0120E030E0A9010E94DCECEA
:103A300087FF04C0F7FAF094F7F8F094A20191011F
:103A4000C701B6010E94B6EA2DEC3CEC4CEC5DE3FC
:103A50000E94DCEC18165CF166961FAF66976796BD
:103A60000FAF67976896BFAE68976996AFAE6997D4
:103A70006A965FAD6A9762965FAF62976B966FAD1D
:103A80006B9763966FAF63976C967FAD6C976496F8
:103A90007FAF64976D968FAD6D9765968FAF659785
:103AA0006CAA98AE8CAE21967FAE2197BCCE25969F
:103AB0007FAD259729966FAD29972D969FAD2D97B0
:103AC00061968FAD6197272F362F492F582FBCA9AC
:103AD000A8ADFCAD2196EFAD21976B2F7A2F8F2FDC
:103AE0009E2F0E94B5EA4B015C0162968FAD6297F2
:103AF00063969FAD63976496AFAD64976596BFADCF
:103B0000659789839A83AB83BC8366968FAD6697EE
:103B100067969FAD67976896AFAD68976996BFAD9A
:103B200069978D839E83AF83B8877CA968AD9CAD70
:103B300021968FAD2197272F362F492F582F60E0E0
:103B400070E080E89FE30E94B5EA6B017C01209160
:103B50003E0430913F0440914004509141040E9442
:103B6000CFE62B013C012091301130913111409171
:103B7000321150913311BCA9A8ADFCAD2196EFAD27
:103B800021976B2F7A2F8F2F9E2F0E94CFE69B01BC
:103B9000AC01C301B2010E94B6EA69877A878B87BC
:103BA0009C872091420430914304409144045091F9
:103BB0004504C701B6010E94CFE66B017C0120914C
:103BC0003411309135114091361150913711BCA903
:103BD000A8ADFCAD2196EFAD21976B2F7A2F8F2FDB
:103BE0009E2F0E94CFE69B01AC01C701B6010E9447
:103BF000B6EA6D877E878F87988BCE0101960E94EB
:103C0000F2C91CA61DA61EA61FA689819A81AB819A
:103C1000BC8188A399A3AAA3BBA38D819E81AF81F8
:103C2000B8858CA39DA3AEA3BFA389859A85AB85D8
:103C3000BC8588A799A7AAA7BBA7AE01485D5F4F1F
:103C4000BE016C5D7F4FCE0180960E943BB6DE01C7
:103C50009C966D01C657DF4FE880CA58D0408E0150
:103C6000005D1F4F9E01235F3F4FAE01485D5F4FD8
:103C7000BE016C5D7F4FCE0180960E94FE59882365
:103C800029F120E030E040E85FE3BCA9A8ADFCAD3D
:103C90002196EFAD21976B2F7A2F8F2F9E2F0E94A9
:103CA0006AE687FF13C03CA925963FAF259748AD2C
:103CB00029964FAF29975CAD2D965FAF2D97219632
:103CC0006FAD219761966FAF619752CB80E1E8E2CB
:103CD000F1E1A6E3B4E001900D928A95E1F70C942E
:103CE000F32E0E94384E0C94F32E80E00E944DACCF
:103CF0000C94F32E83E50E949B4C882321F10E94B3
:103D0000FB4B182F863070F0E5EEF2E084918F01C6
:103D10000F5F1F4F882311F40C94F32E0E94CD895E
:103D2000F801F4CF833009F44AC130F4813091F1C5
:103D3000823009F43FC008C0843009F49FC1853047
:103D400009F4ACC101C010E00E9400AC811103C0B5
:103D5000E5ECF2E013C08091F610882319F063E1DE
:103D600073E002C067E173E08DEB92E00E949AC5B8
:103D70008AE00E94CD890E9475B696C184917F0128
:103D8000BFEFEB1AFB0A882309F48EC10E94CD898C
:103D9000F701F4CF0E9428B710920102109200029E
:103DA00082EB92E09093A8078093A7070E94F9897D
:103DB0000C94F32E809100029091010297FF0EC0A7
:103DC000E9E8F2E084918F010F5F1F4F882311F41F
:103DD0000C94F32E0E94CD89F801F4CF0097A1F442
:103DE0008091520280932C0419821A821B821C82B9
:103DF00018A219A21AA21BA2BE016F5F7F4FCE01AB
:103E000080960E94AFBB27C0815065E00E947EED86
:103E100080FF03C024E0291B922F25E09202F001CD
:103E20001124E80FF11D87FDFA95EE0FFF1FEE0F2D
:103E3000FF1FE758FF4E80913E0490913F04A091F0
:103E40004004B091410480839183A283B383809125
:103E50002C048093520280910002909101028931DA
:103E600091050CF067C0109252029C012F5F3F4FEA
:103E7000309301022093000265E00E947EED80FFF6
:103E800003C024E0291B922F40913E0450913F042F
:103E9000609140047091410448A359A36AA37BA395
:103EA00019821A821B821C8244E084029001112430
:103EB000B9016351764F4B01DB012D913D914D913D
:103EC0005C91B4E09B02C0011124FC01EF5FF54F4F
:103ED0005F016081718182819381DE0111966D01A4
:103EE000E12CF12C00EA10E40E94DFBA19821A8258
:103EF0001B821C82B601CE0180960E94AFBBF501E9
:103F000080819181A281B38180933604909337049C
:103F1000A0933804B0933904F40180819181A28187
:103F2000B38180933A0490933B04A0933C04B093F4
:103F30003D04BCC080E090E0A0EAB0E480933E0481
:103F400090933F04A0934004B09341040E9441AD7C
:103F50000E94226A8FEF9FEF9093010280930002EC
:103F6000E5E7F2E084918F010F5F1F4F882321F076
:103F70000E94CD89F801F6CF83E992E09A83898384
:103F800004E610E019A308A3BE016F5F7F4FCE01C6
:103F900080960E94CABC8AEB92E09A83898319A317
:103FA00008A3BE016F5F7F4FCE0180960E94CABCFE
:103FB00081E00E944DAC81E00E942DAC77C088E585
:103FC0000E949B4C8823A1F00E94EB4B1FEF160F21
:103FD0001530A8F0EEE5F2E084918F010F5F1F4FDE
:103FE000882311F40C94F32E0E94CD89F801F4CFAC
:103FF00088E50E94CD890E94B9E10C94F32E89E5F1
:104000000E949B4C8823A1F00E94EB4B0FEF060F00
:104010000530A8F0E7E4F2E084918F010F5F1F4FB5
:10402000882311F40C94F32E0E94CD89F801F4CF6B
:1040300089E50E94CD890E94B9E10C94F32E8AE5AE
:104040000E949B4C882399F00E941B4C25E0129FF4
:10405000F0011124E00FF11DEE0FFF1FEE0FFF1F07
:10406000E758FF4E608371838283938335C08AE56E
:104070000E94CD890E94B9E10C94F32E8AE50E943A
:104080009B4C8823A1F30E941B4C60937510709386
:10409000761080937710909378101EC080E00E9475
:1040A0002DAC0E9428B718C01230B1F46091000204
:1040B000709101026931710514F069E170E088E3E3
:1040C00092E00E9481C569E170E083E392E00E9482
:1040D00081C58AE00E94CD890E944C950C94F32EF4
:1040E00080912702882311F40C94F32E89E40E9416
:1040F0009B4CE82E882321F00E94EB4B062F01C039
:1041000000E08AE40E949B4CF82E882321F00E9454
:10411000EB4B162F01C010E0EE2011F0053020F41B
:10412000FF2081F0153070F0ECEFF2E084918F0108
:104130000F5F1F4F882311F40C94F32E0E94CD893A
:10414000F801F4CF0E94A74CEE2091F034E0030276
:10415000F0011124EF5FF54F80819181A281B3813D
:104160008093281190932911A0932A11B0932B11B9
:10417000FF2091F044E01402F0011124E351F64FC6
:1041800080819181A281B38180932C1190932D1114
:10419000A0932E11B0932F1180E50E949B4C882391
:1041A00019F00E940C4C03C080E50E94524C86E43A
:1041B0000E949B4C8823D9F00E941B4C6B017C0110
:1041C00020E030E0A9010E94DCEC181684F420E025
:1041D00030E040E752E4C701B6010E9492EB6093E1
:1041E00036027093370280933802909339020E940E
:1041F00089CA0C94F32E20932B040C94F32E97E58C
:10420000292E92E0392E21E5E22E20E1F22E66E3FE
:1042100074E07DAB6CAB38E1C32E34E0D32E00E00C
:1042200010E0D1018D911D010E949B4C882309F45F
:104230004BC00E941B4C2B013C01133049F0F6018E
:1042400020813181428153810E94B5EA2B013C01DA
:10425000ACA9BDA92D913D914D915C91C301B201D5
:104260000E94B5EA4B015C012DEB37E346E855EBC4
:104270000E94DCEC87FD0AC02DEB37E346E855E3EE
:10428000C501B4010E946AE61816F4F4133051F423
:104290004092420450924304609244047092450458
:1042A00001E012C0A5019401F70160817181828152
:1042B00093810E94B6EAD7016D937D938D939C9371
:1042C0001397812F0E9498AD1F5FB4E0EB0EF11C95
:1042D000ECA9FDA93496FDABECABF4E0CF0ED11CFC
:1042E000143009F09ECF002309F4F6CE0E947BBA69
:1042F000F3CE0E94FEBC0C94F32E80911C1890917A
:104300001D188537910511F40C94F32E0CF0C0C0E4
:104310008C34910509F43CC40CF058C08A319105E5
:1043200009F42EC224F58531910509F4E7C184F41E
:104330008231910509F4A9C58431910509F49EC122
:10434000419711F00C94A22E0E94C4A40C94F32E59
:104350008731910509F4DCC10CF4D4C18831910591
:1043600009F4ECC1499709F4F4C10C94A22E8F31E1
:10437000910509F401C39CF48C31910509F4A6C29E
:104380000CF40CC28D31910511F40C94F32E4E9760
:1043900011F00C94A22E0E9417B00C94F32E8A32C6
:1043A000910509F49CC32CF4809709F499C20C94EC
:1043B000A22E8133910509F4C6C38B34910511F007
:1043C0000C94A22E0E94C7780C94F32E8A36910585
:1043D00009F40AC5B4F58435910509F456C5E4F429
:1043E0008135910509F42CC54CF48D34910511F0FB
:1043F0000C94A22E0E94FE780C94F32E8235910527
:1044000009F440C58335910511F00C94A22E81E08A
:1044100080932A040C94F32E8C35910509F47BC506
:1044200034F48535910509F45DC50C94A22E8836C7
:10443000910509F4B1C38936910509F475C40C944A
:10444000A22E8F36910509F4E3C384F48C369105CE
:1044500009F431C40CF4E4C48D36910509F4A6C402
:104460008E36910509F4C1C30C94A22E81379105B3
:1044700009F42DC40CF423C48237910509F4D3C583
:104480008337910511F00C94A22EE3EEF4E008C6F8
:104490008E3221E0920711F40C94DE2C0CF071C0E6
:1044A0008B3C910509F416C7CCF58C38910509F4BD
:1044B00081C4ACF48737910509F49AC60CF44BC655
:1044C0008837910509F497C68937910511F00C9446
:1044D000A22E10923B0510923A050C94F32E8E3BBF
:1044E000910509F47DC434F48B39910509F437C47E
:1044F0000C94A22E883C910509F483C6893C910551
:1045000011F00C94A22EF7E5EF2EF2E0FF2E08E555
:1045100011E1A8E6CA2EA1E1DA2EC3C68C3D9105B1
:1045200011F40C94712B9CF48D3C910509F463C734
:104530000CF4ECC68E3C910509F4EAC7833D910565
:1045400011F00C94A22E0E9438940C94F32E823E0B
:10455000910511F40C94EC2B3CF48D3D910511F474
:104560000C947E2B0C94A22E8C3241E0940711F413
:104570000C94152C8D32914011F40C943E2C0C941B
:10458000A22E853F61E0960711F40C94CB2DDCF54B
:104590008A39A1E09A0709F496C3BCF48033E1E0BC
:1045A0009E0711F40C94352D14F40C94322D83369F
:1045B00021E0920709F45EC08039914011F00C941B
:1045C000A22E0E94226A0C94F32E853A41E09407B1
:1045D00011F40C94C82D4CF4843A914011F00C94D1
:1045E000A22E0E9416960C94F32E8C3A71E0970737
:1045F00009F4B1C7843F914011F00C94A22E0E949F
:1046000069700C94F32E8A39B2E09B0711F40C9474
:104610000A2EB4F4873FF1E09F0711F40C94D12DDA
:1046200014F40C94CE2D883F31E0930711F40C94D0
:10463000DD2D8C30924011F40C94012E0C94A22E9E
:104640008B3853E0950711F40C94F32E3CF4843826
:10465000934011F40C94372E0C94A22E803AA3E0D0
:104660009A0709F47CC1873E934011F40C948F2E75
:104670000C94A22EEDEDFDE10C94B52DEAE2F3E0F1
:1046800084918F010F5F1F4F882321F00E94CD89F5
:10469000F801F6CF1092B30C86E69AE00E943D9A9C
:1046A0008BE1E6E6FAE0DE01159601900D928A951F
:1046B000E1F78091640A9091650A9C838B838DEE6B
:1046C00092E09A83898340E050E0BE016F5F7F4FA4
:1046D00080E090E00E94EA82CE0101960E9499A0BB
:1046E000EBE1F3E084918F010F5F1F4F882311F4FA
:1046F0000C94F32E0E94CD89F801F4CF0E94BC8067
:104700000C94F32E1092350A1092360A0C94F32E64
:10471000E0911A18F0911B188081882329F08032CB
:1047200009F410823196F8CF40E061E080911A18C8
:1047300090911B180E94B8D50C94F32E8091360AE4
:10474000882319F081E08093350A0E94C7780C9481
:10475000F32E1092350A80912F07813011F00C94BE
:10476000F32E82E080932F070E94025960932B075B
:1047700070932C0780932D0790932E070C94F32EA3
:104780008091360A882311F40C94F32E83E50E945D
:104790009B4C81110C94FD2E0C94F32E83E40E940B
:1047A000524C882309F450C0E8E6F3E084918F016D
:1047B0000F5F1F4F882321F00E94CD89F801F6CFAB
:1047C0008091010C811103C0EBE3F3E012C0BE0144
:1047D0006F5F7F4F8EEF9BE00E9405998E010F5F08
:1047E0001F4FF80181918F01882349F10E94CD89E3
:1047F000F8CF84918F010F5F1F4F882301F10E9432
:10480000CD89F801F6CF06EDC02E03E0D02EE12CC5
:10481000F12C20E08091140790E00E2C02C09595B9
:1048200087950A94E2F780FD23C2BFEFEB1AFB0ADB
:10483000E2E0CE0ED11CF5E0EF16F10459F78AE064
:104840000E94CD890C94F32E8091360A882339F08A
:104850008091350A882319F0E5E4F3E003C0E7E529
:10486000F3E028C084918F010F5F1F4F882321F050
:104870000E94CD89F801F6CF6091AF0C7091B00C19
:104880008091B10C9091B20C4AE00E94F08C8FE2C2
:104890000E94CD896091AB0C7091AC0C8091AD0CF5
:1048A0009091AE0C4AE00E94F08C8AE00E94CD8983
:1048B0000C94F32E84918F010F5F1F4F882311F406
:1048C0000C94F32E0E94CD89F801F4CF40E060E013
:1048D00080911A1890911B180E94B8D50C94F32E51
:1048E0008091350A81110E94226A8091360A8823BC
:1048F00011F40C94F32E80E50E949B4C882319F050
:104900000E940C4C03C080E50E94524C182F482F87
:1049100061E080911A1890911B180E94B8D583E528
:104920000E949B4C882381F00E94EB4BAB01BC01A1
:104930004093AF0C5093B00C6093B10C7093B20CD9
:104940008EEF9BE00E94F6978091360A882319F03B
:1049500081E08093350A11110C94F32EF6CE8091EC
:104960001A1890911B1821E02093340A40E060E06F
:104970000E94B8D50C94F32E0E9478787B018C01AC
:1049800020E831E541E050E00E9458EAC9016DE6B7
:1049900071E00E948BED4B015C01C801B70120E181
:1049A0003EE040E050E00E9458EACA01B90128E127
:1049B00030E040E050E00E9458EA762E672EC62E86
:1049C000D72E8CE3282E312C412C512CC801B70155
:1049D000A20191010E9458EAF62EE72ECA01B90100
:1049E000A20191010E9458EACB018E010F5F1F4F77
:1049F00081149104D1F0EF92FF927F936F936F92A5
:104A00007F92BF92AF929F928F928FE993E09F9394
:104A10008F931F930F930E943CE60FB6F894DEBF6E
:104A20000FBECDBFE2EFFDE145C0A114B10489F096
:104A3000EF92FF927F936F936F927F92BF92AF92AC
:104A40008FE893E09F938F931F930F930E943CE610
:104A5000E4CFCD2879F0EF92FF927F936F936F921E
:104A60007F9283E893E09F938F931F930F930E940D
:104A70003CE6D3CF892B69F0EF92FF927F936F933F
:104A80008BE793E09F938F931F930F930E943CE6D5
:104A9000C4CFEF92FF9287E793E09F938F931F938A
:104AA0000F930E943CE60F900F900F900F900F9085
:104AB0000F90B8CF84917F019FEFE91AF90A8823FC
:104AC00021F00E94CD89F701F5CFB80183EB93E087
:104AD0000E949AC58AE00E94CD890C94F32E83E54A
:104AE0000E949B4C882311F40C94F32E0E94FB4BE4
:104AF000E82E80E50E949B4C882339F00E94FB4BF6
:104B0000182F87FF03C00C94F32E1DE089E40E9448
:104B10009B4C882341F00E940C4C81110C94792FFE
:104B2000EBE1F6E00BC089E40E94524CF6CF3196DF
:104B3000A6E0EB34FA0711F40C94792F8491181342
:104B4000F6CF0C944E2FF090240481E0F826F092DA
:104B50002404EBECF3E084918F010F5F1F4F882357
:104B600021F00E94CD89F801F6CFFF2019F0E0EC8A
:104B7000F3E002C0E5ECF3E084918F010F5F1F4F7B
:104B8000882311F40C94F32E0E94CD89F801F4CF00
:104B90000E94E9780C94F32E88E690E00E94D8AD4C
:104BA00081110C94F32E8091140783FF02C00C94A2
:104BB000F32E83E50E949B4C882399F00E941B4CA6
:104BC0000E94FAEBCB010E94F7590E941B4C20E097
:104BD00030E04AEA52E40E946AE6181614F00E9495
:104BE000FE780E94C4C70C94F32E8EE40E949B4C66
:104BF000882311F40C94F32E0E94EB4B6093C7189A
:104C00007093C8188093C9189093CA180C94F32E07
:104C100083E50E94524C882359F083E50E949B4C07
:104C2000882319F00E94FB4B01C080E08093140799
:104C3000E2EFFDE184918F010F5F1F4F811103C0EF
:104C4000E4EEF3E004C00E94CD89F801F3CF849133
:104C50008F010F5F1F4F882321F00E94CD89F8013B
:104C6000F6CF809114078111CECDE0EEF3E018C0AD
:104C7000BB24B394B20E222319F08CE20E94CD899A
:104C8000F60185919491FC0184918F010F5F1F4F74
:104C9000882321F00E94CD89F801F6CF2B2DC5CDB8
:104CA00084918F010F5F1F4F882309F4C8CD0E94A4
:104CB000CD89F801F5CF109220020C94F32E8BEEE3
:104CC00093E00E94BCA00E94CD8E0C94F32E83E54D
:104CD0000E949B4C811103C0E2EFFDE10DC00E94D8
:104CE000FB4B8D3320F480932B020C94F32E8CE33A
:104CF00080932B020C94F32E84918F010F5F1F4F32
:104D0000882321F00E94CD89F801F6CF40912B0233
:104D100050E060E070E084EF93E00E9447C58AE0D5
:104D20000E94CD890C94F32E89E690E00E94D8ADC4
:104D3000811111C0EBEFF3E084918F010F5F1F4FE2
:104D4000882321F00E94CD89F801F6CF0E940076D9
:104D50008AE00E94CD89109243100C948E2F83E537
:104D60000E949B4C882311F40C94F32E0E94FB4B61
:104D7000182F8D3308F01CE3109350100E94025935
:104D80006B017C01212F30E0A8EEB3E00E94A6EA7F
:104D9000C60ED71EE81EF91EC0924C10D0924D10C0
:104DA000E0924E10F0924F100C94F32E0E941AAE27
:104DB0000C94F32E8091140783FF02C00C94F32E01
:104DC00083E50E949B4C882311F40C94F32E0E94DF
:104DD0001B4C0E94FAEBCB010E942A4E0C94F32E3E
:104DE0000E94DDA80C94F32E80E50E949B4C81115B
:104DF00006C083E50E949B4C882359F005C00E94A1
:104E0000FB4B8111F0C7F5CF0E94EB4B6F3F710553
:104E100010F06FEF70E07093470460934604E3C7AF
:104E200080E50E949B4C811105C0109247041092AE
:104E30004604D9C70E94EB4B672B09F0D4C7F5CFC6
:104E40000E9413790E941DB11092470410924604EB
:104E500000E010E062E370E080E090E00E9474BE49
:104E60000E94D07B0F5F1F4F0331110599F762E35A
:104E700070E080E090E00E9474BE0E94D07B0E94AF
:104E8000A82FB1C710922A04AEC783E50E949B4C9D
:104E9000882399F00E941B4C20E030E04AE754E45C
:104EA0000E94CFE60E94FFEB60932C0270932D02CC
:104EB00080932E0290932F0296C788E50E94524C51
:104EC0008111ACC789E50E94524C8111A7C78AE5C0
:104ED0000E94524C8111A2C785E40E94524C81115C
:104EE0009DC7CEC783E50E94524C882309F47BC737
:104EF0000E941B4C20E030E04AE754E40E94CFE6D9
:104F00000E94FFEB609348107093491080934A1001
:104F100090934B1068C7B7E5CB2EB2E0DB2E1CE0B8
:104F2000E12E11E1F12E10E0D6018D916D010E946C
:104F3000524C882309F46DC0133009F063C00E94FD
:104F40001B4C4B015C0120E030E040EA51E40E9440
:104F50006AE687FF4EC0A501940160911811709117
:104F6000191180911A1190911B110E9492EB2B0143
:104F70003C019B01AC016091E3067091E4068091D5
:104F8000E5069091E6060E94CFE66093E3067093F3
:104F9000E4068093E5069093E606A30192016091F2
:104FA00003077091040780910507909106070E94FE
:104FB000CFE66093030770930407809305079093EF
:104FC000060760915411709155118091561190917E
:104FD00057110E946EE6A30192010E94CFE60E9443
:104FE000FFEB609354117093551180935611909379
:104FF00057118092181190921911A0921A11B09223
:105000001B1107C00E941B4CF701608371838283D0
:1050100093831F5FF4E0EF0EF11C143009F084CF8E
:105020000E9465C9E0C60E94226A83E50E949B4CEB
:10503000882309F451C80E94EB4B6230710509F0D6
:105040004BC80E94D6C98BE50E94CD896091AD18EE
:105050007091AE188091AF189091B01842E00E9404
:10506000758D4091B1185091B2186091B31870913C
:10507000B41881E094E00E9464C54091B518509145
:10508000B6186091B7187091B8188EEF93E00E942F
:1050900064C58DE50E94CD898AE00E94CD89A3C6B2
:1050A00084918F010F5F1F4F882321F00E94CD89CB
:1050B000F801F6CF60E083ED94E00E94169561E080
:1050C0008CEC94E00E94169561E081EC94E00E94E3
:1050D000169561E081EB94E00E94169560E088EA05
:1050E00094E00E94169561E08EE994E00E94169586
:1050F00060E084E994E00E94169560E08CE894E01A
:105100000E94169561E08EE794E00E94169560E09B
:1051100080E794E00E94169560E081E694E00E94AA
:10512000169560E083E594E00E94169560E08DE3BB
:1051300094E00E94169560E08CE294E00E9416953F
:1051400060E087E194E00E94169561E084E094E0DD
:105150000E94169548C600911A1810911B1883E0FA
:10516000D12C40E08150E9F0D8019C91292F2B7F70
:105170002134C1F711962C912133A1F7913421F0FC
:10518000953421F441E002C0DD24D39498012E5FD0
:105190003F4F89012F5F3F4FF80190819032C9F353
:1051A000E1CF442369F0E2EFFDE184917F012FEF2D
:1051B000E21AF20A882321F00E94CD89F701F5CF87
:1051C000DD2069F0E9EAF5E084917F013FEFE31A21
:1051D000F30A882321F00E94CD89F701F5CFD80189
:1051E0008D918D01882309F42ACB0E94CD89F7CFB8
:1051F0000E94E7B7F8C581E080933B0580933A05AC
:10520000F2C588EC90E00E94D8AD8111ECC584E431
:105210000E94524C882309F441C00E941B4C6B0130
:105220007C0111E020E030E0A9010E946AE68111D2
:1052300001C010E01093DD1020E030E0A901C701AB
:10524000B6010E946AE6882349F10E941B4CE09156
:105250005207B4E0EB9FF0011124EE51FF4E608342
:1052600071838283938320E030E0A9016091E21092
:105270007091E3108091E4109091E5100E946AE62D
:1052800081110CC080E090E0A0EEBFE38093E210BB
:105290009093E310A093E410B093E5100E945BB1EB
:1052A000A2C5F70181917F010E94524C882351F0E1
:1052B0000E941B4C0E94FFEBD8016D937D938D9350
:1052C0009C9313970C5F1F4FC016D10651F70E9495
:1052D000F4C789C5E7E5EE2EE2E0FE2E07EF16E003
:1052E000F70181917F010E94524C882341F00E9476
:1052F0001B4CD8016D937D938D939C9313970C5FFA
:105300001F4FB7E007301B0759F76DC583E50E94B3
:105310009B4C8823A1F00E941B4C6093EF06709376
:10532000F0068093F1069093F2066093EB0670937B
:10533000EC068093ED069093EE0610E001C011E0BC
:1053400080E50E949B4C882359F00E941B4C60937F
:10535000EF067093F0068093F1069093F20610E04A
:1053600082E50E949B4C882359F00E941B4C60935D
:10537000F3067093F4068093F5069093F60610E01A
:1053800084E50E949B4C882359F00E941B4C60933B
:10539000EB067093EC068093ED069093EE0623C522
:1053A000112309F420C54091EF065091F006609159
:1053B000F1067091F20683EB95E00E9464C540917E
:1053C000F3065091F4066091F5067091F60680EBB5
:1053D00095E00E9464C54091EB065091EC06609107
:1053E000ED067091EE068DEA95E00E9464C58AE0B4
:1053F0000E94CD89F8C481E50E94524C8823C1F0F7
:105400008091250490912604009739F04AE050E0FD
:1054100060E070E00E94E9E403C060E070E0CB016E
:1054200060930707709308078093090790930A0712
:1054300083E50E94524C882351F00E941B4C6093DC
:105440000F0770931007809311079093120784E55C
:105450000E94524C882351F00E941B4C60930B0712
:1054600070930C0780930D0790930E0788E50E94B8
:10547000524C882351F00E941B4C6093D7067093C6
:10548000D8068093D9069093DA0689E50E94524C9B
:10549000882351F00E941B4C6093DB067093DC065E
:1054A0008093DD069093DE068AE50E94524C8823A5
:1054B000F1F00E941B4C6093DF067093E00680932E
:1054C000E1069093E2062DEC3CEC4CEC5DE30E948F
:1054D0006AE6181664F0E3ECF5E084918F010F5F43
:1054E0001F4F882321F00E94CD89F801F6CF85E473
:1054F0000E94524C882309F476C40E941B4C60938E
:10550000E3067093E4068093E5069093E6066BC489
:1055100067E5C62E62E0D62E7CE3E72E75E0F72E17
:1055200010E0F60181916F010E94524C882359F0DE
:105530000E941B4CD7016D937D938D939C93139781
:10554000812F0E9498AD1F5FB4E0EB0EF11C133069
:1055500041F70C946C200E94CDBB811144C407E03C
:1055600013E2E6E3F4E0FDABECAB9E012F5F3F4FAF
:10557000590150E5852E53E2952E1901F8016591E8
:10558000759185919491ACA9BDA9CD90DD90ED90D8
:10559000FD90BDABACABA70196010E94B5EA2B0113
:1055A0003C01F101608371838283938320E030E0CA
:1055B00040EA51EC0E94DCEC87FD0AC020E030E0BC
:1055C00040EA51E4C301B2010E946AE618162CF4C5
:1055D000F401849118160CF456C4D101CD90DD90DD
:1055E000ED90FD901D0120E030E040EA51ECC70154
:1055F000B6010E94DCEC87FD0AC020E030E040EA02
:1056000051E4C701B6010E946AE618164CF5EDEDAB
:10561000FDE184918F010F5F1F4F811103C0E5EF02
:10562000F5E004C00E94CD89F801F3CF84918F0189
:105630000F5F1F4F882321F00E94CD89F801F6CF1C
:1056400088E290E099A388A388EC90E09DA78CA7BE
:10565000BE01605E7F4FCE018C960E94CABCC3C360
:105660000C5F1F4FBFEF8B1A9B0AE3E1F3E2E017D9
:10567000F10709F083CF4CE3E42E45E0F42E10E06F
:10568000F50181919191A191B1915F01F701819310
:105690009193A193B1937F01812F0E9498AD1F5FD9
:1056A000133071F70E944C9583E992E09DA78CA777
:1056B00004E610E019A308A3BE01645D7F4FCE018C
:1056C00080960E94CABC8AEB92E09DA78CA719A382
:1056D00008A3BE01645D7F4FCE0180960E94CABCC4
:1056E00082C383E50E949B4C882309F47CC30E94FB
:1056F000EB4B709303026093020275C38DED90E053
:105700000E94D8AD81116FC383E50E949B4C81112B
:1057100003C0E2EFFDE13AC00091520710E00E94A1
:10572000EB4B000F111FF801EC5CFD4F71836083A0
:105730008091520790E07C01EE0CFF1CEE0CFF1CE8
:1057400087010F5D1D4F880F991FFC01EC5CFD4F19
:1057500060817181072E000C880B990B0E9470E606
:105760002AE037ED43E25CE30E94CFE6F701E25224
:10577000FF4E20813181428153810E94CFE6D801C2
:105780006D937D938D939C9313972DC384918F017B
:105790000F5F1F4F882321F00E94CD89F801F6CFBB
:1057A00085E40E94CD8980915207805D0E94CD8959
:1057B000E0915207F0E0EE0FFF1FEC5CFD4F6081BF
:1057C000718183E196E00E9481C585E20E94CD89C6
:1057D0008AE00E94CD8907C380E50E94524C88234D
:1057E00009F401C30E94EB4B6B017C0183E50E942D
:1057F0009B4C882321F00E94EB4B8B0102C00FEFE2
:105800001FEFC8010196039708F0EDC2D7FCEBC269
:105810008C2DEBE1F6E09491891709F43FC33196A2
:10582000B6E0EB34FB07B9F73CC383E50E949B4C21
:10583000882319F00E94EB4B02C064E071E079A369
:1058400068A380E50E949B4C882339F00E94EB4BB3
:105850006938E3E17E0730F402C068EE73E07A83D2
:10586000698304C088E893E19A838983BE01605EFE
:105870007F4FCE0101960E94CABCB5C285E40E944A
:105880009B4C811110C080E50E94524C882391F0FE
:105890000E941B4C6093400770934107809342071E
:1058A0009093430707C00E94FB4B882361F3EDED03
:1058B000FDE171C089E40E94524C882381F00E946E
:1058C0001B4C2CEA35EC47E25EE30E94CFE6609386
:1058D0003C0770933D0780933E0790933F0784E415
:1058E0000E94524C882381F00E941B4C2CEA35EC1C
:1058F00047E25EE30E9492EB609344077093450792
:105900008093460790934707E2EFFDE184918F0172
:105910000F5F1F4F882321F00E94CD89F801F6CF39
:1059200040914007509141076091420770914307B1
:1059300083E596E00E9464C52CEA35EC47E25EE31D
:1059400060913C0770913D0780913E0790913F0721
:105950000E9492EBAB01BC018FE496E00E9464C50B
:105960002CEA35EC47E25EE360914407709145070D
:1059700080914607909147070E94CFE6AB01BC019A
:105980008BE496E00E9464C58AE00E94CD892BC218
:105990000E94CD89F80184918F010F5F1F4F811103
:1059A000F7CFE7E5F6E084918F010F5F1F4F882363
:1059B00009F419C20E94CD89F801F5CF83E50E9450
:1059C000524C182F882371F00E941B4C0E94FAEB56
:1059D000709326026093250221E0672B09F020E0F6
:1059E0002093130780E50E94524C882359F02091A0
:1059F000250230912602232B11F00E940C4C80933B
:105A00001307F1C11111EFC1E2EFFDE184918F01A4
:105A10000F5F1F4F882321F00E94CD89F801F6CF38
:105A200080911307882319F06BE173E002C06EE1E7
:105A300073E08EE796E00E949AC56091250270910E
:105A400026028DE696E00E9481C5E9E6F6E08491A3
:105A50008F010F5F1F4F882309F4C5C10E94CD89B4
:105A6000F801F5CF0E94098FBEC180E50E94524C1B
:105A7000882351F00E941B4C6093380770933907BC
:105A800080933A0790933B0789E40E94524C882305
:105A900081F00E941B4C2CEA35EC47E25EE30E9449
:105AA000CFE6609334077093350780933607909361
:105AB000370784E40E94524C882381F00E941B4CDB
:105AC0002CEA35EC47E25EE30E9492EB60933007EC
:105AD000709331078093320790933307E2EFFDE133
:105AE00084918F010F5F1F4F882321F00E94CD8981
:105AF000F801F6CF409138075091390760913A0785
:105B000070913B0789E996E00E9464C52CEA35EC68
:105B100047E25EE360913407709135078091360764
:105B2000909137070E9492EBAB01BC0185E996E0AA
:105B30000E9464C52CEA35EC47E25EE360913007D1
:105B40007091310780913207909133070E94CFE620
:105B5000AB01BC0181E996E00E9464C58AE00E9425
:105B6000CD8941C10E94CD89F80184918F010F5FD9
:105B70001F4F8111F7CFEDE9F6E084918F010F5FA0
:105B80001F4F882309F42FC10E94CD89F801F5CF5A
:105B90000E94E68D28C10E945D7025C10E941DC330
:105BA00022C183E50E94524C882321F00E940C4CB4
:105BB00091E089270E94AEBE16C181E080931B0749
:105BC0000E94536A10921B07882309F40CC1E2EF6C
:105BD000FDE184918F010F5F1F4F811103C0ECEA3B
:105BE000F6E004C00E94CD89F801F3CF84918F01C3
:105BF0000F5F1F4F882309F4F6C00E94CD89F8017A
:105C0000F5CF8091350A882309F4EDC081E08093B7
:105C1000380AE9C08AE50E949B4C811103C0EAEB77
:105C2000F6E00BC00E941B4C609340117093411131
:105C30008093421190934311D6C084918F010F5FDE
:105C40001F4F882321F00E94CD89F801F6CF4091A3
:105C5000401150914111609142117091431187EBB5
:105C600096E00E9464C58AE00E94CD89BCC08BE4A6
:105C70000E949B4C811103C0E2EFFDE136C08BE432
:105C80000E949B4C8823C1F00E941B4C6B017C013D
:105C900020E030E0A9010E94DCEC87FD0AC020E092
:105CA00030E040E251E4C701B6010E946AE61816EE
:105CB00034F4E9EDF6E00EC0C12CD12C76010E943F
:105CC000226AC092E706D092E806E092E906F092D6
:105CD000EA0689C084918F010F5F1F4F882309F462
:105CE00082C00E94CD89F801F5CF84918F010F5FAA
:105CF0001F4F882321F00E94CD89F801F6CF4091F3
:105D0000E7065091E8066091E9067091EA0688EF8F
:105D100096E00E9464C58AE00E94CD8964C081E05B
:105D20008093270283E50E949B4C882339F00E94D0
:105D30000C4C811158C00E947ACE55C083E50E9458
:105D4000524CF7CF0E94FEBC4EC0F0901C180E942F
:105D5000226A1091F61080E00E942DACFF2029F1FC
:105D6000E2EFFDE184918F010F5F1F4F882321F047
:105D70000E94CD89F801F6CF84E50E94CD896F2D70
:105D800070E080E090E04AE00E94F08C80E20E94A7
:105D9000CD89E5E1F7E084918F010F5F1F4F8823E4
:105DA00011F10E94CD89F801F6CF10924210812F97
:105DB0000E942DACE2EFFDE184918F010F5F1F4F38
:105DC000882321F00E94CD89F801F6CF609142101E
:105DD00070E083E097E00E9481C58AE00E94CD894F
:105DE00002C00E94FEBC109243100E945DCE96C07D
:105DF0000E94ADAA0E9489CAF6CF0E94EB4BAB016C
:105E0000BC014093AF0C5093B00C6093B10C7093F5
:105E1000B20C8EEF9BE00E94F697E5CF0E94226ABB
:105E200088E50E94524C882331F05F9A80913504B6
:105E30008E7F8093350489E50E94524C882339F087
:105E40008A9A479A809135048D7F809335048AE53C
:105E50000E94524C882361F08091080180958170E6
:105E600080930601479A809135048B7F8093350497
:105E700085E40E94524C882309F4B5CF129AB3CF1F
:105E80000E941DB1B0CFF7FAF094F7F8F094D10169
:105E9000CD92DD92ED92FC9213979FCB0E949EE1F2
:105EA000A2CF0E94226ABC2C60E08C2D0E9471BDA2
:105EB0000F3FBFEF1B0759F48C2D0E941BBD31E033
:105EC00020E0892B09F030E0032F122F05C00130AC
:105ED000110561F401E010E08B2D0E941BBD8017BD
:105EE000910709F480CF0E9403A1F6CF00E010E0F3
:105EF000F3CF61E0812F0E9471BD6E2D812F0E9432
:105F000043BDF12CB701812F0E94ADBD193009F0BE
:105F10006ACFF0924704E092460465CFC657DF4F40
:105F20000FB6F894DEBF0FBECDBFDF91CF911F91AA
:105F30000F91FF90EF90DF90CF90BF90AF909F9028
:105F40008F907F906F905F904F903F902F9008952B
:105F50002F923F924F925F926F927F928F929F9279
:105F6000AF92BF92CF92DF92EF92FF920F931F9367
:105F7000CF93DF93CDB7DEB76F970FB6F894DEBF40
:105F80000FBECDBFC0905004D0905104E090520499
:105F9000F090530420E030E040EA50E4C701B6013D
:105FA0000E946AE687FD19C120E030E041E953E430
:105FB000C701B6010E94DCEC18160CF40EC1109259
:105FC000520E1092510E809109014091500E042EF4
:105FD000000C550B817021E0822790E0481759078B
:105FE00009F433C080910901817028272093500E55
:105FF00081111BC00E94BC80EDE3FDE084918F0104
:10600000882351F0082E000C990B0E94B7800F5F77
:106010001F4FF8018491F4CF8DE090E00E94B7808B
:106020008AE090E00E94B78010C0E1E4FDE0849136
:106030008F01882389F3082E000C990B0E94B780EA
:106040000F5F1F4FF8018491F4CF8091430E83308E
:1060500009F44CC02CF4882351F08130D9F072C07F
:10606000843009F43EC0853009F44DC06BC0809186
:10607000350A882309F466C081E08093430E0E94AC
:1060800002596093470E7093480E8093490E909387
:106090004A0E58C08091350A811154C08091010C7C
:1060A000882321F082E08093430E4CC01092430E6F
:1060B000E9E3FDE084918F01882351F0082E000C64
:1060C000990B0E94B7800F5F1F4FF8018491F4CFA6
:1060D0008DE090E00E94B7808AE090E00E94B78057
:1060E00031C08091900E8823E9F22CC08091350A4E
:1060F000811128C08091B7099091B809891B8F70D0
:1061000009F496C01FC08091350A81111BC080918F
:10611000B7099091B809891B8F7009F4ABC012C000
:106120008DE090E00E94B7808AE090E00E94B78006
:106130001092430E89E19DE09093A8078093A707F2
:106140000E94F9898091380E9091390E03974CF591
:1061500073E4272E79E0372EE0E68E2EEAEE9E2EAF
:10616000A12CB12C8EE99FE00E946D4B18161906E8
:10617000C4F48091380E9091390E049794F48EE90E
:106180009FE00E94314B80933E0EE0913F0EF091D4
:10619000400E8A3019F08D3009F07DC0309709F03B
:1061A00083C08091380E9091390E009711F40C94B1
:1061B000293F01979093390E8093380E80913A0EC3
:1061C00090913B0E019664E070E00E949FED9093E9
:1061D0003B0E80933A0E0C94293F8091510E909182
:1061E000520E8136FAEE9F07E8F01092520E10928E
:1061F000510EE5E4FDE084918F01882351F0082ED3
:10620000000C990B0E94B7800F5F1F4FF80184911B
:10621000F4CF8DE090E00E94B7808AE090E00E9489
:10622000B780D1CE01969093520E8093510ECBCE73
:1062300085E29DE09093A8078093A7070E94F989C3
:106240008091900E882311F082E001C084E0809359
:10625000430EE1E2FDE084918F01882309F438CFF9
:10626000082E000C990B0E94B7800F5F1F4FF8019A
:106270008491F3CFEDE1FDE084918F01882309F44F
:106280004FCF082E000C990B0E94B7800F5F1F4F55
:10629000F8018491F3CF8A3309F480CFEF35F1050B
:1062A00014F40C94BD3C7ACF80913C0E90913D0E3D
:1062B00020E6289F7001299FF00C112487010854C3
:1062C000134FE00FF11F108261E470E0C8010E94DB
:1062D00006EE009711F40C94A13C9093420E80932B
:1062E000410E801B910B8E0D9F1D60E070E0875466
:1062F000934F0E946BE20E94FAEBCB01770FAA0B3F
:10630000BB0B8232910510F00C94A13CFC01882754
:10631000EE58FF4F8F4F0C94B2EDE4E1FDE0849115
:106320008F01882351F0082E000C990B0E94B78032
:106330000F5F1F4FF8018491F4CF20E030E040E080
:106340005FE36091500470915104809152049091E8
:1063500053041EC0EFE0FDE084918F01882351F0CB
:10636000082E000C990B0E94B7800F5F1F4FF80199
:106370008491F4CF60914E0470914F04072E000C6D
:10638000880B990B0E9470E620E030E040E05FE36C
:106390000E94B6EA0E94FAEBCB010E94F44D0E94E3
:1063A000EED78DE090E00E94B7808AE090E00E94F6
:1063B000B7800C94A13CEAE0FDE084918F01882332
:1063C00051F0082E000C990B0E94B7800F5F1F4FF1
:1063D000F8018491F4CF20E030E040E05FE3609189
:1063E0004A0470914B0480914C0490914D04D0CF9D
:1063F000E5E0FDE084918F01882351F0082E000C28
:10640000990B0E94B7800F5F1F4FF8018491F4CF62
:106410006091480470914904B1CF209146043091B5
:10642000470444E6429FC001439F900D11246FEF43
:1064300070E00E949FED8B016536710510F004E657
:1064400010E0E0E0FDE084917F01882359F0082E00
:10645000000C990B0E94B780FFEFEF1AFF0AF701BB
:106460008491F3CFB80180E090E036C7ECEFFCE018
:1064700084918F01882351F0082E000C990B0E9403
:10648000B7800F5F1F4FF8018491F4CF80E290E056
:106490000E94B780E8EFFCE084918F01882351F0DF
:1064A000082E000C990B0E94B7800F5F1F4FF80158
:1064B0008491F4CF60913604709137048091380450
:1064C000909139040E94EFD780E290E00E94B7805B
:1064D000E4EFFCE084918F01882351F0082E000C3A
:1064E000990B0E94B7800F5F1F4FF8018491F4CF82
:1064F00060913A0470913B0480913C0490913D047A
:106500000E94EFD780E290E00E94B780E0EFFCE0CD
:1065100084918F01882351F0082E000C990B0E9462
:10652000B7800F5F1F4FF8018491F4CF60913E0454
:1065300070913F0480914004909141040E94EFD7F4
:1065400080E290E0A0C58091350A882309F450C00C
:10655000EBEEFCE084918F01882351F0082E000CB3
:10656000990B0E94B7800F5F1F4FF8018491F4CF01
:106570008091360A882359F18091010C882329F1F2
:106580008091AB0C9091AC0CA091AD0CB091AE0C85
:106590000097A105B105C1F0BC01CD016D597F4F38
:1065A0008F4F9F4F24E630E040E050E00E9458EAD1
:1065B0006091AF0C7091B00C8091B10C9091B20CC5
:1065C0000E9458EA822F01C080E090E0E6CEE7EE1C
:1065D000FCE084918F01882309F4E3CE082E000C9F
:1065E000990B0E94B7800F5F1F4FF8018491F3CF82
:1065F000EFEDFCE084918F01882309F4D2CE082EC0
:10660000000C990B0E94B7800F5F1F4FF801849117
:10661000F3CFEAEDFCE084918F01882351F0082E3E
:10662000000C990B0E94B7800F5F1F4FF8018491F7
:10663000F4CF8091470E9091480EA091490EB091F1
:106640004A0E892B8A2B8B2B09F477C00E940259A2
:10665000A50194010E9458EA69017A016091470EF0
:106660007091480E8091490E90914A0EA5019401B7
:106670000E9458EA8601021B130BC8016CE370E00C
:106680000E948BEDCB019927EAE0F0E0BF010E9468
:106690009FED282FCB01BF010E949FED805D80936D
:1066A0002D04205D20932E0410922F048DE294E09F
:1066B0000E94EED780E290E00E94B780E8EDFCE017
:1066C00084917F01882359F0082E000C990B0E94B9
:1066D000B780FFEFEF1AFF0AF7018491F3CF80E252
:1066E00090E00E94B780C8016CE370E00E948BEDDF
:1066F0006AE070E00E949FED605D60932D04805D14
:1067000080932E0410922F048DE294E00E94EED725
:1067100080E290E00E94B780E6EDFCE084918F017A
:10672000882309F43ECE082E000C990B0E94B780F6
:106730000F5F1F4FF8018491F3CF80E290E00E9439
:10674000B780EEECFCE084918F01882309F429CE18
:10675000082E000C990B0E94B7800F5F1F4FF801A5
:106760008491F3CF1092710E8091090180FF11C0C6
:10677000EAECFCE084918F01882309F412CE082E04
:10678000000C990B0E94B7800F5F1F4FF801849196
:10679000F3CF83E50E948AD7882341F00E94A5D7D2
:1067A0000E94FFEB7093460E6093450EE6ECFCE012
:1067B00084918F01882351F0082E000C990B0E94C0
:1067C000B7800F5F1F4FF8018491F4CF8DE090E008
:1067D0000E94B7808AE090E00E94B78080918F0E7F
:1067E000882309F442C28091450E9091460E843070
:1067F000910509F4C8C08830910509F47DC1892B41
:1068000009F0E7C3EAEEFAE084918F01882351F0A2
:10681000082E000C990B0E94B7800F5F1F4FF801E4
:106820008491F4CF8DE090E00E94B7808AE090E000
:106830000E94B780EFEDFAE084918F01882351F038
:10684000082E000C990B0E94B7800F5F1F4FF801B4
:106850008491F4CF8DE090E00E94B7808AE090E0D0
:106860000E94B780E3EDFAE084918F01882351F014
:10687000082E000C990B0E94B7800F5F1F4FF80184
:106880008491F4CF8DE090E00E94B7808AE090E0A0
:106890000E94B780E7ECFAE084918F01882351F0E1
:1068A000082E000C990B0E94B7800F5F1F4FF80154
:1068B0008491F4CF8DE090E00E94B7808AE090E070
:1068C0000E94B780E9EBFAE084918F01882351F0B0
:1068D000082E000C990B0E94B7800F5F1F4FF80124
:1068E0008491F4CF8DE090E00E94B7808AE090E040
:1068F0000E94B780EBEAFAE084918F01882351F07F
:10690000082E000C990B0E94B7800F5F1F4FF801F3
:106910008491F4CF8DE090E00E94B7808AE090E00F
:106920000E94B780EEE9FAE084918F01882351F04C
:10693000082E000C990B0E94B7800F5F1F4FF801C3
:106940008491F4CF8DE090E00E94B7808AE090E0DF
:106950000E94B780E1E9FAE084918F01882351F029
:10696000082E000C990B0E94B7800F5F1F4FF80193
:106970008491F4CF8DE090E00E94B7808AE090E0AF
:106980000E94B78026C3E3E8FAE084918F01882350
:1069900051F0082E000C990B0E94B7800F5F1F4F1B
:1069A000F8018491F4CF8DE090E00E94B7808AE0F6
:1069B00090E00E94B780E5E7FAE084918F01882398
:1069C00051F0082E000C990B0E94B7800F5F1F4FEB
:1069D000F8018491F4CF8DE090E00E94B7808AE0C6
:1069E00090E00E94B780EFE5FAE084918F01882360
:1069F00051F0082E000C990B0E94B7800F5F1F4FBB
:106A0000F8018491F4CF8DE090E00E94B7808AE095
:106A100090E00E94B780E9E4FAE084918F01882336
:106A200051F0082E000C990B0E94B7800F5F1F4F8A
:106A3000F8018491F4CF8DE090E00E94B7808AE065
:106A400090E00E94B780E7E3FAE084918F01882309
:106A500051F0082E000C990B0E94B7800F5F1F4F5A
:106A6000F8018491F4CF8DE090E00E94B7808AE035
:106A700090E00E94B780E5E2FAE084918F018823DC
:106A800051F0082E000C990B0E94B7800F5F1F4F2A
:106A9000F8018491F4CF8DE090E00E94B7808AE005
:106AA00090E00E94B780E7E1FAE084918F018823AB
:106AB00051F0082E000C990B0E94B7800F5F1F4FFA
:106AC000F8018491F4CF8DE090E00E94B7808AE0D5
:106AD00090E00E94B780E9E0FAE084918F0188237A
:106AE00009F448CF082E000C990B0E94B7800F5F65
:106AF0001F4FF8018491F3CFE2E0FAE084918F0117
:106B0000882351F0082E000C990B0E94B7800F5F6C
:106B10001F4FF8018491F4CF8DE090E00E94B78080
:106B20008AE090E00E94B780EBEFF9E084918F015A
:106B3000882351F0082E000C990B0E94B7800F5F3C
:106B40001F4FF8018491F4CF8DE090E00E94B78050
:106B50008AE090E00E94B780E4EEF9E084918F0132
:106B6000882351F0082E000C990B0E94B7800F5F0C
:106B70001F4FF8018491F4CF8DE090E00E94B78020
:106B80008AE090E00E94B780EDECF9E084918F01FB
:106B9000882351F0082E000C990B0E94B7800F5FDC
:106BA0001F4FF8018491F4CF8DE090E00E94B780F0
:106BB0008AE090E00E94B780E6EBF9E084918F01D3
:106BC000882351F0082E000C990B0E94B7800F5FAC
:106BD0001F4FF8018491F4CF8DE090E00E94B780C0
:106BE0008AE090E00E94B780EFE9F9E084918F019C
:106BF000882351F0082E000C990B0E94B7800F5F7C
:106C00001F4FF8018491F4CF8DE090E00E94B7808F
:106C10008AE090E00E94B780ECE8F9E084918F016F
:106C2000882351F0082E000C990B0E94B7800F5F4B
:106C30001F4FF8018491F4CF8DE090E00E94B7805F
:106C40008AE090E00E94B780E9E7F9E084918F0143
:106C5000882309F48FCE082E000C990B0E94B78070
:106C60000F5F1F4FF8018491F3CF8091360A88237C
:106C700009F486C181E08093B30C1092B50C109298
:106C8000B40C85E89AE00E943D9A8BE1E5E8FAE0D1
:106C9000DE01159601900D928A95E1F78091830AA5
:106CA0009091840A9C838B838DEE92E09A838983F2
:106CB00040E050E0BE016F5F7F4F80E090E00E94B7
:106CC000EA82CE0101960E9499A0C090B40CD090A7
:106CD000B50C0091450E1091460EC601801B910B1C
:106CE000049720F06801F3E0CF0ED11C5AE6452E40
:106CF00059E0552E6BE5662E69E0762EC016D1065A
:106D000008F467C10115110509F0A1C069E37AE033
:106D100085E89AE00E94059962E273E089E39AE0CF
:106D20000E9411EE892B09F04AC0F20184914AE6D3
:106D3000E42E49E0F42E882359F0082E000C990B1C
:106D40000E94B780FFEFEF1AFF0AF7018491F3CF9B
:106D50008DE090E00E94B7808AE090E00E94B780CA
:106D6000F30184913BE5E32E39E0F32E882359F0BB
:106D7000082E000C990B0E94B780FFEFEF1AFF0A54
:106D8000F7018491F3CF8DE090E00E94B7808AE014
:106D900090E00E94B7804AE060E070E0CB010E9482
:106DA000F08CEBE4F9E084917F012FEFE21AF20A14
:106DB000882309F4E2C00E94CD89F701F4CFE7E40B
:106DC000F9E084917F01882359F0082E000C990B7B
:106DD0000E94B780FFEFEF1AFF0AF7018491F3CF0B
:106DE0008DE090E00E94B7808AE090E00E94B7803A
:106DF000F101849123E4E22E29E0F22E882359F058
:106E0000082E000C990B0E94B780FFEFEF1AFF0AC3
:106E1000F7018491F3CF8DE090E00E94B7808AE083
:106E200090E00E94B7804AE060E070E0CB010E94F1
:106E3000F08CEEE3F9E084917F012FEFE21AF20A81
:106E4000882309F49AC00E94CD89F701F4CF60E04D
:106E500070E0C80101970E94A8848091370A8823B6
:106E600009F45FC0ECE3F9E084917F01882359F0D5
:106E7000082E000C990B0E94B780FFEFEF1AFF0A53
:106E8000F7018491F3CF89E39AE00E94EED78DE079
:106E900090E00E94B7808AE090E00E94B780EAE329
:106EA000F9E084917F01882359F0082E000C990B9A
:106EB0000E94B780FFEFEF1AFF0AF7018491F3CF2A
:106EC00086E49AE00E94EED78DE090E00E94B780C1
:106ED0008AE090E00E94B780C801A0E0B0E04AE0FC
:106EE000BC01CD010E94F08CE8E3F9E084917F01C0
:106EF0002FEFE21AF20A882321F00E94CD89F701D0
:106F0000F5CF96E4E92E9AE0F92EF70181917F0101
:106F1000882319F00E94CD89F8CF8AE00E94CD899C
:106F20002CC089E39AE00E94EED78DE090E00E94A9
:106F3000B7808AE090E00E94B78086E49AE00E94E1
:106F4000EED78DE090E00E94B7808AE090E00E944A
:106F5000B780C801A0E0B0E04AE0BC01CD010E94CA
:106F6000F08C86E4E82E8AE0F82EF70181917F010B
:106F7000882399F20E94CD89F8CF0F5F1F4FBECEB4
:106F8000E9E2F9E084918F01882351F0082E000C8A
:106F9000990B0E94B7800F5F1F4FF8018491F4CFC7
:106FA0008DE090E00E94B7808AE090E00E94B78078
:106FB000EAE1F9E084918F01882309F4DBCC082E03
:106FC000000C990B0E94B7800F5F1F4FF80184914E
:106FD000F3CFE2ECFCE084918F01882309F4E1C94E
:106FE000082E000C990B0E94B7800F5F1F4FF8010D
:106FF0008491F3CF8091350A882339F00E941C8256
:10700000A0C48091350A8823E9F00E9472B899C41F
:107010008091430E823019F0833609F092C40E94A9
:10702000FC81EEEBFCE084918F01882309F4B9C95F
:10703000082E000C990B0E94B7800F5F1F4FF801BC
:107040008491F3CF8091430E833609F07AC4DDCF6B
:1070500085EB9CE00E94BCA08091B7099091B80993
:10706000891B8F7009F06DC48091430E823009F442
:1070700068C4833609F099C464C48DE090E00E942E
:10708000B7808AE090E00E94B7808BC98091B709F1
:107090009091B809891B8F7009F053C48091430EF9
:1070A000823009F44EC4833609F44BC48091010C3C
:1070B0008111CFC446C483E50E948AD7811126C0BE
:1070C00083E40E948AD7882309F43BC48091B709DE
:1070D0009091B809891B8F7009F033C420E030E02B
:1070E00040E251E460913E0470913F04809140047D
:1070F000909141040E946AE687FF08C082EA9CE002
:107100009093A8078093A7070E94F9890E94A5D7AA
:1071100020E030E0A9010E946AE687FD10C00E94CD
:10712000A5D720E030E849E853E40E94DCEC1816CB
:107130004CF00E94A5D70E94FFEBCB0105C080E078
:1071400090E002C083E191E00E94F759FAC383E521
:107150000E948AD7882309F4F4C30E94A5D720E0AF
:1071600030E0A9010E946AE687FD10C00E94A5D701
:1071700020E030E046E153E40E94DCEC18164CF0CD
:107180000E94A5D70E94FFEBCB0105C080E090E0F4
:1071900002C086E990E00E942A4ED3C383E50E9494
:1071A0008AD78823D9F00E94A5D720E030E04FE7A6
:1071B00053E40E94CFE620E030E048EC52E40E9425
:1071C00092EB0E94FFEB6F3F710519F010F06FEF2B
:1071D00070E07093470460934604E3C88FEF90E03B
:1071E0009093470480934604DCC88091B70990913E
:1071F000B809891B8F7009F0D4C88091350A8111B4
:10720000D0C80E94CD8E5F9A809135048E7F809386
:1072100035048A9A479A809135048D7F809335048E
:10722000809108018095817080930601479A809132
:1072300035048B7F80933504129AB3C883E50E948E
:107240008AD7882319F10E94A5D720E030E040E2D8
:1072500052E40E946AE687FD0FC00E94A5D720E095
:1072600030EC49E754E40E94DCEC181644F00E942C
:10727000A5D70E94FAEB05C068E270E002C067EE95
:1072800073E070930302609302025BC3ECE9FCE0DD
:1072900084918F01882351F0082E000C990B0E94D5
:1072A000B7800F5F1F4FF8018491F4CFC0900202A6
:1072B000D09003020D2C000CEE08FF08F7FE0EC064
:1072C0006DE28EE99FE00E94E44A66277727CB01B2
:1072D0006C197D098E099F094AE003C04AE0C70185
:1072E000B6010E94AED75DC88091B7099091B809E8
:1072F000891B8F7009F025C38091430E823009F4F9
:1073000020C3833609F0EBC21CC38091B70990916A
:10731000B809891B8F7009F044C88091430E8230F0
:1073200009F43FC8833609F0B6C33BC88091B7095A
:107330009091B809891B8F7009F003C38091430EA7
:10734000823009F4FEC2833609F0FBC4FAC2809190
:10735000B7099091B809891B8F7009F0F2C280912A
:10736000430E823009F4EDC2833609F020C5E9C22C
:107370008091B7099091B809891B8F7009F0E1C21B
:107380008091430E823009F4DCC2833609F045C592
:10739000D8C28091710E811103C00E94BC80C4C10B
:1073A0008E3271F58091720E8E3209F046C1809155
:1073B000D60B882309F4B8C181508093D60B88235B
:1073C00061F090E001974FE1489F9001499F300D97
:1073D0001124C9018056954F02C082E69AE02BE144
:1073E000FC013496A5E8BAE001900D922A95E1F7E8
:1073F000FC01828193819093840A8093830A94C1D3
:107400008C3309F01AC164E273E081E79EE00E94C8
:1074100011EE892B21F481E080938F0E85C163E307
:1074200073E081E79EE00E9411EE892B79F4E6EF8C
:10743000F8E084918F010F5F1F4F882321F00E9495
:10744000CD89F801F6CF89ED98E0E4C06AE473E0F5
:1074500081E79EE00E9411EE892B79F4E5EBF8E0DC
:1074600084918F010F5F1F4F882321F00E94CD89E7
:10747000F801F6CF82EA98E0CDC061E673E081E7DB
:107480009EE00E9411EE892B79F4E7E8F8E0849100
:107490008F010F5F1F4F882321F00E94CD89F801D3
:1074A000F6CF82E898E0B6C06FE673E081E79EE031
:1074B0000E9411EE892B79F4E2E6F8E084918F01C5
:1074C0000F5F1F4F882321F00E94CD89F801F6CF6E
:1074D0008DE598E09FC062E873E081E79EE00E943E
:1074E00011EE892B79F4E2E4F8E084918F010F5FCB
:1074F0001F4F882321F00E94CD89F801F6CF89E340
:1075000098E088C060E973E081E79EE00E9411EE98
:10751000892B71F406E118E0F8018491882329F0A1
:107520000F5F1F4F0E94CD89F7CF8FE098E072C0A8
:1075300066EA73E081E79EE00E9411EE892B79F400
:10754000E0EFF7E084918F010F5F1F4F882321F058
:107550000E94CD89F801F6CF89EE97E05BC068EB19
:1075600073E081E79EE00E9411EE892B79F4E1ED52
:10757000F7E084918F010F5F1F4F882321F00E9455
:10758000CD89F801F6CF80EC97E044C063EC73E05E
:1075900081E79EE00E9411EE892B79F4E7EAF7E09B
:1075A00084918F010F5F1F4F882321F00E94CD89A6
:1075B000F801F6CF85E997E02DC06FEC73E081E725
:1075C0009EE00E9411EE892B79F4EAE7F7E08491BE
:1075D0008F010F5F1F4F882321F00E94CD89F80192
:1075E000F6CF88E697E016C06DED73E081E79EE088
:1075F0000E9411EE892BA9F4EEE4F7E084918F014B
:107600000F5F1F4F882321F00E94CD89F801F6CF2C
:107610008DE397E09093A8078093A7070E94F989CC
:1076200083C06AEE73E081E79EE00E9411EE892B31
:1076300009F07AC010928F0E77C01D8218861C82C6
:107640001B828DEE92E09A8389838091880A811152
:1076500003C062E67AE002C061E87AE06115710574
:1076600019F06C5F7F4F02C060E070E021E041E7FD
:107670005EE0CE0105960E946C9E882361F18BE14D
:10768000FE013596A5E8BAE001900D928A95E1F7E2
:107690002B813C813093840A2093830A8091D60BFE
:1076A0008A3008F03DC091E0980F9093D60BFFE12F
:1076B0008F9FC0011124DC01AC55B54F4BE1E5E8CB
:1076C000FAE001900D924A95E1F7FC01E056F54F82
:1076D0003383228325C0E2EFFDE184918F010F5FA8
:1076E0001F4F882321F00E94CD89F801F6CFE7E2F1
:1076F000F7E084918F010F5F1F4F882321F00E94D4
:10770000CD89F801F6CF01E71EE0F80181918F01E4
:10771000882319F00E94CD89F8CF8AE00E94CD8994
:10772000CE0101960E9499A01092710E80910901DC
:1077300080FF07C1E0EEFBE084918F01882311F404
:107740000C94D131082E000C990B0E94B7800F5F6A
:107750001F4FF8018491F2CF8FE40E948AD78111E4
:107760000C94D13183E40E948AD70C94D13183E503
:107770000E948AD7811159C08FE40E948AD788233A
:1077800019F088EA9BE007C084E50E948AD7882325
:1077900049F080E89BE09093A8078093A7070E9498
:1077A000F98943C083E40E948AD7882319F087E5CA
:1077B0009BE0F1CF81E50E948AD7882319F08FE200
:1077C0009BE0E9CF88E40E948AD78823C9F0EBE2E6
:1077D000FBE084918F01882351F0082E000C990B57
:1077E0000E94B7800F5F1F4FF8018491F4CF8DE0A6
:1077F00090E00E94B7808AE090E00E94B78015C0B8
:107800008CE40E948AD7882381F0E7E2FBE0849130
:107810008F01882361F3082E000C990B0E94B7801A
:107820000F5F1F4FF8018491F4CFEFEEFBE08491DE
:107830008F01882311F40C94D131082E000C990B80
:107840000E94B7800F5F1F4FF8018491F2CF8091A3
:10785000B7098091B8090C94D13183E50E948AD789
:10786000882309F46EC08FEF9AE09093A807809365
:10787000A7070E94F989EFEEFBE084918F0188232E
:1078800011F40C94D131082E000C990B0E94B78092
:107890000F5F1F4FF8018491F2CFEAEFFAE0849175
:1078A0008F01882351F0082E000C990B0E94B7809D
:1078B0000F5F1F4FF8018491F4CFE5EFFAE0849158
:1078C0008F01882311F40C94D131082E000C990BF0
:1078D0000E94B7800F5F1F4FF8018491F2CF88E5B7
:1078E0000E948AD7811106C089E50E948AD7882321
:1078F00009F4C3C088E50E948AD7882341F086E94D
:107900009CE09093A8078093A7070E94F98989E5D6
:107910000E948AD7882341F080E99CE09093A807D1
:107920008093A7070E94F9898AE50E948AD7882355
:1079300041F08AE89CE09093A8078093A7070E94F3
:10794000F98980913C0E90913D0E019664E070E0C3
:107950000E949FED90933D0E80933C0E8091380ED7
:107960009091390E01969093390E8093380E1092B3
:10797000400E10923F0E0C94B23040913C0E50914C
:107980003D0E9F012F5F3F4F3093400E20933F0EDF
:1079900090E6949F9001959F300D11242854334F09
:1079A000E20FF31F80830C94B2300091410E1091CE
:1079B000420E780124E0E20EF11C6AE270E0C70199
:1079C0000E9406EEF80124812F3221F4B8016B5F8A
:1079D0007F4F03C02C3339F4B70181E79EE00E944A
:1079E0001AEE0C94D1311092710E009719F0FC012F
:1079F000319710828091410E9091420E40E061E0FB
:107A000004960E94B8D58091010C882389F0E1EB9F
:107A1000FCE084918F01882309F42FCB082E000C01
:107A2000990B0E94B7800F5F1F4FF8018491F3CF2D
:107A3000EDEAFCE084918F01882309F41ECB082E27
:107A4000000C990B0E94B7800F5F1F4FF8018491C3
:107A5000F3CF0E94FC81E9EAFCE084918F01882346
:107A600011F40C94D131082E000C990B0E94B780B0
:107A70000F5F1F4FF8018491F2CF8AE50E948AD7E9
:107A8000811138CF83E40E948AD7882309F459CF23
:107A900086E89CE050CF86E40E948AD7882309F4C8
:107AA0004DC10E94A5D70E94FFEB8B0182E89CE0AC
:107AB0009093A8078093A7070E94F98988E50E9400
:107AC0008AD7882309F451C00E94A5D72B013C0115
:107AD0002DEC3CEC4CE45EE30E946AE69E012F5FD5
:107AE0003F4F7901181674F020E030E0A901C3017E
:107AF000B2010E94DCEC18162CF41F930F9387E759
:107B00009CE005C12DEC3CEC4CEC5DEBC301B201FB
:107B10000E946AE618167CF020E030E040E85FEB57
:107B2000C301B2010E94DCEC18162CF41F930F93D2
:107B30008BE69CE0ECC01F930F93C301B2010E943F
:107B4000FAEB7F936F9381E69CE09F938F93FF9274
:107B5000EF920E943CE60FB6F894DEBF0FBECDBF99
:107B6000CE0101960E94D489DFC089E50E948AD7A0
:107B7000882309F441C00E94A5D72B013C012DECBC
:107B80003CEC4CE45EE30E946AE6FE0131967F0124
:107B9000181674F020E030E0A901C301B2010E9480
:107BA000DCEC18162CF41F930F9386E59CE0AFC015
:107BB0002DEC3CEC4CEC5DEBC301B2010E946AE69B
:107BC00018167CF020E030E040E85FEBC301B20122
:107BD0000E94DCEC18162CF41F930F938AE49CE0AF
:107BE00096C01F930F93C301B2010E94FAEB7F93DB
:107BF0006F9380E49CE0A9CF8AE50E948AD788230E
:107C000009F441C00E94A5D72B013C012DEC3CECAE
:107C10004CE45EE30E946AE6FE0131967F0118168D
:107C200074F020E030E0A901C301B2010E94DCEC55
:107C300018162CF41F930F9385E39CE068C02DEC7D
:107C40003CEC4CEC5DEBC301B2010E946AE61816F5
:107C50007CF020E030E040E85FEBC301B2010E941D
:107C6000DCEC18162CF41F930F9389E29CE04FC0B4
:107C70001F930F93C301B2010E94FAEB7F936F939E
:107C80008FE19CE062CF85E40E948AD7882309F4C3
:107C90004BC00E94A5D72B013C012DEC3CEC4CE4E1
:107CA0005EE30E946AE6FE0131967F01181674F0C9
:107CB00020E030E0A901C301B2010E94DCEC1816FB
:107CC0002CF41F930F9384E19CE021C02DEC3CEC3D
:107CD0004CEC5DEBC301B2010E946AE618167CF021
:107CE00020E030E040E85FEBC301B2010E94DCEC31
:107CF00018162CF41F930F9388E09CE008C0C30172
:107D0000B2010E94FAEB7F936F938DEF9BE09F93FC
:107D10008F93FF92EF920E943CE60F900F900F908E
:107D20000F900F900F901CCF89EF9BE09093A807C6
:107D30008093A7070E94F9890C94D13100E010E0EC
:107D4000B5CE20E030E040E251E460913E04709115
:107D50003F0480914004909141040E946AE687FFAD
:107D600008C082EF9BE09093A8078093A7070E942A
:107D7000F98982E390E090934904809348040E943B
:107D8000BA7688EC90E00E94F759EFEEFBE0849120
:107D90008F01882311F40C94D131082E000C990B1B
:107DA0000E94B7800F5F1F4FF8018491F2CF20E04F
:107DB00030E040E251E460913E0470913F048091D4
:107DC0004004909141040E946AE687FF08C088EE53
:107DD0009BE09093A8078093A7070E94F98980E50C
:107DE00090E090934904809348040E94BA7680EF13
:107DF00090E00E94F759EFEEFBE084918F01882319
:107E000011F40C94D131082E000C990B0E94B7800C
:107E10000F5F1F4FF8018491F2CF80E090E00E9445
:107E2000F75910924904109248040E94BA76E4EE81
:107E3000FBE084918F01882311F40C94D131082E3A
:107E4000000C990B0E94B7800F5F1F4FF8018491BF
:107E5000F2CF6F960FB6F894DEBF0FBECDBFDF91A5
:107E6000CF911F910F91FF90EF90DF90CF90BF9037
:107E7000AF909F908F907F906F905F904F903F90CA
:107E80002F9008952F923F924F925F926F927F9220
:107E90008F929F92AF92BF92CF92DF92EF92FF921A
:107EA0000F931F93CF93DF93CDB7DEB762970FB6D3
:107EB000F894DEBF0FBECDBFF8948FEF9FEF909385
:107EC0008900809388002AE02A8B212C312C789419
:107ED0008091A6049091A704A091A804B091A90450
:107EE000892B8A2B8B2B09F016C280911E078823C1
:107EF000E1F010921E0780911C0790911D07892BBD
:107F000009F409C210925E0410921D0710921C071A
:107F10009091B7098091B809981709F4FCC1809134
:107F2000B8098F5F8F708093B80980911C0790917A
:107F30001D07892B09F4EFC14091A2045091A304BD
:107F40006091A4047091A50480919E0490919F0477
:107F5000A091A004B091A1040091950410E020E04C
:107F600030E0841B950BA60BB70B081719072A07DF
:107F70003B0710F4D901C801E82F840F951FA61FF5
:107F8000B71F8093A2049093A304A093A404B0937A
:107F9000A5042091840030918500225E3F4F4091DE
:107FA0007A0450917B0460917C0470917D048091EF
:107FB0006A0490916B04A0916C04B0916D04840FDD
:107FC000951FA61FB71F80937A0490937B04A093FC
:107FD0007C04B0937D04B7FD1CC0889A8091FC108E
:107FE0009091FD10A091FE10B091FF1040910402FD
:107FF000042E000C550B660B770B840F951FA61FE4
:10800000B71F8093FC109093FD10A093FE10B093C7
:10801000FF1040917E0450917F0460918004709124
:10802000810480916E0490916F04A0917004B091CE
:108030007104840F951FA61FB71F80937E04909331
:108040007F04A0938004B0938104B7FD1CC08E9A76
:108050008091001190910111A0910211B091031132
:1080600040910502042E000C550B660B770B840F14
:10807000951FA61FB71F8093001190930111A09325
:108080000211B093031140918204509183046091D6
:108090008404709185048091720490917304A0917E
:1080A0007404B0917504840F951FA61FB71F8093A9
:1080B000820490938304A0938404B0938504B7FD55
:1080C0003FC080915804F09106028823C9F0809146
:1080D000560482FF02C0F7FD06C080915504882334
:1080E00011F40C94F748809156049091570493FF33
:1080F00002C0F7FD0CC080915404811108C006C075
:1081000080910B018095887080930901419A40917C
:1081100004115091051160910611709107118F2F74
:10812000FF0F990BAA0BBB0B840F951FA61FB71F40
:108130008093041190930511A0930611B093071139
:10814000409186045091870460918804709189045D
:108150008091760490917704A0917804B09179048D
:10816000840F951FA61FB71F8093860490938704E2
:10817000A0938804B0938904B7FD3AC040910811D8
:108180005091091160910A1170910B11C090070272
:108190000C2C000CDD08EE08FF084C0D5D1D6E1D5B
:1081A0007F1D409308115093091160930A11709339
:1081B0000B114091660450916704609168047091BE
:1081C0006904841B950BA60BB70B809386049093D0
:1081D0008704A0938804B0938904909159048091F6
:1081E000930493FF02C0815001C08F5F809393047A
:1081F000809184009091850082179307C8F3809145
:108200007A0490917B04A0917C04B0917D04B7FD29
:1082100015C04091660450916704609168047091A4
:108220006904841B950BA60BB70B80937A0490937B
:108230007B04A0937C04B0937D04889880917E0495
:1082400090917F04A0918004B0918104B7FD15C086
:1082500040916604509167046091680470916904CC
:10826000841B950BA60BB70B80937E0490937F0421
:10827000A0938004B09381048E98809182049091A1
:108280008304A0918404B0918504B7FD3AC0409165
:108290006604509167046091680470916904841BBE
:1082A000950BA60BB70B8093820490938304A09345
:1082B0008404B0938504809158048823E1F0809170
:1082C000560482FF04C08091060287FD05C080919C
:1082D0005504882309F493C780915604909157045C
:1082E00093FF04C08091060287FD0BC08091540467
:1082F000811107C005C080910B018870809309012E
:108300004198E15041F0809184009091850082175E
:108310009307C8F342CE8091110290911202A0916E
:108320001302B0911402892B8A2B8B2B09F091C078
:1083300080919404882309F453C08090A204909003
:10834000A304A090A404B090A504C0908F04D09082
:108350009004E0909104F090920440919304C8142A
:10836000D904EA04FB0480F480915F0490916004D6
:1083700020916304309164042817390728F4415090
:1083800040939304019714C08C149D04AE04BF0461
:10839000E0F480915F049091600420916104309139
:1083A00062048217930788F44F5F40939304019609
:1083B0009093600480935F0440910D0250910E02EF
:1083C00060910F02709110020EC08FEF9FEFDC01E1
:1083D00080930D0290930E02A0930F02B0931002AF
:1083E0004FEF5FEFBA018091930487FD02C0169AA8
:1083F00001C0169880918400909185004E9620913E
:1084000093042223F1F0149A209184003091850086
:1084100028173907C8F32091930427FF02C02F5F64
:1084200001C0215020939304149820919304222397
:1084300031F3209184003091850028173907C8F363
:10844000DDCF409311025093120260931302709398
:1084500014028091A6049091A704A091A804B09161
:10846000A904892B8A2B8B2B09F046C6A0911C07E7
:10847000B0911D07109711F40C94A04A8090A204AB
:108480009090A304A090A404B090A50440919E04F1
:1084900050919F046091A0047091A10484169506E8
:1084A000A606B706D8F010925E0410921D0710922F
:1084B0001C079091B7098091B809981711F40C9492
:1084C000A04A8091B8098F5F8F708093B80940ED02
:1084D000C42E47E0D42EE12CF12C1AC440919A040A
:1084E00050919B0460919C0470919D04481559051E
:1084F0006A057B0508F4AAC140919604509197043F
:108500006091980470919904D6960D911D912D91CA
:108510003C91D997401751076207730708F077C15C
:10852000411551056105710549F480905A049090F8
:108530005B04A0905C04B0905D0464C1E12CF98000
:10854000842E952F862F0A811B81FD81EE813F812C
:1085500028859C80E091F817E89D912CFF273091A9
:10856000F917389D900CF11D1090FA17189CF00D1A
:10857000E99F900CF11D399FF00DE89FF00D092D3A
:108580001F2F099DE12D332722270F9FE00D311D5D
:108590002E1D199DE00D311D2E1D1F9F300D211D1B
:1085A000032F122F099DF12C332722270F9FF00C48
:1085B000311D2E1D199DF00C311D2E1D1F9F300DDC
:1085C000211D032F122FEE2780905A0490915B04F7
:1085D00080915C040090B6040E2809F483C03091A9
:1085E000B204309FE1198E089E098E092091B304D0
:1085F000209FE01981089E098E09F090B404F09E36
:10860000801891098E09319FE01981089E098E0911
:10861000219F801891098E09F19E90198109099D69
:10862000F12C332722270F9FF00C311D2E1D199D91
:10863000F00C311D2E1D1F9F300D211D032F122FF9
:108640003091AE04309FE10D8E1C9E1D8E1D209139
:10865000AF04209FE00D811C9E1D8E1DF090B00484
:10866000F09E800C911D8E1D319FE00D811C9E1D82
:108670008E1D219F800C911D8E1DF19E900D811DE0
:10868000099DF12C332722270F9FF00C311D2E1D41
:10869000199DF00C311D2E1D1F9F300D211D032F24
:1086A000122F3091AA04309FE1198E089E098E097D
:1086B0002091AB04209FE01981089E098E09F0905B
:1086C000AC04F09E801891098E09319FE019810851
:1086D0009E098E09219F801891098E09F19E90199B
:1086E000810982C03091B204309FE10D8E1C9E1D25
:1086F0008E1D2091B304209FE00D811C9E1D8E1DB8
:10870000F090B404F09E800C911D8E1D319FE00D01
:10871000811C9E1D8E1D219F800C911D8E1DF19E22
:10872000900D811D099DF12C332722270F9FF00CFE
:10873000311D2E1D199DF00C311D2E1D1F9F300D5A
:10874000211D032F122F3091AE04309FE1198E08A6
:108750009E098E092091AF04209FE01981089E098F
:108760008E09F090B004F09E801891098E09319F17
:10877000E01981089E098E09219F801891098E09B0
:10878000F19E90198109099DF12C332722270F9F13
:10879000F00C311D2E1D199DF00C311D2E1D1F9F3B
:1087A000300D211D032F122F3091AA04309FE10DAF
:1087B0008E1C9E1D8E1D2091AB04209FE00D811C00
:1087C0009E1D8E1DF090AC04F09E800C911D8E1DA0
:1087D000319FE00D811C9E1D8E1D219F800C911DDF
:1087E0008E1DF19E900D811D11249C82F9820A83B9
:1087F0001B83FD83EE833F832887912C992AA12C2C
:10880000B12CA82A89E495E121E0298B14C0D296E5
:108810008D909D90AD90BC90D597F4CFB694A794D1
:1088200097948794D988DD0CD98A049625E18536FA
:10883000920709F4EAC4FC01059115912591349140
:10884000081519052A053B0548F3DFC440908F043D
:1088500050909004609091047090920448145904D0
:108860006A047B0408F0C3C180918E04811121C089
:10887000FD01EE5BFF4FE080F1800281138178966D
:108880002081318142815381D2966D917D918D916C
:108890009C91D5970E9490C4DD24D394D0928E04ED
:1088A000E0911C07F0911D0782A993A9A4A9B5A97D
:1088B0008EC140918A0450918B0460918C04709118
:1088C0008D04DA960D911D912D913C91DD97401705
:1088D00051076207730708F073C14115510561051F
:1088E000710549F480915A0490915B04A0915C0455
:1088F000B0915D046CC1F0E0E985842F352F262FFF
:10890000AA857B856C855D85BE854F859889B091EC
:10891000F817B89F612D55274091F917489F600DB2
:10892000511D1090FA17189E500DB39F600D511DE8
:10893000439F500DB29F500DA62F752FA69FB12DAE
:1089400044279927A59FB00D411D9F1F769FB00D0D
:10895000411D9F1F759F400D911DA42F792FA69F2C
:10896000E12D44279927A59FE00D411D9F1F769F6C
:10897000E00D411D9F1F759F400D911DA42F792F64
:10898000BB2780915A0430915B0420915C040090D5
:10899000B6040F2A09F483C04091B2044A9FB1196A
:1089A0008F0B3F0B2F0B9091B3049A9FB019810945
:1089B0003F0B2F0BE091B404EA9F801931092F0B74
:1089C000479FB01981093F0B2F0B979F80193109E1
:1089D0002F0BE79F30192109A69FE12D44279927E6
:1089E000A59FE00D411D9F1F769FE00D411D9F1F1C
:1089F000759F400D911DA42F792F4091AE044A9F81
:108A0000B10D8F1F3F1F2F1F9091AF049A9FB00D84
:108A1000811D3F1F2F1FE091B004EA9F800D311D83
:108A20002F1F479FB00D811D3F1F2F1F979F800D48
:108A3000311D2F1FE79F300D211DA69FE12D4427DB
:108A40009927A59FE00D411D9F1F769FE00D411DB9
:108A50009F1F759F400D911DA42F792F4091AA044F
:108A60004A9FB1198F0B3F0B2F0B9091AB049A9F2C
:108A7000B01981093F0B2F0BE091AC04EA9F8019DC
:108A800031092F0B479FB01981093F0B2F0B979F7F
:108A9000801931092F0BE79F3019210982C04091BD
:108AA000B2044A9FB10D8F1F3F1F2F1F9091B30437
:108AB0009A9FB00D811D3F1F2F1FE091B404EA9FC4
:108AC000800D311D2F1F479FB00D811D3F1F2F1F90
:108AD000979F800D311D2F1FE79F300D211DA69FF1
:108AE000E12D44279927A59FE00D411D9F1F769FEB
:108AF000E00D411D9F1F759F400D911DA42F792FE3
:108B00004091AE044A9FB1198F0B3F0B2F0B9091F0
:108B1000AF049A9FB01981093F0B2F0BE091B0046D
:108B2000EA9F801931092F0B479FB01981093F0B2C
:108B30002F0B979F801931092F0BE79F30192109BF
:108B4000A69FE12D44279927A59FE00D411D9F1F5A
:108B5000769FE00D411D9F1F759F400D911DA42F15
:108B6000792F4091AA044A9FB10D8F1F3F1F2F1FDD
:108B70009091AB049A9FB00D811D3F1F2F1FE09174
:108B8000AC04EA9F800D311D2F1F479FB00D811D42
:108B90003F1F2F1F979F800D311D2F1FE79F300D07
:108BA000211D1124E987AA877B876C875D87BE8793
:108BB0004F87988B90E0932BA0E0B0E0A22B07C0EA
:108BC000A65ABF4F8D919D910D90BC91A02D29E487
:108BD00035E141E0498BF9014591559165917491D9
:108BE000481759076A077B0708F499C3A6C3809101
:108BF00093048823E1F0FD01E85BFF4F4081518140
:108C000060E070E000910D0210910E0220910F02C1
:108C100030911002401751076207730741F010921C
:108C2000110210921202109213021092140240913B
:108C3000090250910A0260910B0270910C0277FFB9
:108C40005FC0AE5ABF4FCD90DD90ED90FC9089E4AF
:108C500095E121E0FC0145915591659174914C1588
:108C60005D056E057F0550F4F694E794D794C7949C
:108C7000220F049675E18536970761F720939504D6
:108C800080E2C816D104E104F10428F470E2C72E92
:108C9000D12CE12CF12C90E2C91AD108E108F1089D
:108CA000C114A8E0DA06E104F10408F402C4B4E057
:108CB000DB9EC0011124875B9E4EFC0132962591FC
:108CC0003491EC2D6627E39FA001E29F410D561FD2
:108CD0000694461F561F112460E070E0FC012591A8
:108CE0003491C901A0E0B0E0841B950BA60BB70B33
:108CF0008093090290930A02A0930B02B0930C0296
:108D0000C0900902D0900A02E0900B02F0900C0291
:108D100080911C0790911D07892B09F0E5C10E94E5
:108D200012C590931D0780931C07892B09F4DCC1A1
:108D3000E0911C07F0911D07808183FF3EC085896B
:108D40009689A789B08D8093FC109093FD10A09315
:108D5000FE10B093FF10818D928DA38DB48D809302
:108D6000001190930111A0930211B0930311858D0E
:108D7000968DA78DB0A18093041190930511A093B7
:108D80000611B093071181A192A1A3A1B4A1809370
:108D9000081190930911A0930A11B0930B119091AF
:108DA000B7098091B809981709F4B9CF8091B8092B
:108DB0008F5F8F708093B809B2CFC588D688E78857
:108DC000F08C81E0C114D104E104F10409F480E0E5
:108DD000018D128D238D348D01151105210531056D
:108DE00009F08260458D568D678D70A14115510542
:108DF0006105710509F0846080935E0410928A0415
:108E000010928B0410928C0410928D041092960490
:108E100010929704109298041092990485A196A13B
:108E2000A7A1B0A580939E0490939F04A093A00453
:108E3000B093A104882499245401881A990AAA0A93
:108E4000BB0A8092860490928704A0928804B09214
:108E500089048092820490928304A0928404B09248
:108E6000850480927E0490927F04A0928004B09248
:108E7000810480927A0490927B04A0927C04B09248
:108E80007D04CC0CDD1CEE1CFF1CC0926A04D09249
:108E90006B04E0926C04F0926D04000F111F221F0E
:108EA000331F00936E0410936F042093700430936B
:108EB0007104440F551F661F771F4093720450932F
:108EC0007304609374047093750441A152A163A16B
:108ED00074A1440F551F661F771F4093760450936B
:108EE00077046093780470937904880F991FAA1F00
:108EF000BB1F8093660490936704A0936804B093AB
:108F000069041092A2041092A3041092A404109277
:108F1000A50482A593A5A4A5B5A580939A049093D2
:108F20009B04A0939C04B0939D0486A597A5A0A93B
:108F3000B1A980938F0490939004A0939104B0936F
:108F4000920481A580936504DF01A95BBF4F9C91CA
:108F500090939404992339F115962D913C91119792
:108F6000309364042093630412972D913C911197E0
:108F70003093620420936104109211021092120245
:108F8000109213021092140212972D913C91A90194
:108F900060E070E040930D0250930E0260930F0268
:108FA000709310020CC088248A94982C54018092EB
:108FB0000D0290920E02A0920F02B0921002EA5B94
:108FC000FF4F90812091590492130AC0209108020A
:108FD00030E0482F082E000C550B4217530731F094
:108FE00090935904809308020E94E2C40E9438B70B
:108FF0002FEF3FEFA9012093090230930A0240931B
:109000000B0250930C02E0911C07F0911D07DF0149
:10901000DE96ED90FD900D911C9122A933A944A9F3
:1090200055A9EA5AFF4F60817181828193810E9424
:1090300090C410928E04E0911C07F0911D07EA5A2B
:10904000FF4F80809180A280B38089E495E121E088
:10905000FC014591559165917491481559056A0532
:109060007B0558F4B694A79497948794220F04969E
:10907000A5E6B5E1A817B90759F720939504B0E222
:109080008B169104A104B10428F4B0E28B2E912C2C
:10909000A12CB12C30E2831A9108A108B1088114E7
:1090A00048E09406A104B10408F427C254E0959E58
:1090B000C0011124875B9E4EFC01329625913491AC
:1090C000782D6627739FA001729F410D561F06944D
:1090D000461F561F1124FC01C590D490E12CF12CA1
:1090E000C41AD50AE108F108C092A604D092A704D8
:1090F000E092A804F092A9040091A6041091A7049C
:109100002091A8043091A9044091110250911202BB
:109110006091130270911402F02E198BF22FE32F3D
:10912000401751076207730720F4F42E598BF62F6E
:10913000E72F8F2D9989AF2FBE2F0097E1E0AE0763
:10914000B10520F08FEF9FEFA0E0B0E0081B190BF6
:109150002A0B3B0B0093A6041093A7042093A804AA
:109160003093A9044F3FFFEF5F076F077F0761F060
:10917000481B590B6A0B7B0B409311025093120250
:109180006093130270931402F8942091840030913C
:109190008500205F3F4F4A8941504A8B442341F06C
:1091A000280E391E2216330610F40C94673F01C0B6
:1091B00019013092890020928800789462960FB647
:1091C000F894DEBF0FBECDBFDF91CF911F910F91FD
:1091D000FF90EF90DF90CF90BF90AF909F908F90D7
:1091E0007F906F905F904F903F902F900895809167
:1091F0000B0180958870809309010C9473408091D5
:109200000B0188708093090167C8398930939504F0
:1092100080E288169104A104B10428F430E2832E80
:10922000912CA12CB12C30E2831A9108A108B1082D
:10923000811488E09806A104B10420F1E4E09E9E28
:10924000C0011124875B9E4EFC013296259134911A
:10925000F82DEE27F39F7001F29FE10CFE1E06949D
:10926000EE1EFE1E1124FC01C590D490860120E064
:1092700030E0480159018E189F08A108B108750116
:10928000640122C0950184013695279517950795AD
:10929000F801EC7FCF01875B924FFC01C590D49021
:1092A000FC01329625913491E82DE770E29FC001D0
:1092B000E39F900D112423E0969587952A95E1F779
:1092C000C81AD90AE12CF12C4C0D5D1D6E1D7F1DB5
:1092D0004093960450939704609398047093990474
:1092E0009091940480919304992309F473C0882386
:1092F00009F40ECDA85BBF4F8D919C91A0E0B0E02A
:1093000040910D0250910E0260910F027091100277
:1093100084179507A607B70709F05FC0F9CCB69583
:10932000A79597958795D988DD0CD98A2C5F3F4FF3
:1093300045E12536340709F04ECC59895093950400
:1093400080329105A105B10520F480E290E0A0E013
:10935000B0E08097A109B109811558E09507A105F2
:10936000B10508F443C074E0979F90011124275B76
:109370003E4EF901329645915491EE27859FB001FA
:10938000849F610D7E1F06946E1F7E1F1124F901BC
:10939000C590D490E12CF12CC61AD70AE108F10847
:1093A00080918A0490918B04A0918C04B0918D04DB
:1093B0008C0D9D1DAE1DBF1D80938A0490938B0460
:1093C000A0938C04B0938D0480919404811130C0DB
:1093D00080919304882309F49BCC1092110210927F
:1093E0001202109213021092140292CCAC01BD0131
:1093F0007695679557954795FA01EC7F9F01275B16
:10940000324FF901C590D490F901329645915491AB
:109410008770849F9001859F300D1124F3E036956D
:109420002795FA95E1F7C21AD30AE12CF12CB8CFAF
:109430008989480E511C611C711C80911C079091F8
:109440001D07481459046A047B04D8F4209193043E
:10945000222309F45DCCFC01E85BFF4F20813181C0
:10946000A90160E070E000910D0210910E022091C0
:109470000F0230911002401751076207730709F479
:1094800047CC109211021092120210921302109205
:109490001402FC01E85BFF4F80819181A0E0B0E005
:1094A00080930D0290930E02A0930F02B0931002CE
:1094B0002FCCD701C601B695A79597958795FC0146
:1094C000EC7FCF01875B924FFC0125913491FC0129
:1094D0003296459154916C2D6770649FC001659FD1
:1094E000900D112463E0969587956A95E1F7281B06
:1094F000390BC901A0E0B0E0FBCBD501C401B695A2
:10950000A79597958795FC01EC7FCF01875B924FDC
:10951000FC01C590D490FC01329625913491482DE0
:109520004770429FC001439F900D1124A3E0969580
:109530008795AA95E1F7C81AD90AE12CF12CD4CD68
:1095400080EDC82E87E0D82EE12CF12CE8CBCF920D
:10955000DF92EF92FF92CF93DF936B017C01EA01E0
:1095600021E338E040EA50EC0E94DCEC87FD23C0A8
:1095700022E430E04CE553E4C701B6010E946AE6FC
:109580001816CCF0C880D980EA80FB802FE632E143
:1095900043E85AEBC701B6010E94DCEC87FD0BC023
:1095A000C1E022E430E04CE553E4C701B6010E947B
:1095B0006AE618160CF4C0E08C2FDF91CF91FF9073
:1095C000EF90DF90CF9008950F931F93CF93DF9389
:1095D000FC01A685B7858D0100581F4FE8018881E1
:1095E000998101968F779927AD014E575F4FEA0118
:1095F0002881398128173907D1F3E8012881398179
:10960000A20FB31F6C93A685B785A058BF4F1196C4
:109610009C938E93A689B7892C9181E090E0078C6A
:1096200002C0880F991F0A94E2F7822B8C9381E085
:1096300081A30488F589E02D80818064808381E0A6
:1096400090E0DF91CF911F910F910895FC0181A1CE
:10965000882329F0A489B5898C9186FFFBCF11A2BC
:109660000895FC01A485B585FD01E058FF4F2081D8
:1096700031813296808191812817390779F0808174
:109680009181A80FB91F8C91208131812F5F3F4FAD
:109690002F7733273183208390E008958FEF9FEF5A
:1096A0000895DC011C96ED91FC911D97DF01A058F7
:1096B000BF4F2D913C91119712968D919C911197CE
:1096C0002817390739F08D919C91E80FF91F808197
:1096D00090E008958FEF9FEF0895FC012485358574
:1096E000F901E058FF4F80819181329620813181CC
:1096F00080589F4F821B930B60E870E00C949FEDA5
:109700000895089580E090E00895CF92DF92EF925F
:10971000FF92C0903602D0903702E0903802F0906D
:109720003902FC0180819181A281B381809336024C
:1097300090933702A0933802B09339020E9489CAED
:10974000C0923602D0923702E0923802F09239028B
:10975000FF90EF90DF90CF90089580919F189091A7
:10976000A018981759F0E92FF0E0E15EF74E8081DC
:109770009F5F9F779093A01890E008958FEF9FEFE1
:1097800008951F920F920FB60F9211240BB60F92ED
:109790002F938F939F93EF93FF932091A018E091C5
:1097A0009F1881E08E0F8F779091C600281729F0BF
:1097B000F0E0E15EF74E9083E82FE0939F18FF9171
:1097C000EF919F918F912F910F900BBE0F900FBE35
:1097D0000F901F9018958091250490912604009772
:1097E00031F04AE050E060E070E00C94BEE360E0ED
:1097F00070E0CB010895EFDF97FD0AC0ECDF6F3F0B
:1098000071058105910509F02CF4E5DF862F089597
:1098100080E008958FEF08958091250490912604AB
:10982000892B31F0E8DF91E0811103C090E001C0A5
:1098300091E0892F08950F931F93CF938091250472
:1098400090912604009711F1FC018F01C1912C2FFA
:109850002F7DA9F0C53411F0C536B9F7F801108293
:1098600060E070E080912504909126040E946BE2F4
:10987000F801C083562F472F382F292F0BC060E0E7
:1098800070E0CF911F910F910C946BE250E040E09B
:1098900030E020E0652F742F832F922FCF911F91FE
:1098A0000F91089581548A3108F042C0E82FF0E00A
:1098B0004091161850911718609118187091191846
:1098C00004C076956795579547958A95D2F7842F6A
:1098D000817040FF2FC0E450F84E9081992309F128
:1098E000E091EC10F091ED10E90FF11D908120ED69
:1098F000290F2A3098F09E3211F491810CC09D32CC
:1099000011F09B3271F4918120ED290F2A3030F053
:109910009E3239F4928190539A3018F42E2F9F2F53
:1099200002C020E090E0209325049093260408953F
:1099300080E008950895B6DF882341F081E020910A
:10994000250430912604232B09F480E0089580E15A
:10995000E6E3F4E0A8E2B1E101900D928A95E1F727
:1099600008952F923F924F925F926F927F928F92C3
:109970009F92AF92BF92CF92DF92EF92FF920F939E
:109980001F93CF93DF9300D01F921F92CDB7DEB706
:109990007C018B016A011901809036049090370494
:1099A000A0903804B0903904A5019401FC016081B5
:1099B0007181828193810E946AE6F1E0FD838111C9
:1099C00012C020913A0430913B0440913C045091E4
:1099D0003D04F80160817181828193810E946AE671
:1099E000811101C01D82F601408051806280738028
:1099F00020911502309116024091170250911802E1
:109A0000C301B2010E946AE6882309F453C0409260
:109A1000150250921602609217027092180220E00E
:109A200030E040E450E46091FF06709100078091BF
:109A30000107909102070E9492EB69837A838B83DE
:109A40009C838092281190922911A0922A11B092A1
:109A50002B1180913A0490913B04A0913C04B09169
:109A60003D0480932C1190932D11A0932E11B0934F
:109A70002F11F60180819181A281B38180933011F1
:109A800090933111A0933211B0933311809142041D
:109A900090914304A0914404B09145048093341103
:109AA00090933511A0933611B0933711CE010196E2
:109AB0002CDE4DDFFD81FF2309F16090FB067090E5
:109AC000FC068090FD069090FE06A090F706B090F0
:109AD000F806C090F906D090FA069501A601B301E8
:109AE000C4010E94DCEC181614F05301640120E05C
:109AF00030E040E251E4B501C6010CC020E030E0A6
:109B000040EC5FE3609103077091040780910507C3
:109B1000909106070E9492EB69837A838B839C83E2
:109B200020912404222349F0AB01BC0189E695E190
:109B30000E9464C58AE00E94CD89F70180819181ED
:109B4000A281B3818093281190932911A0932A11A7
:109B5000B0932B11F80180819181A281B381809310
:109B60002C1190932D11A0932E11B0932F11F10170
:109B7000208131814281538160913411709135117E
:109B800080913611909137110E94B6EA609334119A
:109B9000709335118093361190933711CE01019651
:109BA000B4DDD5DE0F900F900F900F900F90DF91E6
:109BB000CF911F910F91FF90EF90DF90CF90BF90CA
:109BC000AF909F908F907F906F905F904F903F905D
:109BD0002F90089580E1E8E2F1E1A6E3B4E001907E
:109BE0000D928A95E1F708959C0197FD0EC0843689
:109BF000910584F064E670E00E949FEDCB016AE07D
:109C000070E00E949FED805D06C03195219531097D
:109C10008DE201C080E2809331042A30310564F086
:109C2000EAE0F0E0C901BF010E949FEDCB01BF0156
:109C30000E949FED805D01C080E280933204C901E3
:109C40006AE070E00E949FED805D8093330481E3C1
:109C500094E00895883791051CF028E780E002C061
:109C6000282F892F20934804809349040C94BA76B6
:109C70002F923F924F925F926F927F928F929F921C
:109C8000AF92BF92CF92DF92EF92FF920F931F930A
:109C9000CF93DF93CDB7DEB7C455D1090FB6F89493
:109CA000DEBF0FBECDBFE8E2F8E184918F010F5F08
:109CB0001F4F882321F00E94CD89F801F6CF0E9422
:109CC000CDBB81110C941A5880E090E0A0E8BFE36E
:109CD0008093201190932111A0932211B09323110E
:109CE00080E090E0A0ECB0E48093241190932511E3
:109CF000A0932611B09327118DEC9CECACE4BEE34D
:109D000080931C1190931D11A0931E11B0931F11ED
:109D100080E090E0A8ECB1E48093280590932905B9
:109D2000A0932A05B0932B058CE390E09093270530
:109D30008093260588EC90E0909325058093240578
:109D4000109223058FE4F7DD882311F074DD04C041
:109D500060E070E080E190E46BAF7CAF8DAF9EAFD0
:109D600083E4E9DD882311F057DD02C083E49ADD46
:109D700061968FAF61978BE4DEDD882311F04CDDB7
:109D800002C08BE48FDD60968FAF609782E4D3DDF5
:109D90008823E9F050DD0E94FAEB70932705609369
:109DA00026056115710599F06852710965367105CE
:109DB00070F0E3EFF7E184918F010F5F1F4F88236D
:109DC00011F40C941A580E94CD89F801F4CF8CE458
:109DD000B2DD882351F12FDD6B017C0160931C11F2
:109DE00070931D1180931E1190931F1120E030E09D
:109DF000A9010E94DCEC87FD0AC020E030E040E0D1
:109E000050E4C701B6010E946AE6181674F4EBEC40
:109E1000F7E184918F010F5F1F4F882311F40C9499
:109E20001A580E94CD89F801F4CF81E53BDD8823E3
:109E300009F440C08091250490912604892B19F4DF
:109E4000E0EAF7E12BC0F7DC6B017C0160932411A1
:109E50007093251180932611909327112DEC3CECE3
:109E60004CE45DE30E94DCEC87FD0AC020E030E0BA
:109E700040E751E4C701B6010E946AE61816D4F41F
:109E8000EFE6F7E184918F010F5F1F4F882311F4F4
:109E90000C941A580E94CD89F801F4CF84918F0157
:109EA0000F5F1F4F882311F40C941A580E94CD891C
:109EB000F801F4CF83E53FDD882319F1BCDC4B01C9
:109EC0005C012DEC3CEC4CEC5DE30E94DCEC87FD8E
:109ED0000AC020E030E040E85FE3C501B4010E9421
:109EE0006AE61816ACF4E8E4F7E184918F010F5F9D
:109EF0001F4F882311F40C941A580E94CD89F80141
:109F0000F4CF5DEC852E5CEC952EA92C5EE3B52E8E
:109F100080E5C8DC882309F443C080912504909132
:109F20002604892B71F4E0E1F7E184918F010F5F42
:109F30001F4F882311F40C941A580E94CD89F80100
:109F4000F4CF809123058F5F8093230574DC6B0130
:109F50007C01609328057093290580932A059093CE
:109F60002B0520E030E0A9010E94DCEC87FD0AC04F
:109F700020E030E048EC51E4C701B6010E946AE6F7
:109F8000181674F4E8EEF6E184918F010F5F1F4F0D
:109F9000882311F40C941A580E94CD89F801F4CF4B
:109FA00086E4C9DC882319F146DC6B017C0120E0E2
:109FB00030E040E85FE30E94DCEC87FD0AC020E06F
:109FC00030E040E850E4C701B6010E946AE6181686
:109FD000A4F4EFEBF6E184918F010F5F1F4F88230C
:109FE00011F40C941A580E94CD89F801F4CFC12CB9
:109FF000D12C40EEE42E4FE3F42EA7019601C701C9
:10A00000B6010E94CFE69B01AC0160E070E084E401
:10A0100090E40E9492EB2091201130912111409107
:10A020002211509123110E94CFE62B013C01A50182
:10A030009401C501B4010E94CFE6A70196010E94D8
:10A04000CFE62CEE31E548EB5DE30E9492EB9B01FD
:10A05000AC01C301B2010E94CFE66093201170935E
:10A060002111809322119093231188E464DC8823CA
:10A07000C9F0E1DB0E94FAEB70932505609324059B
:10A08000655A71096437710568F0E1E9F6E1849178
:10A090008F010F5F1F4F882309F4CCC70E94CD8921
:10A0A000F801F5CF85E5FEDB8823E9F00E9402592F
:10A0B000611571058105910511F00E9462E28091A0
:10A0C000250490912604892B11F0B5DB04C060E0D3
:10A0D00070E088E492E460931F05709320058093FC
:10A0E00021059093220582E5DDDB81110DC0EDE5B0
:10A0F000F6E184918F010F5F1F4F882309F49AC7FF
:10A100000E94CD89F801F5CF809125049091260415
:10A11000892BA9F060DB2F967FAF6EAF2F971616B5
:10A1200017069CF0E9E2F6E184918F010F5F1F4F63
:10A13000882309F47FC70E94CD89F801F5CF8AE111
:10A1400090E02F969FAF8EAF2F9788E5F4DB8823A2
:10A1500061F071DB209118043091190440911A04C8
:10A1600050911B040E94B5EA08C0609136047091BA
:10A170003704809138049091390460931B057093E3
:10A180001C0580931D0590931E0589E5D4DB88236B
:10A1900061F051DB20911C0430911D0440911E049C
:10A1A00050911F040E94B5EA08C060913A04709172
:10A1B0003B0480913C0490913D046093170570939B
:10A1C00018058093190590931A0560911B057091ED
:10A1D0001C0580911D0590911E0547E155E0B7D9FA
:10A1E00081110DC0EFEFF5E184918F010F5F1F4FDB
:10A1F000882309F41FC70E94CD89F801F5CF84E4B4
:10A2000051DB91E089270E942DAC20E030E040EA4C
:10A2100050E460913E0470913F048091400490911D
:10A2200041040E946AE687FF14C0198A1A8A1B8AB1
:10A230001C8A80E090E0A0EAB0E489839A83AB8333
:10A24000BC83BE016F5E7F4FCE0101960E94AFBB03
:10A25000C1DCD8D76B017C01A8E8CA0EA3E1DA1EE5
:10A26000E11CF11C8091260590912705F3DC60919B
:10A27000260570912705072E000C880B990B0E946C
:10A2800070E69B01AC0160914A0470914B0480918F
:10A290004C0490914D040E94B5EA4B015C0120E012
:10A2A00030E0A9010E94DCEC87FF04C0B7FAB0944B
:10A2B000B7F8B09420E030E040E450E4C501B401C8
:10A2C0000E94DCEC1816F4F49DD7DC01CB018C194C
:10A2D0009D09AE09BF09B7FD0EC094D76B017C0183
:10A2E000B8E8CB0EB3E1DB1EE11CF11C0E94007646
:10A2F0008AE00E94CD890E9403A180919F188093DB
:10A30000A018B5CF80912405909125050E94F7599A
:10A310006091240570912505072E000C880B990B80
:10A320000E9470E69B01AC01609150047091510451
:10A3300080915204909153040E94B5EA4B015C0154
:10A3400020E030E0A9010E94DCEC87FF04C0B7FAEE
:10A35000B094B7F8B09420E030E040E450E4C50198
:10A36000B4010E94DCEC1816F4F44CD7DC01CB01EC
:10A370008C199D09AE09BF09B7FD0EC043D76B010B
:10A380007C01E8E8CE0EE3E1DE1EE11CF11C0E9438
:10A3900000768AE00E94CD890E9403A180919F18D7
:10A3A0008093A018B5CF10924204109243041092EB
:10A3B0004404109245040E947BBA809123058823AF
:10A3C00099F1C5DA209128053091290540912A0597
:10A3D00050912B0560913411709135118091361197
:10A3E000909137110E94B6EA609334117093351141
:10A3F000809336119093371120E030E040E751E42C
:10A4000060910307709104078091050790910607FA
:10A410000E9492EB69837A838B839C83CE010196A1
:10A4200074D995DA0E9488B880E2E7EFF4E0DF01A2
:10A43000282F1D922A95E9F7E7EDF4E0DF01282F98
:10A440001D922A95E9F7E7EBF4E0DF011D928A956A
:10A45000E9F77DDA80911C1190911D11A0911E11D8
:10A46000B0911F118093301190933111A09332114C
:10A47000B093331119821A821B821C829E012F5FB6
:10A480003F4F40E351E16CE271E188E291E169DA2A
:10A490009E01255C3F4F40E351E16CE271E188E2AF
:10A4A00091E15FDA6196BFAD6197BB2329F06AE362
:10A4B00074E086E394E004C067E175E08BE195E029
:10A4C0000E94BAD8298F3A8F4B8F5C8F6D8F7E8F09
:10A4D0003FAF2D962FAF2D972D96EFAD2D97E7FD22
:10A4E00081C4FFADF7FD7EC424E0E202F001112437
:10A4F000EF5FF54F40805180628073803FAD84E014
:10A500003802F0011124E351F64FD080C18032802F
:10A5100023808D2D9C2DA32DB22D8FAB98AFA9AF8D
:10A52000BAAFAE01495C5F4FB201C30110D88823B6
:10A5300009F45CC420E030E040EA50E4B201C30119
:10A540000E94B6EAF62E072F182FE92E862F902F9D
:10A55000A12FBE2D8BAB9CABADABBEAB8D2D9C2D7F
:10A56000A32DB22D8FA798ABA9ABBAAB2D969FADFB
:10A570002D97911152C0AFADA11105C05F2D402F95
:10A58000312F2E2D04C0542D452D362D272D852FEE
:10A59000942FA32FB22F8BAB9CABADABBEABBFAD9B
:10A5A000B43034F4F42C052D162DE72CBB2369F0C0
:10A5B00020E030E040EA50E46D2D7C2D832D922D7B
:10A5C0000E94B5EA362F272F03C09601832D922DC6
:10A5D000432F522FBC014FA758AB69AB7AABEFADFD
:10A5E000E4300CF0A7C020E030E040EA50E46D2DEC
:10A5F0007C2D832D922D0E94B6EA21966FAF219774
:10A6000023967FAF239725968FAF259727969FAFE9
:10A610002797FFADF11185C099C02D962FAD2D97CD
:10A6200024300CF453C03FAD34305CF020E030E017
:10A6300040EA50E4B201C3010E94B5EA362F272F49
:10A6400003C0342D252DC301432F522FBC014BAB2A
:10A650005CAB6DAB7EAB8FAD8111E3C420E030E02D
:10A6600040EA50E4B201C3010E94B5EAF62E072F7A
:10A67000182FE92E20E030E040EA50E46D2D7C2DCB
:10A68000832D922D0E94B6EA6FA778AB89AB9AAB67
:10A690009FAD992309F44EC020E030E040EA50E439
:10A6A0006D2D7C2D832D922D0E94B5EA21966FAFE2
:10A6B000219723967FAF239725968FAF25972796CF
:10A6C0009FAF2797AFADA43064F140C0BFADB111CB
:10A6D0000DC020E030E040EA50E4B201C3010E9426
:10A6E000B5EAF62E072F182FE92E0FC0EFADE43094
:10A6F000B4F120E030E040EA50E4B201C3010E942E
:10A70000B5EA6BAB7CAB8DAB9EAB2196DFAE2197F0
:10A710002396CFAE239725963FAE259727962FAE4B
:10A72000279732ED832E33E5932E3BE7A32E31E4BA
:10A73000B32E29C02196DFAE21972396CFAE239763
:10A7400025963FAE259727962FAE279722ED822E8E
:10A7500023E5922E2BEFA22E20E4B22E14C02196D8
:10A76000DFAE21972396CFAE239725963FAE259750
:10A7700027962FAE279792ED892E93E5992E9BEF82
:10A78000A92E91E4B92E8BA99CA9ADA9BEA92C969E
:10A790008CAF9DAFAEAFBFAF2C979C01AD01B201A6
:10A7A000C3010E94B5EA698B7A8B8B8B9C8B4FA47B
:10A7B00058A869A87AA8A30192016D2D7C2D832D3C
:10A7C000922D0E94B5EA6D8B7E8B8F8B988F2C9685
:10A7D0002CAD3DAD4EAD5FAD2C97609136047091C0
:10A7E000370480913804909139040E94B5EA2C9680
:10A7F0006CAF7DAF8EAF9FAF2C97A301920160919C
:10A800003A0470913B0480913C0490913D040E9475
:10A81000B5EA2B013C018F2D902FA12FBE2D8983EE
:10A820009A83AB83BC8321968FAD219723969FADEE
:10A8300023972596AFAD25972796BFAD27978D8394
:10A840009E83AF83B88780911C1190911D11A091B8
:10A850001E11B0911F1189879A87AB87BC872DEC99
:10A860003CEC4CEC5CE3C501B4010E94CFE62091C6
:10A8700020113091211140912211509123110E94F9
:10A88000CFE620914204309143044091440450911A
:10A8900045040E94B6EA6D877E878F87988B2C9639
:10A8A0002CAD3DAD4EAD5FAD2C97CA01B9010E94F4
:10A8B000CFE66B017C01A3019201C301B2010E94AA
:10A8C000CFE69B01AC01C701B6010E94B6EA20E0C9
:10A8D00030E040E050E40E94DCEC18160CF046C07A
:10A8E0000E9488B81BA21CA21DA21EA220E030E07C
:10A8F00040E05FE360913E0470913F04809140042A
:10A90000909141040E94B6EA6F8F78A389A39AA31D
:10A910009E012D5D3F4FAE01415E5F4F6AE374E0E3
:10A9200086E394E01ED81BA21CA21DA21EA220E05A
:10A9300030E040E05FE360911C1170911D11809147
:10A940001E1190911F110E94B6EA6F8F78A389A300
:10A950009AA39E012D5D3F4FAE01415E5F4FBE0148
:10A96000615D7F4FCE01C3960E94B14C1F8E18A22D
:10A9700019A21AA29E01215E3F4F4CE151E1BE0196
:10A98000615D7F4FCE01C3960E94B14C0E94B4B866
:10A990004090360250903702609038027090390231
:10A9A000E090FB06F090FC060091FD061091FE067B
:10A9B000A090F706B090F806C090F906D090FA067D
:10A9C0009501A601B701C8010E94DCEC181614F429
:10A9D0007501860120E030E040E251E4B701C80192
:10A9E0000E9492EB60933602709337028093380294
:10A9F0009093390240E0BE016F5E7F4FCE01019619
:10AA00000E94CFA4409236025092370260923802E0
:10AA1000709239020E94A74CA1E0BAE02496BFAF21
:10AA2000AEAF249722961FAE1EAE229701E010E033
:10AA300021960FAC219702C0000F111F0A94E2F774
:10AA40002296EEADFFAD229731962296FFAFEEAF84
:10AA5000229721E030E021960FAC219702C0220F0F
:10AA6000331F0A94E2F763963FAF2EAF639787EBED
:10AA7000282E84E0382E87EF94E02A969FAF8EAF81
:10AA80002A97A7EDB4E02896BFAFAEAF2897EDEEBA
:10AA9000F9E02696FFAFEEAF26972A962EAD3FAD92
:10AAA0002A9765963FAF2EAF6597D9018D919C91FE
:10AAB0009C0120233123232B09F4ADC06396EEAD16
:10AAC000FFAD63978E239F23892B09F4A4C028969A
:10AAD000AEADBFAD28978D919C9180239123892B9A
:10AAE00009F099C020E030E040E050E42496AEAD9B
:10AAF000BFAD24976D917D918D919C910E94B6EA96
:10AB00006B017C0120E030E040E050E42496EEADA3
:10AB1000FFAD249764817581868197810E94B5EA93
:10AB20004B015C0120E030E040E850ECC701B60189
:10AB30000E946AE687FD70C120E030E04BE553E4F7
:10AB4000C701B6010E94DCEC181634F4C12CD12CDC
:10AB5000BBE5EB2EB3E4FB2ECBA6DCA6EDA6FEA652
:10AB60002696AEADBFAD26974D905D906D907C90D2
:10AB700020E030E040E85FE3C301B2010E946AE6F2
:10AB800087FD51C120E030E04BE553E4C301B20141
:10AB90000E94DCEC181634F4412C512CFBE56F2E8E
:10ABA000F3E47F2E4F8E58A269A27AA24FA258A634
:10ABB00069A67AA620E030E040E850ECC501B40177
:10ABC0000E946AE687FD36C120E030E04BE553E4A1
:10ABD000C501B4010E94DCEC181634F4812C912CD0
:10ABE0007BE5A72E73E4B72E8BA29CA2ADA2BEA2DA
:10ABF000AE01495D5F4FC701B6010E94A74A8111AE
:10AC000020C12896EEADFFAD289780819181802BE1
:10AC1000912B918380832A962EAD3FAD2A972E5F8C
:10AC20003F4F2A963FAF2EAF2A976596AEADBFAD88
:10AC300065978D919C9180239123892B09F4A6C05F
:10AC4000F9018081918180239123892B09F49EC091
:10AC5000F1018081918180239123892B09F096C095
:10AC600020E030E040E050E42696AEADBFAD269740
:10AC70006D917D918D919C910E94B6EA2B013C01D2
:10AC800020E030E040E050E42696EEADFFAD2697A0
:10AC900064817581868197810E94B5EA4B015C01D0
:10ACA0002496AEADBFAD2497CD90DD90ED90FC9095
:10ACB00020E030E040E850ECC701B6010E946AE6AF
:10ACC00087FDFFC020E030E04BE553E4C701B6014B
:10ACD0000E94DCEC181634F4C12CD12C5BE5E52E77
:10ACE00053E4F52ECBA2DCA2EDA2FEA2CBA6DCA6FD
:10ACF000EDA6FEA620E030E040E85FE3C301B2012C
:10AD00000E946AE687FDE4C020E030E04BE553E4B2
:10AD1000C301B2010E94DCEC181634F4412C512C12
:10AD20003BE5632E33E4732E4FA258A669A67AA69C
:10AD300020E030E040E85FE3C501B4010E946AE62C
:10AD400087FDCDC020E030E04BE553E4C501B40100
:10AD50000E94DCEC181634F4812C912C9BE5A92E72
:10AD600093E4B92E8F8E98A2A9A2BAA2AE01495D32
:10AD70005F4FC701B6010E94A74A8111B7C0F10118
:10AD800080819181802B912B91838083F2E02F0E23
:10AD9000311C28962EAD3FAD28972E5F3F4F289649
:10ADA0003FAF2EAF289726968EAD9FAD269704967F
:10ADB00026969FAF8EAF269791EC291694E0390620
:10ADC00009F06BCE2496AEADBFAD249714962496B1
:10ADD000BFAFAEAF24972296EEADFFAD2297359769
:10ADE00009F024CE80919F188093A0182F962EAD45
:10ADF0003FAD2F97215031092F963FAF2EAF2F97A0
:10AE0000232B09F4B3C02D963FAD2D9737FDAEC06F
:10AE10008FAD87FF47CBAAC0C12CD12CA0E8EA2E6A
:10AE2000A0ECFA2E99CE412C512CE0E86E2EEFE3E7
:10AE30007E2EB8CE812C912C60E8A62E60ECB62E2A
:10AE4000D3CEAE01415E5F4FC501B4010E94A74A57
:10AE5000882309F4D6CE80912404882321F1B701F8
:10AE6000A60189ED95E10E9464C54FA158A569A589
:10AE70007AA583ED95E10E9464C54BA15CA16DA10B
:10AE80007EA189EC95E10E9464C54F8D58A169A10E
:10AE90007AA183EC95E10E9464C589E20E94CD8984
:10AEA0008AE00E94CD899E01215E3F4FAE014D5D3B
:10AEB0005F4FBE01695D7F4FCE018B960E94E4B863
:10AEC000A0CEC12CD12C40E8E42E40ECF42E0ACFC9
:10AED000412C512C20E8622E2FE3722E25CF812C9D
:10AEE000912C80E8A82E8FE3B82E3CCFAE01415EB6
:10AEF0005F4FC701B6010E94A74A882309F43FCFDC
:10AF000080912404882321F1B701A6018FE995E1FE
:10AF10000E9464C54FA158A569A57AA589E995E164
:10AF20000E9464C54BA15CA16DA17EA18FE895E153
:10AF30000E9464C54F8D58A169A17AA189E895E165
:10AF40000E9464C589E20E94CD898AE00E94CD8971
:10AF50009E01215E3F4FAE014D5D5F4FBE01695DB9
:10AF60007F4FCE018B960E94E4B809CF0E9488B82B
:10AF700080E090E0A0EAB0E480933011909331112A
:10AF8000A0933211B093331119821A821B821C8252
:10AF90009E012F5F3F4F40E351E16CE271E188E297
:10AFA00091E10E94B14C80911B0590911C05A091EC
:10AFB0001D05B0911E058093281190932911A0932F
:10AFC0002A11B0932B118091170590911805A0912B
:10AFD0001905B0911A0580932C1190932D11A0930F
:10AFE0002E11B0932F1119821A821B821C829E018E
:10AFF0002F5F3F4F40E351E16CE271E188E291E164
:10B000000E94B14C6096FFAD6097F11113C0109291
:10B010004904109248040E94BA7680E090E0E7D19B
:10B0200009C02FADF42C052D162DE72C24300CF083
:10B0300033CB20CBCC5ADF4F0FB6F894DEBF0FBE18
:10B04000CDBFDF91CF911F910F91FF90EF90DF90D7
:10B05000CF90BF90AF909F908F907F906F905F90B8
:10B060004F903F902F9008951F920F920FB60F921E
:10B0700011240BB60F922F933F938F939F93EF93CF
:10B08000FF932091160F3091170F8091180F909118
:10B09000190F2817390731F4809131018F7D809382
:10B0A000310114C0E091180FF091190FEA56F14FD9
:10B0B00020818091180F9091190F01968F77992711
:10B0C0009093190F8093180F20933601FF91EF9101
:10B0D0009F918F913F912F910F900BBE0F900FBEBC
:10B0E0000F901F9018951F920F920FB60F92112478
:10B0F0000BB60F922F934F935F938F939F93EF9382
:10B10000FF938091300182FD1CC020913601809117
:10B110009A0F90919B0F40919C0F50919D0F01961B
:10B120008F7799274817590771F0E0919A0FF0919E
:10B130009B0FE65EF04F208390939B0F80939A0FB6
:10B1400002C080913601FF91EF919F918F915F91A5
:10B150004F912F910F900BBE0F900FBE0F901F902D
:10B160001895CF92DF92EF92FF920F931F93CF9398
:10B17000DF936C017A018B01C0E0D0E0CE15DF05D2
:10B1800081F0D8016D918D01D601ED91FC91019076
:10B19000F081E02DC6011995892B11F02196EECF93
:10B1A0007E01C701DF91CF911F910F91FF90EF902A
:10B1B000DF90CF9008950E94C6ED3FB7F89480913C
:10B1C000D3069091D406A091D506B091D60626B5A7
:10B1D000A89B05C02F3F19F00196A11DB11D3FBFCF
:10B1E000BA2FA92F982F8827820F911DA11DB11D5D
:10B1F000BC01CD0142E0660F771F881F991F4A9559
:10B20000D1F708952FB7F8946091CF067091D006CA
:10B210008091D1069091D2062FBF08951F920F9270
:10B220000FB60F9211242F933F938F939F93AF9359
:10B23000BF938091CF069091D006A091D106B09196
:10B24000D2063091CE0623E0230F2D3720F401964D
:10B25000A11DB11D05C026E8230F0296A11DB11D39
:10B260002093CE068093CF069093D006A093D1066C
:10B27000B093D2068091D3069091D406A091D506C2
:10B28000B091D6060196A11DB11D8093D30690936F
:10B29000D406A093D506B093D606BF91AF919F91E7
:10B2A0008F913F912F910F900FBE0F901F90189587
:10B2B0001F920F920FB60F9211240BB60F922F937D
:10B2C0003F934F935F936F937F938F939F93AF932E
:10B2D000BF93EF93FF9380912F0590913005A0913C
:10B2E0003105B0913205892B8A2B8B2B59F1909126
:10B2F0002E05E0912C05F0912D0580818927808312
:10B3000080912F0590913005A0913105B0913205C3
:10B31000181619061A061B060CF056C080912F0548
:10B3200090913005A0913105B09132050197A109A6
:10B33000B10980932F0590933005A0933105B09308
:10B34000320542C080911902E5E5F8E1E4919FEFF2
:10B3500090931902E230C9F050F4EE2399F0E130F5
:10B3600081F590916F009D7F90936F002AC0E4302B
:10B3700019F1E0F0E53029F5909173009D7F9093ED
:10B3800073001FC010926E001CC0909170009D7FD2
:10B390009093700091E09093B0009091B100987FED
:10B3A00094609093B1001092B3000BC09091710023
:10B3B0009D7F9093710005C0909172009D7F909346
:10B3C000720060E00E9443BDFF91EF91BF91AF9189
:10B3D0009F918F917F916F915F914F913F912F91AD
:10B3E0000F900BBE0F900FBE0F901F90189590936B
:10B3F0004F0480934E0480E00C9406772F923F9286
:10B400004F925F926F927F928F929F92AF92BF9274
:10B41000CF92DF92EF92FF920F931F93CF93DF9320
:10B42000CDB7DEB7C857D1090FB6F894DEBF0FBE4F
:10B43000CDBFE0914E07F0914F07EF2B11F00C9428
:10B44000BE622896DFAECEAE28976E2C79016A01D7
:10B450005B01FC0120813181428153816C962CAFCC
:10B460003DAF4EAF5FAF6C9720910C1130910D1135
:10B4700040910E1150910F116C966CAD7DAD8EAD5B
:10B480009FAD6C970E94CFE60E94E7ECE0966CAF10
:10B490007DAF8EAF9FAFE097D5018D919D910D90BF
:10B4A000BC91A02DA0968CAF9DAFAEAFBFAFA097C3
:10B4B00020911011309111114091121150911311DE
:10B4C000BC01CD010E94CFE60E94E7ECE4966CAF90
:10B4D0007DAF8EAF9FAFE497D6012D913D914D91F9
:10B4E0005C91A4962CAF3DAF4EAF5FAFA497209177
:10B4F0001411309115114091161150911711A49605
:10B500006CAD7DAD8EAD9FADA4970E94CFE60E943D
:10B51000E7ECE8966CAF7DAF8EAF9FAFE897D701B1
:10B520002D913D914D915C9122962CAF3DAF4EAF48
:10B530005FAF2297209118113091191140911A1183
:10B5400050911B1122966CAD7DAD8EAD9FAD2297B3
:10B550000E94CFE60E94E7EC60966CAF7DAF8EAFA5
:10B560009FAF60978091140783FF1CC060962CAD3D
:10B570003DAD4EAD5FAD60972093E9093093EA0988
:10B580004093EB095093EC0922968CAD9DADAEAD86
:10B59000BFAD22978093D9099093DA09A093DB0974
:10B5A000B093DC09D801BC91B9A7F801F181F9ABDE
:10B5B000D8011296BC91BEABF801F381FAAF80912D
:10B5C000B7099091B809891B8F708F3019F40E94C8
:10B5D00003A1F5CF0091B709E9960FAFE9978091E4
:10B5E000B709082F10E01CA30BA38091DD099091EF
:10B5F000DE09A091DF09B091E009E0968CAC9DAC2A
:10B60000AEACBFACE097881A990AAA0ABB0A80912F
:10B61000E1099091E209A091E309B091E409E4966F
:10B620002CAC3DAC4EAC5FACE497281A390A4A0A00
:10B630005B0A8091E5099091E609A091E709B09134
:10B64000E809E8962CAD3DAD4EAD5FADE897281BFF
:10B65000390B4A0B5B0B2DA33EA34FA358A7809138
:10B66000E9099091EA09A091EB09B091EC09609683
:10B670000CAD1DAD2EAD3FAD6097081B190B2A0B0D
:10B680003B0B0DA71EA72FA738AB012B022B032BBB
:10B6900009F4BCC08091130781114BC06091500424
:10B6A0007091510480915204909153040E94FAEBDE
:10B6B0002091250230912602621773070CF039C0E1
:10B6C00060962CAD3DAD4EAD5FAD60972093E9091E
:10B6D0003093EA094093EB095093EC0922968CAD24
:10B6E0009DADAEADBFAD22978093D9099093DA0995
:10B6F000A093DB09B093DC09E2EFFDE184918F01B7
:10B700000F5F1F4F811103C0E9ECF9E104C00E94F3
:10B71000CD89F801F3CF84918F010F5F1F4F8823EC
:10B7200021F00E94CD89F801F6CF1DA61EA61FA606
:10B7300018AA94E0699E800111240F5D1D4F6DA52C
:10B740007EA58FA598A90E9470E6D8012D913D9104
:10B750004D915C910E94CFE66B017C0120E030E0CE
:10B76000A9010E94DCEC87FF04C0F7FAF094F7F817
:10B77000F094609118117091191180911A119091A3
:10B780001B110E94FAEB9B01AC01A8ECB0E00E94F7
:10B7900096EA0E9470E6A70196010E946AE687FF7A
:10B7A00039C060960CAD1DAD2EAD3FAD60970093D6
:10B7B000E9091093EA092093EB093093EC092296EA
:10B7C0002CAD3DAD4EAD5FAD22972093D90930939E
:10B7D000DA094093DB095093DC09E2EFFDE1849143
:10B7E0008F010F5F1F4F811103C0EAEAF9E104C026
:10B7F0000E94CD89F801F3CF84918F010F5F1F4F15
:10B80000882321F00E94CD89F801F6CF1DA61EA63F
:10B810001FA618AAD501C4018827B7FD83959927CB
:10B82000AA27BB27782E57FE03C0382F3260732E0D
:10B830008DA19EA1AFA1B8A5B7FF03C0972D9460BD
:10B84000792E0DA51EA52FA538A937FF03C0172DEA
:10B850001860712E24E0629E800111240F5D1D4F3F
:10B860006DA57EA58FA598A90E9470E6D8012D919F
:10B870003D914D915C910E94CFE66B017C0120E0EF
:10B8800030E0A9010E94DCEC87FF04C0C701B601CB
:10B89000905802C0C701B60120E030E040E05FE30D
:10B8A0000E94B6EA0E94FFEB6AAB7BAB8CAB9DAB10
:10B8B00088E60BA11CA1809FF001819FF00D11244F
:10B8C000E858FE4E1082EA5BFF4F7082B501A4017A
:10B8D000B7FE07C044275527BA01481959096A0914
:10B8E0007B0988E60BA11CA1809FF001819FF00DD0
:10B8F0001124E858FE4E458B568B678B708F2C9623
:10B900002CAE3DAE4EAE5FAE2C9757FE0DC08827D5
:10B910009927DC0182199309A409B5092C968CAFEB
:10B920009DAFAEAFBFAF2C9728E60BA11CA1209F07
:10B93000F001219FF00D1124E858FE4E2C968CAD9D
:10B940009DADAEADBFAD2C97818F928FA38FB48F7D
:10B950000DA11EA12FA138A537FF07C03095209556
:10B96000109501951F4F2F4F3F4FE8E67E2EABA15C
:10B97000BCA17A9EF0017B9EF00D1124E858FE4E8A
:10B98000058F168F278F30A38AA99BA9ACA9BDA9C3
:10B9900081A392A3A3A3B4A323964FAF2397752E9D
:10B9A000F62FE72F2C968CAD9DADAEADBFAD2C978D
:10B9B000481759076A077B0778F429969FAD29979E
:10B9C00023969FAF23972A967FAC2A972B96FFAD9D
:10B9D0002B972C96EFAD2C9723968FAD2397972D11
:10B9E000AF2FBE2F80179107A207B30710F4D9011C
:10B9F000C8010AA91BA92CA93DA980179107A20774
:10BA0000B30710F4D901C80128E60BA11CA1209F9F
:10BA1000F001219FF00D1124E858FE4E85A396A356
:10BA2000A7A3B0A70697A105B10508F4A0C5DF013B
:10BA3000AE59BF4F80914604909147048D939C93DB
:10BA400061A6452B462B472B09F05F9888E60BA192
:10BA50001CA1809FF001819FF00D1124E858FE4E3B
:10BA6000818D928DA38DB48D892B8A2B8B2B11F018
:10BA70008A98479888E60BA11CA1809FF001819FBE
:10BA8000F00D1124E858FE4E858D968DA78DB0A13E
:10BA9000892B8A2B8B2B31F0809108018170809348
:10BAA000060147982AA93BA94CA95DA9232B242B61
:10BAB000252B09F465C580911907882319F0815059
:10BAC00080931907611004C0129880E280931907CF
:10BAD00060900F07709010070091110710911207E6
:10BAE0009301A80169A579A98EA99AAD0E946AE679
:10BAF00087FF04C069A679AA0EAB1AAFC501B401CD
:10BB00000E9470E6209168113091691140916A118C
:10BB100050916B110E94CFE626966CAF7DAF8EAF31
:10BB20009FAF2697698B7A8B8B8B9C8BC201B1015F
:10BB30000E9470E620916C1130916D1140916E1150
:10BB400050916F110E94CFE62B013C016D8B7E8BD3
:10BB50008F8B988F6DA17EA18FA198A50E9470E612
:10BB600020917011309171114091721150917311A7
:10BB70000E94CFE64B015C01698F7A8F8B8F9C8F7F
:10BB80002091741130917511409176115091771177
:10BB9000C701B6010E94CFE66B017C016D8F7E8FDD
:10BBA0008F8F98A388E60BA11CA1809FF001819F35
:10BBB000F00D1124E858FE4E258936894789508DAD
:10BBC0002DA33EA34FA358A72630310541055105AB
:10BBD00008F4DFC42896AEADBFAD2897CD90DD90B8
:10BBE000ED90FC9020E030E0A901C701B6010E9471
:10BBF0006AE68111EDC426962CAD3DAD4EAD5FAD2C
:10BC00002697CA01B9010E94CFE66B017C01A3010E
:10BC10009201C301B2010E94CFE69B01AC01C701B2
:10BC2000B6010E94B6EA6B017C01A5019401C50131
:10BC3000B4010E94CFE69B01AC01C701B6010E948E
:10BC4000B6EA0E9421ED28E60BA11CA1209FF0017D
:10BC5000219FF00D1124E858FE4E6587768787876F
:10BC6000908B88E60BA11CA1809FF001819FF00DB5
:10BC70001124E858FE4E4584568467847088A301D9
:10BC8000920160E070E080E89FE30E9492EB64968E
:10BC90006CAF7DAF8EAF9FAF649729A539A94EA930
:10BCA0005AAD0E94CFE64B015C018091B70990919B
:10BCB000B509891B8F7027968FAF2797A50194012F
:10BCC00060E074E284E799E40E9492EB0E94E7EC62
:10BCD0006B017C0127968FAD27978250863008F440
:10BCE00086C4A5019401C301B2010E94CFE69B0165
:10BCF000AC010E94CFE668966CAF7DAF8EAF9FAF70
:10BD0000689788E6ABA1BCA18A9F80018B9F100D2C
:10BD1000112408581E4E68962CAD3DAD4EAD5FAD5A
:10BD20006897D80111962D933D934D935C9314978A
:10BD300095962D913D914D915C9198972EAB3FAB8F
:10BD400048AF59AFCA01B9010E946EE66AAF7BAF36
:10BD50008CAF9DAF9B01AC01C501B4010E94CFE641
:10BD60000E947CEB0E94FFEBA8966CAF7DAF8EAF7C
:10BD70009FAFA897F801EE5AFF4F608371838283CB
:10BD800093838E010F5E1F4F2A961FAF0EAF2A9727
:10BD90000051110924961FAF0EAF249707EF16E04C
:10BDA000AC961FAF0EAFAC978E010F5D1F4F1AA35D
:10BDB00009A324960EAD1FAD2497AA961FAF0EAF10
:10BDC000AA97312C212C10E819A70FE309AB2A966A
:10BDD000AEADBFAD2A972D913D914D915D912A96C3
:10BDE000BFAFAEAF2A97C501B4010E94CFE66B0189
:10BDF0007C01AA96EEADFFADAA97619371938193F2
:10BE00009193AA96FFAFEEAFAA9720E030E0A90188
:10BE10000E94DCEC87FF04C0F7FAF094F7F8F09486
:10BE2000AC96AEADBFADAC974D905D906D907D90F2
:10BE3000AC96BFAFAEAFAC97A7019601C301B201FC
:10BE40000E946AE687FD0DC409A11AA12A962EADAB
:10BE50003FAD2A970217130709F0B9CF20E030E071
:10BE600040E85FE3632D722D89A599A90E946AE6D7
:10BE700087FF58C07E0131E1E30EF11C24960EAD20
:10BE80001FAD2497232D322D49A559A9D8016D91B5
:10BE90007D918D919C910E94CFE6F8016193719301
:10BEA000819391938F01EE16FF0661F728E60BA1AF
:10BEB0001CA1209FC001219F900D11249C01285896
:10BEC0003E4E790189010E5A1F4FA8966CAD7DAD8B
:10BED0008EAD9FADA8970E946EE6232D322D49A509
:10BEE00059A90E94CFE60E94FFEBD8016D937D9384
:10BEF0008D939C931397232D322D49A559A9632D1A
:10BF0000722D89A599A90E94CFE668962CAD3DAD0A
:10BF10004EAD5FAD68970E94CFE6F70161837283F3
:10BF2000838394832AAD3BAD4CAD5DAD64966CAD1F
:10BF30007DAD8EAD9FAD64970E94CFE669A77AA7CD
:10BF40008BA79CA70DA11EA12FA138A5012B022B09
:10BF5000032B09F09EC388E62BA13CA1829F8001A0
:10BF6000839F100D112408581E4EF801818D928D6B
:10BF7000A38DB48D892B8A2B8B2B09F08AC3858DD9
:10BF8000968DA78DB0A1892B8A2B8B2B09F081C3AD
:10BF90002091F3063091F4064091F5065091F60693
:10BFA00069A57AA58BA59CA50E94CFE60E947CEB93
:10BFB0000E94FFEB2B013C01F801E95BFF4F10826F
:10BFC00088E62BA13CA1829F8001839F100D112444
:10BFD00008581E4EF801E25AFF4F40825182628299
:10BFE0007382C301B2010E946EE629A53AA54BA552
:10BFF0005CA50E9492EB6AAF7BAF8CAF9DAFD8017E
:10C0000051966D937D938D939C935497F801E95BC2
:10C01000FF4F8081882381F17801B8E4EB0EF11C99
:10C0200037962091E7063091E8064091E906509155
:10C03000EA0660817181828193810E94CFE62AADF8
:10C040003BAD4CAD5DAD0E94CFE620911811309113
:10C05000191140911A1150911B110E94CFE69B01BA
:10C06000AC0160E074E284EF99E40E9492EB0E94DC
:10C07000FFEBF7017183608388E60BA11CA1809F11
:10C08000F001819FF00D1124E858FE4E218132818C
:10C09000438154812C962CAF3DAF4EAF5FAF2C97B0
:10C0A000CA01B9010E9421ED362E272E8C0147EDE1
:10C0B00056E062965FAF4EAF62973E0151E1650E6A
:10C0C000711C87ED96E09FAB8EAB24964EAC5FACB7
:10C0D00024973DA62DA209A719AB1AAAD201CD908B
:10C0E000DD90ED90FD902D0120E030E0A901C70129
:10C0F000B6010E94DCEC87FF04C0F7FAF094F7F871
:10C10000F094EEA9FFA981909190A190B190FFAB1E
:10C11000EEABA7019601C501B4010E946AE687FD56
:10C12000D8C564147504D1F627965FAD27975523BB
:10C1300009F448C6C090B909D090BA09E090BB098B
:10C14000F090BC092DEB37E346E855E3C701B60193
:10C150000E946AE687FD36C6C701B6010E9421ED3E
:10C160006B017C019B01AC01632D722DC8010E9403
:10C170006AE687FD03C03C2C2D2C87019601A701A0
:10C18000632D722DC8010E9492EB68966CAF7DAF53
:10C190008EAF9FAF68978DEB99E028969FAF8EAFDB
:10C1A000289720E030E040E85FE32AAB3BAB4CABA4
:10C1B0005DAB1EAA2896AEADBFAD28972D913D91DF
:10C1C0004D915D912896BFAFAEAF289768966CAD44
:10C1D0007DAD8EAD9FAD68970E94CFE64B015C01AF
:10C1E0002496EEADFFAD2497C190D190E190F190EF
:10C1F0002496FFAFEEAF2497FEA9FF2391F02AA962
:10C200003BA94CA95DA90E94CFE64B015C012AA97C
:10C210003BA94CA95DA9C701B6010E94CFE66B01FD
:10C220007C01A7019601C501B4010E94DCEC20E06D
:10C2300030E0A90118160CF092C5C701B6010E94A2
:10C24000DCEC18160CF486C520E030E0A901C5012D
:10C25000B4010E946AE687FD7DC52601370177FAA1
:10C26000709477F87094A3019201C501B4010E9403
:10C27000DCEC181614F4240135016296AEADBFADA6
:10C280006297CD90DD90ED90FD906296BFAFAEAF1E
:10C290006297A3019201C701B6010E946AE687FF77
:10C2A00015C0A3019201C701B6010E9492EB9B0148
:10C2B000AC016AA97BA98CA99DA90E94CFE66AABB3
:10C2C0007BAB8CAB9DABBEA9BF5FBEABEDECF9E029
:10C2D00028962EAD3FAD2897E217F30709F06ACFF5
:10C2E0003EA9332361F02AA93BA94CA95DA9632D7E
:10C2F000722DC8010E94CFE6362E272E8C0124EA2B
:10C3000030E74DE75FE3632D722DC8010E94CFE651
:10C310006B017C012091150730911607409117079A
:10C32000509118070E946AE687FD42C58DA59DA120
:10C33000A9A5B9A98093150790931607A09317078D
:10C34000B093180728E64BA15CA1249FC001259F4C
:10C35000900D1124DC01A858BE4E7D01232D322DF5
:10C36000A801632D722DC8010E94CFE6F7016187F5
:10C370007287838794876AAD7BAD8CAD9DAD9058F5
:10C380009B01AC010E94B6EAD7011D962D913D910B
:10C390004D915C9150970E94CFE69B01AC016BE000
:10C3A00077ED83E29BE30E94B5EA9B01AC018BE051
:10C3B00097EDA3E2BBE3F70185839683A783B0875C
:10C3C00010812C966CAD7DAD8EAD9FAD2C970E94EB
:10C3D0006AE618160CF4FBC483E0182B88E62BA140
:10C3E0003CA1829FF001839FF00D1124E858FE4E7E
:10C3F000108380E1FE013196ADEBB9E001900D9222
:10C400008A95E1F72C968CAD9DADAEADBFAD2C9766
:10C410008093B9099093BA09A093BB09B093BC0962
:10C42000E0960CAD1DAD2EAD3FADE0970093DD095C
:10C430001093DE092093DF093093E009E4962CADD8
:10C440003DAD4EAD5FADE4972093E1093093E20935
:10C450004093E3095093E409E8968CAD9DADAEADF1
:10C46000BFADE8978093E5099093E609A093E709AB
:10C47000B093E80960960CAD1DAD2EAD3FAD609751
:10C480000093E9091093EA092093EB093093EC0932
:10C490006C962CAD3DAD4EAD5FAD6C972093CD0944
:10C4A0003093CE094093CF095093D009A0968CAD1C
:10C4B0009DADAEADBFADA0978093D1099093D20949
:10C4C000A093D309B093D409A4960CAD1DAD2EADA5
:10C4D0003FADA4970093D5091093D6092093D709AF
:10C4E0003093D80922962CAD3DAD4EAD5FAD22976D
:10C4F0002093D9093093DA094093DB095093DC0982
:10C500009091B7098091B809981303C084E680938D
:10C51000B409E9968FADE9978F5F8F708093B70963
:10C520008091B7099091B60981508F70891351C4D9
:10C530001091B8091BA30091B7090DA728E61BA10C
:10C540000DA51013D1C4812C912CA12CB12C1DA2AE
:10C5500019A619AA1EAE212C312C00E010E02DA541
:10C560003BA12313CEC42114310409F07FC580916F
:10C570006F00826080936F0081E0ECC680E0EAC6C5
:10C5800060900B0770900C0700910D0710910E073B
:10C59000A7CA818D928DA38DB48D0697A105B10593
:10C5A00008F018CB858D968DA78DB0A10697A105B3
:10C5B000B10508F00FCB20E030E0A901C701B601BA
:10C5C0000E94DCEC87FF04C0F7FAF094F7F8F094CF
:10C5D00088E60BA11CA1809FF001819FF00D112422
:10C5E000E858FE4EC586D686E786F08A3ACB80911B
:10C5F000070790910807A0910907B0910A07C8168C
:10C60000D906EA06FB0608F06CCB8C199D09AE0929
:10C61000BF09BC01CD01660F771F881F991F2796A0
:10C620004FAD2797042F10E020E030E0A9019801DA
:10C630000E9458EACA01B9010E946EE60E94E7EC26
:10C640006C0D7D1D8E1D9F1D0E946EE69B01AC0131
:10C6500060E074E284E799E40E9492EB4B015C0194
:10C6600040CBA7019601C301B2010E9492EB7B016E
:10C670008C019B01AC01632D722D89A599A90E94A3
:10C68000DCEC18160CF0E0CB3E2C2F2C09A719ABD4
:10C69000DBCB0AA91BA92CA93DA9012B022B032B3B
:10C6A00049F02091EF063091F0064091F10650914B
:10C6B000F20608C02091EB063091EC064091ED06A1
:10C6C0005091EE0669A57AA58BA59CA50E94CFE6A0
:10C6D0000E947CEB0E94FFEB2B013C012AA93BA9A5
:10C6E0004CA95DA9232B242B252BC9F020E030E099
:10C6F000A9016091E7067091E8068091E9069091A2
:10C70000EA060E946AE6882351F081E00DA51EA585
:10C710002FA538A910161106120613060CF080E09A
:10C7200098E62BA13CA1929F8001939F100D1124AC
:10C7300008581E4E180137E4230E311CD1018C938A
:10C74000882309F4B3C02091CD093091CE094091DE
:10C75000CF095091D0096C966CAD7DAD8EAD9FAD7B
:10C760006C970E94B5EA6DA77EA78FA798AB209122
:10C77000D1093091D2094091D3095091D409A096A2
:10C780006CAD7DAD8EAD9FADA0970E94B5EA4B011B
:10C790005C012091D5093091D6094091D70950917B
:10C7A000D809A4966CAD7DAD8EAD9FADA4970E94C7
:10C7B000B5EA6B017C012DA53EA54FA558A9CA017C
:10C7C000B9010E94CFE66DA77EA78FA798ABA50100
:10C7D0009401C501B4010E94CFE69B01AC016DA597
:10C7E0007EA58FA598A90E94B6EA4B015C01A7011E
:10C7F0009601C701B6010E94CFE69B01AC01C501BD
:10C80000B4010E94B6EA0E9421ED6B017C012091E7
:10C81000D9093091DA094091DB095091DC0922965F
:10C820006CAD7DAD8EAD9FAD22970E94B5EAA7019C
:10C8300096010E9492EB6B017C01F801E25BFF4FD5
:10C84000608371838283938320E030E040E450E48E
:10C850000E94DCEC18161CF4F101108227C0209114
:10C86000E7063091E8064091E9065091EA06C701D3
:10C87000B6010E94CFE69B01AC016091E306709186
:10C88000E4068091E5069091E6060E9492EB29A5C8
:10C890003AA54BA55CA50E94CFE60E94FFEB64156C
:10C8A00075058605970510F42B013C018091441114
:10C8B00090914511A0914611B09147110EA91FA961
:10C8C00028AD39AD80179107A207B30708F4DFC080
:10C8D0002DA13EA14FA158A5232B242B252B41F19F
:10C8E000609148117091491180914A1190914B11BA
:10C8F0006415750586059705D8F42EA93FA948AD9E
:10C9000059AD0E9449EA6B017C012DA13EA14FA1C6
:10C9100058A5C301B2010E9449EAC616D706E80627
:10C92000F90630F4C701B6010E9458EA29013A011C
:10C9300088E60BA11CA1809FF001819FF00D1124BE
:10C94000E858FE4EC18CD28CE38CF48CC114D10417
:10C95000E104F10431F160914C1170914D1180911D
:10C960004E1190914F116415750586059705C8F411
:10C970002EA93FA948AD59AD0E9449EA4B015C017F
:10C98000A7019601C301B2010E9449EA86169706E3
:10C99000A806B90630F4C501B4010E9458EA29017D
:10C9A0003A0188E60BA11CA1809FF001819FF00D48
:10C9B0001124E858FE4EC58CD68CE78CF0A0C1142B
:10C9C000D104E104F10431F16091501170915111E1
:10C9D0008091521190915311641575058605970544
:10C9E000C8F42EA93FA948AD59AD0E9449EA4B01B0
:10C9F0005C01A7019601C301B2010E9449EA8616B3
:10CA00009706A806B90630F4C501B4010E9458EA99
:10CA100029013A0188E60BA11CA1809FF001819FAA
:10CA2000F00D1124E858FE4EC1A0D2A0E3A0F4A05E
:10CA3000C114D104E104F10409F4C2CA6091541193
:10CA4000709155118091561190915711641575058B
:10CA50008605970508F0B4CA2EA93FA948AD59AD7F
:10CA60000E9449EA4B015C01A7019601C301B20192
:10CA70000E9449EA86169706A806B90608F0A0CAD9
:10CA8000C501B4010E9458EA29013A0199CA2DA1B1
:10CA90003EA14FA158A5232B242B252BC9F1609132
:10CAA00048117091491180914A1190914B11641570
:10CAB00075058605970560F50E946EE62AAD3BADCB
:10CAC0004CAD5DAD0E94CFE66B017C016DA17EA1F6
:10CAD0008FA198A50E946EE64B015C01C301B201D3
:10CAE0000E946EE6A50194010E94CFE69B01AC0175
:10CAF000C701B6010E946AE687FF0AC0A50194013A
:10CB0000C701B6010E9492EB0E94FFEB2B013C0192
:10CB100088E60BA11CA1809FF001819FF00D1124DC
:10CB2000E858FE4E818C928CA38CB48C81149104B5
:10CB3000A104B104B9F160914C1170914D11809133
:10CB40004E1190914F11641575058605970550F5A6
:10CB50000E946EE62AAD3BAD4CAD5DAD0E94CFE6C6
:10CB60006B017C01C501B4010E946EE64B015C01C2
:10CB7000C301B2010E946EE6A50194010E94CFE6B6
:10CB80009B01AC01C701B6010E946AE687FF0AC09B
:10CB9000A5019401C701B6010E9492EB0E94FFEB30
:10CBA0002B013C0188E60BA11CA1809FF001819F15
:10CBB000F00D1124E858FE4E858C968CA78CB0A001
:10CBC00081149104A104B104B9F1609150117091E4
:10CBD000511180915211909153116415750586057C
:10CBE000970550F50E946EE62AAD3BAD4CAD5DADAC
:10CBF0000E94CFE66B017C01C501B4010E946EE684
:10CC00004B015C01C301B2010E946EE6A5019401D3
:10CC10000E94CFE69B01AC01C701B6010E946AE603
:10CC200087FF0AC0A5019401C701B6010E9492EBDB
:10CC30000E94FFEB2B013C0188E60BA11CA1809F09
:10CC4000F001819FF00D1124E858FE4EC1A0D2A042
:10CC5000E3A0F4A0C114D104E104F10409F4B0C9C3
:10CC60006091541170915511809156119091571106
:10CC7000641575058605970508F0A2C90E946EE641
:10CC80002AAD3BAD4CAD5DAD0E94CFE64B015C01E2
:10CC9000C701B6010E946EE66B017C01C301B201BF
:10CCA0000E946EE6A70196010E94CFE69B01AC01AF
:10CCB000C501B4010E946AE687FF82C9A7019601F7
:10CCC000C501B4010E9492EB0E94FFEB2B013C01D5
:10CCD00077C9FAA9FF2331F1A5019401632D722DC3
:10CCE000C8010E94CFE64B015C012DA53DA149A5DD
:10CCF00059A9C701B6010E94CFE69B01AC01C5014D
:10CD0000B4010E946AE687FF22C0A7019601C5010F
:10CD1000B4010E9492EB6DA77DA389A799AB21E096
:10CD20002AABFFC9A7019601C501B4010E9492EB8D
:10CD30009B01AC016DA57DA189A599A90E94CFE6B3
:10CD40006DA77DA389A799AB31E03AABEAC941E071
:10CD50004AABE7C9A7019601C501B40113C0C701D9
:10CD6000B6010E946AE687FD09C020E030E0A90113
:10CD7000C501B4010E94DCEC18164CF4A501940125
:10CD8000C701B6010E94B5EA2B013C0176CA240115
:10CD9000350177FA709477F87094A3019201C70176
:10CDA000B6010E946AE687FD68CA2601370165CA96
:10CDB0002DA53DA149A559A9C701B6010E946AE662
:10CDC00087FFB4CA3DA42DA009A519A9AFCA81E067
:10CDD00004CBF090B7098FEF8F0D8F708BA3B090BD
:10CDE000B6098091B709B81609F454C0C12CD12CEA
:10CDF0000BA10B1509F44EC0602E712C28E6269D60
:10CE00008001279D100D112408581E4ED8018C91C9
:10CE100083FD2BC00EAF1AAB0115110541F1199618
:10CE2000BC91BDA7F801F285FDA3D8011B96BC916A
:10CE3000B9A7F801F485F9ABD80115962D903D906E
:10CE40004D905C901897A20191016DA57DA189A5D7
:10CE50009F2F0E946AE6811186C1C114D10439F066
:10CE6000F601808180FD7FC102C0CEAEDAAA8BA11F
:10CE700081508F708BA38091B6098B1103C0CEAC0B
:10CE8000DAA8B6CF0BA10B1529F081E08B0D8F70BE
:10CE9000B82EF1CF1091B6091BA3C12CD12C8091D3
:10CEA000B7090BA1801709F443CB802E912C28E6FB
:10CEB000289D8001299D100D112408581E4ED8016F
:10CEC0008C9183FD0AC05801C114D10439F0C60108
:10CED0000E94487F811102C0C5C156018BA18F5F9E
:10CEE0008F708BA36501DBCF802F81508F70289FBF
:10CEF000F0011124E858FE4E908193FF24CB8DA7BA
:10CF00001ECB48E6439FC0011124DC01A858BE4E49
:10CF10001D018C9183FD19C015966D917D918D91A8
:10CF20009C9118970E9421EDF62EE72ED82EC92E3F
:10CF30000115110509F48CC0F801808180FD0AC03B
:10CF4000D1018C9180FD06C083C0FDA0E9A4D9A8C1
:10CF5000CEAC83C0F801808181608083C8010E94CB
:10CF6000487F811171C0F801618172818381948150
:10CF70000E9421ED2B013C019B01AC0160E070E0BF
:10CF800080E89FE30E9492EB4B015C019B01AC01A6
:10CF90006F2D7E2D8D2D9C2D0E94CFE669837A8387
:10CFA0008B839C832DA139A549A95EADC501B40130
:10CFB0000E94CFE6698B7A8B8B8B9C8BAE014F5F87
:10CFC0005F4FBE016F5E7F4FC8010E94C0B1F80184
:10CFD000E95BFF4F80818823B9F12091E70630910A
:10CFE000E8064091E9065091EA0637966081718122
:10CFF000828193810E94CFE62091181130911911FE
:10D0000040911A1150911B110E94CFE64B015C0117
:10D010009B01AC01C301B2010E94CFE60E94FFEB6D
:10D02000F801E65BFF4F71836083A50194016F2DCA
:10D030007E2D8D2D9C2D0E94CFE60E94FFEBF801E6
:10D04000E45BFF4F71836083D8018C918E7F8C935A
:10D050008F2C9E2CAD2CBC2C81018BA18F5F8F70EF
:10D060008BA3FDA2E9A6D9AACEAE79CAF10180812F
:10D0700081608083C8010E94487F81116FC0D10107
:10D0800011966D917D918D919C9114970E9421ED47
:10D090006B017C019B01AC0160E070E080E89FE3E4
:10D0A0000E9492EB2B013C012DEC3CEC4CE45DE347
:10D0B0000E94CFE669837A838B839C839401A501C8
:10D0C000C301B2010E94CFE6698B7A8B8B8B9C8B5C
:10D0D000AE014F5F5F4FBE016F5E7F4FC1010E9487
:10D0E000C0B1F101E95BFF4F80818823B9F1209144
:10D0F000E7063091E8064091E9065091EA06379636
:10D1000060817181828193810E94CFE62091181104
:10D110003091191140911A1150911B110E94CFE6C4
:10D120004B015C019B01AC01C701B6010E94CFE637
:10D130000E94FFEBF101E65BFF4F718360832DECF2
:10D140003CEC4CE45DE3C501B4010E94CFE60E94D3
:10D15000FFEBF101E45BFF4F71836083F10180819C
:10D160008E7F808304CA28E6269DF001279DF00D5E
:10D170001124E858FE4E808181FD43C0C114D104C2
:10D1800041F0D6011596CD90DD90ED90FC9018976A
:10D1900008C08BE0C82E87EDD82E83E2E82E8BE303
:10D1A000F82EB8E6B69DF001B79DF00D1124E858B1
:10D1B000FE4E81899289A389B489BC01CD01905822
:10D1C0009B01AC010E94B6EAF801258536854785AA
:10D1D00050890E94CFE69B01AC01C701B6010E94B5
:10D1E000B5EAE62E872E982EA92E262F372F482F08
:10D1F000592F6DA57DA189A599A90E946AE687FF8F
:10D2000004C0EDA48DA099A4A9A82E2D382D492DD8
:10D210005A2DC201B1010E946AE6882309F427CE83
:10D22000F8E6F69DC001F79D900D11249C01285849
:10D230003E4E6901D9018C9181608C93C8010E9496
:10D24000487F882329F0F60180818E7F80830FCE6E
:10D250008E2D982DA92DBA2DF60185839683A7834F
:10D26000B08705CED6018C9181FD52C0D6011596AE
:10D270002D913D914D915C9118972DA73EA74FA7F9
:10D2800058AB1501B5E02B0E311CF80145805680D6
:10D2900067807084A30192016DA57EA58FA598A9D2
:10D2A0000E946AE687FF34C0F60181899289A389CA
:10D2B000B489BC01CD0190589B01AC010E94B6EA33
:10D2C000D6011D962D913D914D915C9150970E94F4
:10D2D000CFE69B01AC016DA57EA58FA598A90E9404
:10D2E000B5EA6B017C019B01AC01C301B2010E9454
:10D2F000DCEC18166CF4D8018C9181608C93C5011C
:10D300000E94487F8823E1F0F80180818E7F80832E
:10D3100018E6189DF001199DF00D1124E858FE4EF5
:10D320002185328543855485658176818781908505
:10D330000E946AE68111D2CD0BA10093B609CECD31
:10D34000D101CD92DD92ED92FC9213970BA1009347
:10D35000B609DECFC858DF4F0FB6F894DEBF0FBE58
:10D36000CDBFDF91CF911F910F91FF90EF90DF9094
:10D37000CF90BF90AF909F908F907F906F905F9075
:10D380004F903F902F9008958091B7099091B809E0
:10D39000891B8F708F3019F40E9403A1F5CF809103
:10D3A000B7098F5F8F70E091B70998E69E9FF001F3
:10D3B0001124E858FE4EDF011D929A95E9F798E096
:10D3C00090834091DD095091DE096091DF097091F1
:10D3D000E009458B568B678B708F4091E109509126
:10D3E000E2096091E3097091E409418F528F638FE4
:10D3F000748F4091E5095091E6096091E7097091B9
:10D40000E809458F568F678F70A34091E9095091C5
:10D41000EA096091EB097091EC0941A352A363A35F
:10D4200074A32091B7099091B809291303C094E619
:10D430009093B4098093B70980916F0082608093C4
:10D440006F0008959091B7098091B809981306C0AC
:10D4500080914E0790914F07892B19F00E9403A1EC
:10D46000F1CF0895CF93DF938B3D9240B1F0EDED76
:10D47000FDE18491EF012196882321F00E94CD895E
:10D48000FE01F7CFE4EEF9E18491EF0121968823C4
:10D4900031F00E94CD89FE01F7CF80E001C081E02C
:10D4A000DF91CF9108952F923F924F925F926F92AA
:10D4B0007F928F929F92AF92BF92CF92DF92EF9224
:10D4C000FF920F931F93CF93DF93CDB7DEB7C7576C
:10D4D000D1090FB6F894DEBF0FBECDBF2DB63EB654
:10D4E000A7961FAE1EAEA79784E690E0A9969FAFC1
:10D4F0008EAFA99701E09E012B593F4F44E050E0C9
:10D50000BE01655A7F4FCE0189599F4F0E9425D099
:10D510009E012B593F4F42E050E0BE0167597F4FBB
:10D52000CE0189599F4F0E9425D043E050E0BE01B3
:10D53000655A7F4F8FED92E00E9421EE892B09F40E
:10D540003FC06F968FAD6F97882339F08FE36C964D
:10D550008FAF6C976D961FAE6D97E2EFFDE18491F2
:10D560007F012FEFE21AF20A811103C0E7EAFAE124
:10D5700004C00E94CD89F701F2CF84917F013FEF73
:10D58000E31AF30A882321F00E94CD89F701F5CF31
:10D59000BE01655A7F4F8EE99AE10E949AC5E0E983
:10D5A000FAE184917F019FEFE91AF90A882321F0BB
:10D5B0000E94CD89F701F5CF81E080931A0754C509
:10D5C000EDB7FEB7E696FFAFEEAFE6976B961CAEF3
:10D5D0001DAE1EAE1FAE6B97A7961FAE1EAEA797D1
:10D5E00001E09E012B593F4F41E050E0BE016059E0
:10D5F0007F4FCE0189599F4F0E9425D080E1EBE5F6
:10D60000F2E0DE01919601900D928A95E1F780E1BA
:10D61000EBE6F2E0DE01519601900D928A95E1F77A
:10D6200080E1EBE7F2E0DE01119601900D928A9520
:10D63000E1F7E1964FADE19750E04D5F5F4F440F4A
:10D64000551F440F551F2DB73EB7241B350B0FB682
:10D65000F8943EBF0FBE2DBF8DB79EB701967C01DB
:10D6600000E09E012B593F4FBC01CE0189599F4FCD
:10D670000E9425D09E012B593F4F44E050E067E0C7
:10D6800077E0CE0189599F4F0E9425D0E1968FAC5B
:10D69000E197912C93E0890E911C880C991C880CC1
:10D6A000991CEDB7FEB7E819F9090FB6F894FEBF5B
:10D6B0000FBEEDBF2DB73EB72F5F3F4F69018DB74E
:10D6C0009EB7881999090FB6F8949EBF0FBE8DBFFB
:10D6D000EDB7FEB731965F019E012B593F4FA40174
:10D6E000B601CE0189599F4F0E9425D09E012B592A
:10D6F0003F4FA401B501CE0189599F4F0E9425D00B
:10D7000010911B07112309F4A7C000E09E012B59BB
:10D710003F4F44E050E06FEE76E0CE0189599F4FD5
:10D720000E9425D09E012B593F4F44E050E063EF0B
:10D7300076E0CE0189599F4F0E9425D09E012B593A
:10D740003F4F44E050E06BEE76E0CE0189599F4FA9
:10D750000E9425D09E012B593F4F44E050E06FE0DE
:10D7600077E0CE0189599F4F0E9425D09E012B5909
:10D770003F4F44E050E06BE077E0CE0189599F4F86
:10D780000E9425D09E012B593F4F40E150E067EDAC
:10D7900076E0CE0189599F4F0E9425D09E012B59DA
:10D7A0003F4F44E050E0BE01695A7F4FCE01895996
:10D7B0009F4F0E9425D09E012B593F4F4CE050E0D7
:10D7C0006CE375E0CE0189599F4F0E9425D09E01E0
:10D7D0002B593F4F44E050E06CE371E1CE01895991
:10D7E0009F4F0E9425D09E012B593F4F44E050E0AF
:10D7F000BE01695A7F4FCE0189599F4F0E9425D0A3
:10D8000001E09E012B593F4F41E050E0BE016159BC
:10D810007F4FCE0189599F4F0E9425D09E012B59E1
:10D820003F4F41E050E0BE0162597F4FCE01895920
:10D830009F4F0E9425D011118AC06B968CAD9DAD73
:10D84000AEADBFAD6B978093751090937610A0939B
:10D850007710B09378107BC0E1968FADE19790E0A0
:10D86000029627EF36E0E4963FAF2EAFE497B5017E
:10D87000DE011196ECE08E2EE1E19E2EAE014F5EB0
:10D880005F4FF8E5AF2EF1E1BF2EE896FFAEEEAEAA
:10D89000E8977E0131E2E30EF11C20E030E08217D0
:10D8A00093072CF0E896EEADFFADE89701C0F701C5
:10D8B0004080518062807380F50141925192619263
:10D8C00071925F018217930714F0F60101C0FA010B
:10D8D0004080518062807380F40141925192619244
:10D8E00071924F018217930734F0FB014080518001
:10D8F0006280738005C04D905D906D907C90139711
:10D90000E496EEADFFADE49741925192619271922F
:10D91000E496FFAFEEAFE4972F5F3F4F6C5F7F4F12
:10D920001496F4E0CF0ED11C4C5F5F4FE896EEAD3D
:10D93000FFADE8973496E896FFAFEEAFE897F4E0D6
:10D94000EF0EF11C2430310509F0A9CFDECEE096B0
:10D950008FADE097853099F4AF968FADAF97853056
:10D9600071F400E09E012B593F4F44E650E069E717
:10D9700070E1CE0189599F4F0E9425D024C011111A
:10D9800002C00E9428B7E0968FADE097AF96CFAC6B
:10D99000AF978C9D60011124E12CF12CEC14FD0457
:10D9A00091F000E09E012B593F4F44E050E0BE0152
:10D9B000695A7F4FCE0189599F4F0E9425D02FEF82
:10D9C000E21AF20AEBCF00E09E012B593F4F44E0F0
:10D9D00050E0BE016D5A7F4FCE0189599F4F0E9482
:10D9E00025D01AE0115079F000E09E012B593F4FED
:10D9F00044E050E0BE01695A7F4FCE0189599F4FE4
:10DA00000E9425D0EFCF01E09E012B593F4F41E00E
:10DA100050E0BE0163597F4FCE0189599F4F0E944C
:10DA200025D09E012B593F4F41E050E0BE01645983
:10DA30007F4FCE0189599F4F0E9425D000E09E0163
:10DA40002B593F4F44E050E0BE01635C7F4FCE0155
:10DA500089599F4F0E9425D09E012B593F4F44E08A
:10DA600050E0BE016F5C7F4FCE0189599F4F0E94ED
:10DA700025D0AE968FADAE97AD96CFACAD978C9DC1
:10DA800060011124E12CF12C00E09E012B593F4F45
:10DA9000CE14DF0471F044E050E0BE01695A7F4FBC
:10DAA000CE0189599F4F0E9425D03FEFE31AF30A18
:10DAB000EBCF41E050E0BE016F587F4FCE01895956
:10DAC0009F4F0E9425D09E012B593F4F41E050E0CF
:10DAD000BE0165597F4FCE0189599F4F0E9425D0C5
:10DAE0009E012B593F4F44E050E0BE01695A7F4FE1
:10DAF000CE0189599F4F0E9425D09E012B593F4F3F
:10DB000044E050E0BE01695A7F4FCE0189599F4FD2
:10DB10000E9425D09E012B593F4F44E050E060E425
:10DB200071E1CE0189599F4F0E9425D09E012B594A
:10DB30003F4F44E050E0BE01615B7F4FCE01895909
:10DB40009F4F0E9425D09E012B593F4F44E050E04B
:10DB5000BE01655B7F4FCE0189599F4F0E9425D042
:10DB60009E012B593F4F44E050E0BE01695B7F4F5F
:10DB7000CE0189599F4F0E9425D010E000E09E0100
:10DB80002B593F4F44E050E0BE01695A7F4FCE0110
:10DB900089599F4F0E9425D0111110C06B96CCACB3
:10DBA000DDACEEACFFAC6B9720E030E84BE355E426
:10DBB000C701B6010E946AE6811103C054E0F52E48
:10DBC00033C080911B07811108C0C0924007D092DA
:10DBD0004107E0924207F092430700E09E012B5973
:10DBE0003F4F44E050E06CE377E0CE0189599F4F0E
:10DBF0000E9425D09E012B593F4F44E050E064E441
:10DC000077E0CE0189599F4F0E9425D09E012B5964
:10DC10003F4F44E050E0BE01695A7F4FCE01895921
:10DC20009F4F0E9425D012C0FA94FF2079F000E0A7
:10DC30009E012B593F4F44E050E0BE01695A7F4F8F
:10DC4000CE0189599F4F0E9425D0EECF1F5F15301E
:10DC500009F094CF00E09E012B593F4F42E050E085
:10DC6000BE016D597F4FCE0189599F4F0E9425D02B
:10DC70009E012B593F4F44E050E0BE01695A7F4F4F
:10DC8000CE0189599F4F0E9425D06B96CCACDDAC5C
:10DC9000EEACFFAC6B9720E030E84BE355E4C701F6
:10DCA000B6010E946AE6882329F180911B07811141
:10DCB00008C0C0923807D0923907E0923A07F09234
:10DCC0003B0700E09E012B593F4F44E050E064E3E6
:10DCD00077E0CE0189599F4F0E9425D09E012B5994
:10DCE0003F4F44E050E060E377E0CE0189599F4F19
:10DCF0000E9425D000E09E012B593F4F42E050E0AA
:10DD0000BE016F597F4FCE0189599F4F0E9425D088
:10DD10009E012B593F4F41E050E0BE016F587F4FAD
:10DD2000CE0189599F4F0E9425D019E0115000E083
:10DD30009E012B593F4F112359F044E050E0BE01A2
:10DD4000695A7F4FCE0189599F4F0E9425D0EECF4F
:10DD500041E050E06DED70E1CE0189599F4F0E9486
:10DD600025D0F12C00E09E012B593F4F44E050E0BC
:10DD7000BE01695A7F4FCE0189599F4F0E9425D01D
:10DD800010911B07111110C0F1100EC06B968CADD5
:10DD90009DADAEADBFAD6B978093E2109093E31055
:10DDA000A093E410B093E510F39485E0F812DACF75
:10DDB000111102C00E94E2C44CE0F42EFA94F1105A
:10DDC00003C03CE0F32E0FC000E09E012B593F4FF3
:10DDD00042E050E0BE01615A7F4FCE0189599F4F0A
:10DDE0000E9425D0EBCFFA9400E09E012B593F4FC3
:10DDF000FF2059F044E050E0BE016D5B7F4FCE0143
:10DE000089599F4F0E9425D0EECF46E050E0BE01D9
:10DE1000635C7F4FCE0189599F4F0E9425D09E01A0
:10DE20002B593F4F44E050E067EE76E0CE01895930
:10DE30009F4F0E9425D09E012B593F4F4CE050E050
:10DE4000BE016F5C7F4FCE0189599F4F0E9425D044
:10DE50002CE1F22EFA94F11003C094E0F92E1DC0CB
:10DE600000E09E012B593F4F44E050E0BE01695A4B
:10DE70007F4FCE0189599F4F0E9425D0EBCF00E004
:10DE80009E012B593F4F44E050E0BE01695A7F4F3D
:10DE9000CE0189599F4F0E9425D0FA94F110EFCFFF
:10DEA0008BE0F82EFA94FF2079F000E09E012B59C8
:10DEB0003F4F44E050E0BE01695A7F4FCE0189597F
:10DEC0009F4F0E9425D0EECFA9968EAD9FADA9970A
:10DED00084569109C7DA80931A07882309F1E2EF83
:10DEE000FDE184917F019FEFE91AF90A882321F06F
:10DEF0000E94CD89F701F5CFA9966EAD7FADA997A8
:10DF00006456710988E89AE10E9481C56BED72E060
:10DF100080E89AE10E9481C58AE00E94CD8999C07B
:10DF2000A7962EAD3FADA797AB968EAD9FADAB97A5
:10DF30002817390709F44BC081E080931A07EDEDEB
:10DF4000FDE184917F012FEFE21AF20A811103C0F3
:10DF5000E0E6FAE104C00E94CD89F701F2CF849196
:10DF60007F013FEFE31AF30A882321F00E94CD8955
:10DF7000F701F5CFAB966EAD7FADAB9780E090E04B
:10DF80004AE00E94F08CEBE5FAE184917F019FEF7B
:10DF9000E91AF90A882321F00E94CD89F701F5CF0B
:10DFA000A7966EAD7FADA79780E090E04AE00E9413
:10DFB000F08CEBE4FAE184917F012FEFE21AF20A90
:10DFC000882309F446C00E94CD89F701F4CF1111CE
:10DFD00042C0E2EFFDE184917F013FEFE31AF30AD3
:10DFE000811103C00FED12E004C00E94CD89F7013A
:10DFF000F2CFF80181918F01882319F00E94CD8919
:10E00000F8CFA9966EAD7FADA997645671098EE2DF
:10E010009AE10E9481C5A7964EAD5FADA79760E0DB
:10E0200070E081E29AE10E9447C5EEE1FAE1849155
:10E030007F012FEFE21AF20A811107C080911A07BF
:10E04000811109C00E94E6D006C00E94CD89F70167
:10E05000EECF112399F3E6968EAD9FADE6970FB6FE
:10E06000F8949EBF0FBE8DBF80911B07811102C027
:10E070000E94AEBE90911A0781E089270FB6F894EE
:10E080003EBE0FBE2DBEC958DF4F0FB6F894DEBF9F
:10E090000FBECDBFDF91CF911F910F91FF90EF90F9
:10E0A000DF90CF90BF90AF909F908F907F906F90B8
:10E0B0005F904F903F902F90089581E080931B07D1
:10E0C000F2D910921B078111EEC90E941DC381E095
:10E0D00008958F929F92AF92BF92CF92DF92EF926C
:10E0E000FF920F931F93CF93DF93CDB7DEB7CA5A3A
:10E0F000D1090FB6F894DEBF0FBECDBFE9961CAEB6
:10E100001DAE1EAE1FAEE9978091F1039091F20310
:10E11000A091F303B091F403ED968CAF9DAFAEAF39
:10E12000BFAFED97C556DF4F19821882CB59D0404B
:10E1300084E690E0C356DF4F99838883CD59D04061
:10E1400010921A079E0125563F4F44E050E0BE0151
:10E1500067587F4FCE0183569F4F0E9472D0C3569F
:10E16000DF4F88819981CD59D0400296C356DF4F49
:10E1700099838883CD59D040C556DF4F19821882C4
:10E18000CB59D04081E0CD55DF4F8883C35AD04072
:10E190009E0125563F4F41E050E0BE016D557F4F37
:10E1A000CE0183569F4F0E9472D09E0125563F4F4D
:10E1B00040E150E068E571E1CE0183569F4F0E9437
:10E1C00072D09E0125563F4F44E050E067E077E073
:10E1D000CE0183569F4F0E9472D09E0125563F4F1D
:10E1E00040E150E06CE071E1CE0183569F4F0E9408
:10E1F00072D09E0125563F4F40E150E067EF76E038
:10E20000CE0183569F4F0E9472D09E0125563F4FEC
:10E2100044E050E06FEE76E0CE0183569F4F0E94BF
:10E2200072D09E0125563F4F44E050E063EF76E008
:10E23000CE0183569F4F0E9472D09E0125563F4FBC
:10E2400044E050E06BEE76E0CE0183569F4F0E9493
:10E2500072D09E0125563F4F44E050E06FE077E0DA
:10E26000CE0183569F4F0E9472D09E0125563F4F8C
:10E2700044E050E06BE077E0CE0183569F4F0E9470
:10E2800072D09E0125563F4F40E150E067ED76E0A9
:10E29000CE0183569F4F0E9472D08AE097EDA3EA89
:10E2A000BCE3E9968CAF9DAFAEAFBFAFE9979E01DF
:10E2B00025563F4F44E050E0BE016B587F4FCE01E2
:10E2C00083569F4F0E9472D09E0125563F4F4CE0CF
:10E2D00050E06CE375E0CE0183569F4F0E9472D0F0
:10E2E0008091F7109091F810A091F910B091FA1068
:10E2F000C358DF4F88839983AA83BB83CD57D0400F
:10E300009E0125563F4F44E050E0BE0163587F4FC9
:10E31000CE0183569F4F0E9472D085E0CC55DF4FCF
:10E320008883C45AD040CB55DF4F8883C55AD0402C
:10E330009E0125563F4F44E050E065E770E1CE0175
:10E3400083569F4F0E9472D09E0125563F4F41E059
:10E3500050E0BE016C557F4FCE0183569F4F0E9407
:10E3600072D09E0125563F4F41E050E0BE016B55F3
:10E370007F4FCE0183569F4F0E9472D09E0125563B
:10E380003F4F44E650E069E770E1CE0183569F4F6E
:10E390000E9472D0CF57DF4F188219821A821B82D7
:10E3A000C158D0409E0125563F4F44E050E0BE0189
:10E3B0006F577F4FCE0183569F4F0E9472D0E996D0
:10E3C0001CAE1DAE1EAE1FAEE9971AE0115071F0E3
:10E3D0009E0125563F4F44E050E0BE016B587F4FF1
:10E3E000CE0183569F4F0E9472D0F0CF83E0CA5572
:10E3F000DF4F8883C65AD040C955DF4F8883C75A3C
:10E40000D040CB57DF4F188219821A821B82C55821
:10E41000D040C757DF4F188219821A821B82C95811
:10E42000D040E9961CAE1DAE1EAE1FAEE9979E0110
:10E4300025563F4F41E050E0BE016A557F4FCE0167
:10E4400083569F4F0E9472D09E0125563F4F41E058
:10E4500050E0BE0169557F4FCE0183569F4F0E9409
:10E4600072D09E0125563F4F44E050E0BE016757F1
:10E470007F4FCE0183569F4F0E9472D09E0125563A
:10E480003F4F44E050E0BE016B577F4FCE018356B3
:10E490009F4F0E9472D00AE010E00150110971F004
:10E4A0009E0125563F4F44E050E0BE016B587F4F20
:10E4B000CE0183569F4F0E9472D0EFCFC855DF4FD9
:10E4C0001882C85AD0408FEFC755DF4F8883C95A8A
:10E4D000D0409E0125563F4F41E050E0BE016855B7
:10E4E0007F4FCE0183569F4F0E9472D09E012556CA
:10E4F0003F4F41E050E0BE0167557F4FCE0183564C
:10E500009F4F0E9472D0E9961CAE1DAE1EAE1FAE8C
:10E51000E9979E0125563F4F44E050E0BE016B58FD
:10E520007F4FCE0183569F4F0E9472D09E01255689
:10E530003F4F44E050E0BE016B587F4FCE01835601
:10E540009F4F0E9472D09E0125563F4F44E050E0FD
:10E5500060E471E1CE0183569F4F0E9472D080919A
:10E560008B0290918C02A0918D02B0918E02C357C4
:10E57000DF4F88839983AA83BB83CD58D040809195
:10E580008F0290919002A0919102B0919202CF5689
:10E59000DF4F88839983AA83BB83C159D040CB5670
:10E5A000DF4F19821882C559D040C956DF4F1982F2
:10E5B0001882C759D0409E0125563F4F44E050E095
:10E5C000BE0163577F4FCE0183569F4F0E9472D08A
:10E5D0009E0125563F4F44E050E0BE016F567F4FED
:10E5E000CE0183569F4F0E9472D09E0125563F4F09
:10E5F00044E050E0BE016B567F4FCE0183569F4FE3
:10E600000E9472D010E0C12C80E8D82E8BE3E82E57
:10E6100085E4F82E812C912C90E8A92E9FE3B92E49
:10E62000111138C09E0125563F4F44E050E060E490
:10E6300077E0CE0183569F4F0E9472D09E012556EF
:10E640003F4F44E050E06CE377E0CE0183569F4FAC
:10E650000E9472D09E0125563F4F44E050E064E492
:10E6600077E0CE0183569F4F0E9472D0E9968CAE20
:10E670009DAEAEAEBFAEE9979E0125563F4F44E03A
:10E6800050E0BE016B587F4FCE0183569F4F0E94D2
:10E6900072D02AC0E996CCAEDDAEEEAEFFAEE99701
:10E6A0009E0125563F4F44E050E0BE016B587F4F1E
:10E6B000CE0183569F4F0E9472D0E9961CAE1DAECC
:10E6C0001EAE1FAEE99704E0015071F09E01255681
:10E6D0003F4F44E050E0BE016B587F4FCE01835660
:10E6E0009F4F0E9472D0F0CF1F5F153009F098CF76
:10E6F00084E190E0C156DF4F99838883CF59D040A1
:10E700009E0125563F4F42E050E0BE0161567F4FCB
:10E71000CE0183569F4F0E9472D09E0125563F4FD7
:10E7200044E050E068E377E0CE0183569F4F0E94BB
:10E7300072D09E0125563F4F44E050E064E377E0FD
:10E74000CE0183569F4F0E9472D09E0125563F4FA7
:10E7500044E050E060E377E0CE0183569F4F0E9493
:10E7600072D080E290E0CF55DF4F99838883C15A01
:10E77000D0409E0125563F4F42E050E0BE016F550C
:10E780007F4FCE0183569F4F0E9472D0C655DF4FF8
:10E790001882CA5AD04080E2E3E9F2E0DE019D9699
:10E7A00001900D928A95E1F79E0125563F4F41E079
:10E7B00050E0BE0166557F4FCE0183569F4F0E94A9
:10E7C00072D09E0125563F4F40E250E0BE01635D8E
:10E7D0007F4FCE0183569F4F0E9472D09E012556D7
:10E7E0003F4F41E050E06DED70E1CE0183569F4F09
:10E7F0000E9472D010E011110EC08091E210909131
:10E80000E310A091E410B091E510E9968CAF9DAFB4
:10E81000AEAFBFAFE9979E0125563F4F44E050E0B1
:10E82000BE016B587F4FCE0183569F4F0E9472D01E
:10E830001F5F153001F7BE01635B7F4F86E1FB016F
:10E8400011928A95E9F79E0125563F4F46E150E027
:10E85000CE0183569F4F0E9472D08CE2E3EBF2E030
:10E86000DE01119601900D928A95E1F79E012556E1
:10E870003F4F4CE250E0BE016F5F7F4FCE018356A9
:10E880009F4F0E9472D0BE0161597F4F86E0FB010D
:10E8900011928A95E9F79E0125563F4F46E050E0D8
:10E8A000CE0183569F4F0E9472D09E0125563F4F46
:10E8B00044E050E067EE76E0CE0183569F4F0E9421
:10E8C00072D0BE016D597F4F8CE0FB0111928A9589
:10E8D000E9F79E0125563F4F4CE050E0CE018356AC
:10E8E0009F4F0E9472D0E9961CAE1DAE1EAE1FAEA9
:10E8F000E9971CE1115071F09E0125563F4F44E00D
:10E9000050E0BE016B587F4FCE0183569F4F0E944F
:10E9100072D0F0CFE9961CAE1DAE1EAE1FAEE997C9
:10E9200014E0115071F09E0125563F4F44E050E035
:10E93000BE016B587F4FCE0183569F4F0E9472D00D
:10E94000F0CFE9961CAE1DAE1EAE1FAEE9971BE0E0
:10E95000115071F09E0125563F4F44E050E0BE013A
:10E960006B587F4FCE0183569F4F0E9472D0F0CFDD
:10E9700080911A07811167C0C356DF4FE880F98084
:10E98000CD59D040F4E6EF1AF108C556DF4F888123
:10E990009981CB59D040C756DF4F99838883C95995
:10E9A000D04084E690E0C356DF4F99838883CD59E9
:10E9B000D0409E0125563F4F44E050E06FED72E09D
:10E9C000CE0183569F4F0E9472D09E0125563F4F25
:10E9D00042E050E0BE0167567F4FCE0183569F4F05
:10E9E0000E9472D0E2EFFDE184918F010F5F1F4F13
:10E9F000882321F00E94CD89F801F6CFB7018CE081
:10EA00009AE10E9481C5C756DF4F48815981C95993
:10EA1000D04060E070E08FEF99E10E9447C5ECEFD5
:10EA2000F9E184918F010F5F1F4F882321F00E942D
:10EA3000CD89F801F6CFC7010E94326A90911A077A
:10EA4000892B80931A0790911A0781E08927C65570
:10EA5000DF4F0FB6F894DEBF0FBECDBFDF91CF9171
:10EA60001F910F91FF90EF90DF90CF90BF90AF90EC
:10EA70009F908F900895FF920F931F93CF93DF93F2
:10EA80008C01EB01F42E80E20E94CD898FEFF81605
:10EA900011F084E501C082E40E94CD898AE30E94DE
:10EAA000CD89F801608171818281938142E00E9469
:10EAB000758D488159816A817B818BE59DE10E943A
:10EAC00064C562E070E080E090E0DF91CF911F913B
:10EAD0000F91FF900C9474BE8F929F92AF92BF9251
:10EAE000CF92DF92EF92FF920F931F93CF93DF931A
:10EAF000F0E2FF2EE12CAE2DB0E0BD016F0D711DD7
:10EB0000759567956E1511F0F6120BC0EEE3FBE1FB
:10EB100065917491072E000C880B990B0E9470E68A
:10EB200062C09B0121503109220F331F220F331F76
:10EB3000F901E054F54E05911491AB01440F551FB6
:10EB4000440F551FFA01E054F54EC591D49180173A
:10EB5000910714F4F62ED1CFC817D90714F4E62E76
:10EB6000CACFF901EE53F54EE590F490FA01EE5359
:10EB7000F54EC590D490BC01601B710B072E000CA4
:10EB8000880B990B0E9470E64B015C01B6016E196F
:10EB90007F09072E000C880B990B0E9470E69B01E1
:10EBA000AC01C501B4010E94CFE64B015C01C01B62
:10EBB000D10BBE01DD0F880B990B0E9470E69B0103
:10EBC000AC01C501B4010E9492EB4B015C01B7019D
:10EBD000FF0C880B990B0E9470E69B01AC01C501EC
:10EBE000B4010E94B6EADF91CF911F910F91FF907F
:10EBF000EF90DF90CF90BF90AF909F908F9008954F
:10EC00000F931F93CF93DF93CDB7DEB728970FB63F
:10EC1000F894DEBF0FBECDBF60914E0470914F04DB
:10EC2000072E000C880B990B0E9470E66D837E8383
:10EC30008F8398878091500490915104A091520441
:10EC4000B091530489839A83AB83BC834DEFBE019B
:10EC50006B5F7F4FCE0101960EDF6091480470918B
:10EC60004904072E000C880B990B0E9470E66D83F7
:10EC70007E838F83988780914A0490914B04A09162
:10EC80004C04B0914D0489839A83AB83BC834FEFCE
:10EC9000BE016B5F7F4FCE010196EDDEE3E6FDE145
:10ECA00084918F010F5F1F4F882321F00E94CD892F
:10ECB000F801F6CFE0915207F0E0E05BF84F608199
:10ECC00070E080E090E00E945B8DEEE5FDE18491D4
:10ECD0008F010F5F1F4F882321F00E94CD89F8011B
:10ECE000F6CF6091510770E080E090E00E945B8D6C
:10ECF00028960FB6F894DEBF0FBECDBFDF91CF913F
:10ED00001F910F9108950F930FB70F9300916E000D
:10ED10000B7F00936E0078940F930BB70F930CB793
:10ED20000F921F922F933F934F935F936F937F9315
:10ED30008F939F93AF93BF93EF93FF931124EFD2E1
:10ED4000FF91EF91BF91AF919F918F917F916F91C3
:10ED50005F914F913F912F911F900F900CBF0F919A
:10ED60000BBF0F910460F89400936E000F910FBFDA
:10ED70000F911895CF92DF92EF92FF92C0904A04C4
:10ED8000D0904B04E0904C04F0904D046091480406
:10ED90007091490466507109072E000C880B990B7D
:10EDA0000E9470E69B01AC01C701B6010E946AE6B1
:10EDB00087FF1FC020E030E040E050E4C701B6010B
:10EDC0000E94B6EA0E94FFEB70938A07609389075E
:10EDD0000E940259DC01CB01805A9541AF4FBF4FD1
:10EDE0008093850790938607A0938707B093880741
:10EDF00008C010928507109286071092870710921C
:10EE00008807FF90EF90DF90CF900895CF92DF9228
:10EE1000EF92FF92C0905004D0905104E0905204C1
:10EE2000F090530460914E0470914F046750710943
:10EE3000072E000C880B990B0E9470E69B01AC0119
:10EE4000C701B6010E946AE687FF1FC020E030E0DC
:10EE500040E450E4C701B6010E94B6EA0E94FFEB0D
:10EE600070938407609383070E940259DC01CB01F1
:10EE7000805A9541AF4FBF4F80937F079093800793
:10EE8000A0938107B093820708C010927F07109269
:10EE900080071092810710928207FF90EF90DF9019
:10EEA000CF9008958F929F92AF92BF92CF92DF92B0
:10EEB000EF92FF920F931F93CF93DF93F0E4FF2E17
:10EEC000E12CAE2DB0E0BD016F0D711D75956795FC
:10EED0006E1511F0F6120BC0E0EBFCE16591749138
:10EEE000072E000C880B990B0E9470E662C09B01F4
:10EEF00021503109220F331F220F331FF901EE5425
:10EF0000F44E05911491AB01440F551F440F551F4A
:10EF1000FA01EE54F44EC591D4918017910714F480
:10EF2000F62ED1CFC817D90714F4E62ECACFF901AF
:10EF3000EC54F44EE590F490FA01EC54F44EC59084
:10EF4000D490BC01601B710B072E000C880B990B31
:10EF50000E9470E64B015C01B6016E197F09072E15
:10EF6000000C880B990B0E9470E69B01AC01C50157
:10EF7000B4010E94CFE64B015C01C01BD10BBE0166
:10EF8000DD0F880B990B0E9470E69B01AC01C50157
:10EF9000B4010E9492EB4B015C01B701FF0C880B9E
:10EFA000990B0E9470E69B01AC01C501B4010E945F
:10EFB000B6EADF91CF911F910F91FF90EF90DF9014
:10EFC000CF90BF90AF909F908F90089560E0809118
:10EFD00095079091960780DD6093500470935104DB
:10EFE00080935204909353048091930790919407D7
:10EFF00059DF60934A0470934B0480934C049093C0
:10F000004D04A89510924D0708957F928F929F927C
:10F01000AF92BF92CF92DF92EF92FF920F931F9326
:10F02000CF93DF9320E030E048E452E46091500455
:10F030007091510480915204909153040E94DCEC31
:10F0400018164CF4E6E4FBE1E491C1E001C0CC0FFA
:10F05000EA95EAF701C0C0E080E4E82E8BE1F82EE3
:10F0600006E41BE196E0A92E912CD0E0CC24C394B9
:10F07000D12CF7017490F801849077FC23C0892D7E
:10F0800090E0082C02C0959587950A94E2F780FDE0
:10F0900019C0BE01082C02C0759567950A94E2F765
:10F0A0006170B62EB1946B2D872D0E9443BD6B2DE0
:10F0B00070E0872D0E94ADBDC60101C0880F8A9403
:10F0C000EAF7982AAA94FFEFEF1AFF0A0F5F1F4F83
:10F0D000A110CFCFDF91CF911F910F91FF90EF90B3
:10F0E000DF90CF90BF90AF909F908F907F900895CA
:10F0F0000F931F9380912F07813019F40E940259BA
:10F1000008C060912B0770912C0780912D0790917A
:10F110002E070091570710915807209159073091F9
:10F120005A07601B710B820B930B28EE33E040E013
:10F1300050E00E9458EA8091530790915407A091A3
:10F140005507B0915607BC01CD01620F731F841F94
:10F15000951F1F910F91089510922F071092570736
:10F16000109258071092590710925A0710922B07C5
:10F1700010922C0710922D0710922E071092530711
:10F1800010925407109255071092560708958091D7
:10F190002F078130E1F0823051F4AADF60935307EA
:10F1A00070935407809355079093560701C0D4DF9E
:10F1B00081E080932F070E94025960935707709354
:10F1C00058078093590790935A0781E0089580E08B
:10F1D000089580912F07813079F482E080932F0782
:10F1E0000E94025960932B0770932C0780932D0780
:10F1F00090932E0781E0089580E0089580912F0775
:10F200008150823010F080E0089510922F070E9404
:10F21000025960932B0770932C0780932D079093CE
:10F220002E0781E0089510924C0780E090E00E9444
:10F23000F75910924904109248049CDDDFDF80E00A
:10F2400090E00E94F759109250072C9810924904B0
:10F2500010924804109251078091020180728093AD
:10F2600000010895DF92EF92FF920F931F93CF93C7
:10F27000DF93F82ED62EE72E8A018091270288236D
:10F2800009F439C0EDEDFDE18491EF012196882369
:10F2900021F00E94CD89FE01F7CFED2DFE2D849146
:10F2A000EF012196882321F00E94CD89FE01F7CF3E
:10F2B000E1E5FBE18491EF012196882321F00E9492
:10F2C000CD89FE01F7CFF7FC0BC06F2DFF0C770B3C
:10F2D000880B990B0E945B8D8AE00E94CD890BC040
:10F2E000ECE4FBE18491EF012196882321F00E9458
:10F2F000CD89FE01F7CF80915B07811108C0109284
:10F30000270281E080935B07C8010E94BCA0DF91C7
:10F31000CF911F910F91FF90EF90DF9084CFEF92EC
:10F32000FF920F931F93CF93DF9380912A028F3721
:10F33000A0F08F57909150079093A607992311F052
:10F340002C9A01C02C98209151072093A5079091E9
:10F350000201222369F090950BC09091A6078917AE
:10F3600008F02C989091A507891728F09091020138
:10F370009072909300018F5F80932A029091A4076E
:10F3800081E089278093A4078091290285301CF4AD
:10F39000C1E0C80F01C0C0E0823009F4B4C054F429
:10F3A000882301F1813009F0E3C088E080937B007D
:10F3B00085E4C0C0843009F4C5C00CF4B7C0853002
:10F3C00009F0D6C09091A307911102C08093A307C2
:10F3D0008091A30781508093A307882309F4C8C0B4
:10F3E000C5E0C6C0809128028F5F80311CF48093F5
:10F3F0002802BEC01092280280914D07811113C0CF
:10F400008091990790919A0790939607809395071A
:10F410008091970790919807909394078093930712
:10F4200081E080934D078AE0E9E9F7E0DF011D9272
:10F430008A95E9F71092980710929707009195071F
:10F440001091960711950195110980914E049091A4
:10F450004F04D1E0181619062CF080915007811145
:10F4600001C0D0E080913605909137059195819546
:10F4700091098017910734F449EE5CE16AE07DE17F
:10F4800080E0F0DE80911C0290911D0291958195A3
:10F4900091090817190744F4DD2331F04CE15DE1CF
:10F4A0006DE37DE180E0DEDE8091480490914904C7
:10F4B00011E0181619062CF080915107811101C036
:10F4C00010E0E0909307F0909407809134059091BC
:10F4D00035058E159F0534F049EF5CE16AE07DE16A
:10F4E0008FEFC0DE80911A0290911B02E816F90698
:10F4F0000CF43EC01123E1F14CE25DE16DE37DE1EE
:10F500008FEFB0DE35C080917A0086FD2EC08091ED
:10F510007800909179002091990730919A07820F95
:10F52000931F90939A078093990722C088E0809355
:10F530007B0086E480937C0080917A0080648093D5
:10F540007A0016C080917A0086FD11C08091780003
:10F55000909179002091970730919807820F931F1F
:10F56000909398078093970703C0C2E001C0C4E05E
:10F57000C09329020E9438B780914E0790914F079F
:10F580000097A9F0019790934F0780934E07892B1E
:10F5900071F48FE49DE19093A8078093A707DF9112
:10F5A000CF911F910F91FF90EF900C94F989DF910B
:10F5B000CF911F910F91FF90EF9008952F923F925E
:10F5C0004F925F926F927F928F929F92AF92BF9273
:10F5D000CF92DF92EF92FF920F931F93CF93DF931F
:10F5E00000D01F92CDB7DEB75C017A8369834A01F0
:10F5F000170107FD07C0802F002E000C990B9C837C
:10F600008B8304C0E1E0F0E0FC83EB83F9014080F0
:10F610005180628073808B819C81880F991F880F35
:10F62000991F9C838B838557984F7C01A30192017E
:10F63000FC0160817181828193810E946AE6882346
:10F6400091F0F701408251826282738211E020E0E2
:10F6500030E0A901C301B2010E94DCEC18160CF0E5
:10F6600010E0F5011083F50180818230D1F0833004
:10F6700009F45EC0813009F07CC0EB81FC81E55764
:10F68000F84F2081318142815381F4016081718181
:10F69000828193810E946AE687FD6BC082E0F5015A
:10F6A00080838B819C818557984F9C838B83B60187
:10F6B00080E090E00E946EE69B01AC01EB81FC8152
:10F6C00060817181828193810E94B5EA9B01AC01C6
:10F6D000F40160817181828193810E94DCEC87FD5D
:10F6E00014C00E9402596B017C019101A8EEB3E0A5
:10F6F0000E94A6EAC60ED71EE81EF91EE981FA810D
:10F70000C082D182E282F38234C00E940259E98130
:10F71000FA81C080D180E280F380DC01CB018C19BA
:10F720009D09AE09BF09B7FD24C083E0F5018083C0
:10F730000F3F19F042EB5CE102C045EC5CE169ED82
:10F740007CE1802F0F900F900F900F90DF91CF9161
:10F750001F910F91FF90EF90DF90CF90BF90AF90EF
:10F760009F908F907F906F905F904F903F902F90E1
:10F7700079CD0F900F900F900F90DF91CF911F9147
:10F780000F91FF90EF90DF90CF90BF90AF909F9040
:10F790008F907F906F905F904F903F902F90089543
:10F7A0004F925F926F927F928F929F92AF92BF9291
:10F7B000CF92DF92EF92FF920F931F93CF93DF933D
:10F7C000CDB7DEB760970FB6F894DEBF0FBECDBFE2
:10F7D00080914D07811117C060960FB6F894DEBF77
:10F7E0000FBECDBFDF91CF911F910F91FF90EF9092
:10F7F000DF90CF90BF90AF909F908F907F906F9051
:10F800005F904F900895E2DB0E9402594B015C012A
:10F8100060914E0470914F04072E000C880B990BD9
:10F820000E9470E669837A838B839C8344E1C42EB3
:10F83000D12C5CE3E52EF12C00E09E012F5F3F4FC1
:10F8400040E554E06BE777E08AE797E0B7DEC090E9
:10F850005004D0905104E0905204F0905304609111
:10F86000380570913905072E000C880B990B0E9402
:10F8700070E69B01AC01C701B6010E94DCEC1816D2
:10F880000CF009C160911E0270911F02072E000C3E
:10F89000880B990B0E9470E69B01AC01C701B60171
:10F8A0000E946AE687FFF7C000914E0410914F0452
:10F8B000B801012E000C880B990B0E9470E6A7017D
:10F8C00096010E94B5EA2B013C0120ED3CEC4CE492
:10F8D0005DE36091440770914507809146079091E0
:10F8E00047070E94CFE66D837E838F8398872091A0
:10F8F0007107309172074091730750917407C701E7
:10F90000B6010E94B5EA9B01AC016D817E818F81B9
:10F9100098850E94CFE66D837E838F83988723E34B
:10F9200033E343E75FE360916D0770916E07809169
:10F930006F07909170070E94CFE69B01AC016D812B
:10F940007E818F8198850E94B6EA6D837E838F8346
:10F95000988760936D0770936E0780936F079093FD
:10F960007007C0927107D0927207E0927307F0920D
:10F97000740720E030E040E251E4C301B2010E948C
:10F98000DCEC18160CF431C220E030E040E251EC1F
:10F99000C301B2010E946AE687FD2FC2012B09F460
:10F9A0002CC280916C0781112CC220916807309184
:10F9B000690740916A0750916B0729873A874B87FF
:10F9C0005C87209140073091410740914207509158
:10F9D0004307C301B2010E94CFE66B017C01A30182
:10F9E000920169857A858B859C850E94B6EA698734
:10F9F0007A878B879C8760936807709369078093E9
:10FA00006A0790936B0720913C0730913D07409126
:10FA10003E0750913F070E94CFE6A70196010E9442
:10FA2000B6EA2D813E814F8158850E94B5EA6B016F
:10FA30007C0120E030E04FE753E40E94DCEC20E062
:10FA400030E0A90118160CF4E3C1C701B6010E9409
:10FA50006AE687FD07C0C701B6010E94FAEB7595FB
:10FA600067951AC020E030E0A901C301B2010E94ED
:10FA70006AE687FF10C0A301920169857A858B85AC
:10FA80009C850E94B5EA609368077093690780932C
:10FA90006A0790936B0760E06093500780917F073F
:10FAA00090918007A0918107B09182070097A105EE
:10FAB000B10521F1A5019401281B390B4A0B5B0B01
:10FAC00057FD1CC0609183077091840780E090E02F
:10FAD0000E946EE69B01AC0160915004709151044C
:10FAE00080915204909153040E946AE687FF82C17C
:10FAF00041E95BE163EA7BE180E0B4DB80914807A8
:10FB000090914907A0914A07B0914B07A501940134
:10FB1000281B390B4A0B5B0B57FD0FC076DAD5015A
:10FB2000C4018C53964FAF4FBF4F809348079093BB
:10FB30004907A0934A07B0934B078091850790919E
:10FB40008607A0918707B09188070097A105B105A6
:10FB500011F1881A990AAA0ABB0AB7FC1CC0609165
:10FB6000890770918A0780E090E00E946EE69B0111
:10FB7000AC0160914A0470914B0480914C049091C7
:10FB80004D040E946AE687FF20C14FE65BE162E810
:10FB90007BE18FEF67DB6091480470914904072E89
:10FBA000000C880B990B0E9470E669837A838B8323
:10FBB0009C8395E0C92ED12C24E1E22EF12C0FEF8D
:10FBC0009E012F5F3F4F4AE454E065E777E089E705
:10FBD00097E0F4DCC0904A04D0904B04E0904C04D1
:10FBE000F0904D0420E030E040EA50E4C701B60157
:10FBF0000E94DCEC87FDE5C020E030E040EF52E4FD
:10FC0000C701B6010E946AE618160CF4DAC06091CA
:10FC1000480470914904072E000C880B990B0E9430
:10FC200070E6A70196010E94B5EA4B015C012091A4
:10FC300038073091390740913A0750913B070E94AD
:10FC4000CFE669877A878B879C87209164073091FC
:10FC500065074091660750916707C501B4010E948E
:10FC6000B6EA6D837E838F83988760936407709371
:10FC7000650780936607909367072091340730915A
:10FC8000350740913607509137070E94CFE66D87C0
:10FC90007E878F87988B20ED3CEC4CE45DE3609190
:10FCA00030077091310780913207909133070E949D
:10FCB000CFE62B013C012091600730916107409114
:10FCC000620750916307C701B6010E94B5EA9B0124
:10FCD000AC01C301B2010E94CFE62B013C0123E33A
:10FCE00033E343E75FE360915C0770915D078091C8
:10FCF0005E0790915F070E94CFE69B01AC01C301B4
:10FD0000B2010E94B6EA2B013C0160935C0770933C
:10FD10005D0780935E0790935F07C0926007D09263
:10FD20006107E0926207F09263072D853E854F855B
:10FD3000588969857A858B859C850E94B6EAA301DE
:10FD400092010E94B5EA6B017C0120E030E04FE7B0
:10FD500053E40E94DCEC20E030E0A9011816C4F561
:10FD6000C501B4010E94DCEC181684F4A5019401CD
:10FD70006D817E818F8198850E94B5EA60936407CA
:10FD80007093650780936607909367076FE71AC0C3
:10FD900020E030E0A901C501B4010E946AE687FFB6
:10FDA00010C0A50194016D817E818F8198850E948C
:10FDB000B5EA609364077093650780936607909334
:10FDC000670760E06093510707CD0E94BA76E3CEE3
:10FDD000C701B6010E946AE687FDDACFC701B60106
:10FDE0000E94FAEB75956795EDCF81E080936C07E3
:10FDF0006FE752CE80E00AD881CE81E080936C0715
:10FE00004ACE10926C0719861A861B861C86D9CD9D
:10FE1000C301B2010E94DCEC181654F7A301920151
:10FE200069857A858B859C850E94B5EA6093680711
:10FE30007093690780936A0790936B076FE72CCEE6
:10FE400090916F00292F227091FF05C090916F0053
:10FE50009D7F90936F0034E0839FC0011124FC01CB
:10FE6000E450FF4E4081518162817381FC01E15E6B
:10FE7000F84F408351836283738381E080931E0730
:10FE8000222329F080916F00826080936F00089593
:10FE9000BC0120911C0730911D0740911C07509117
:10FEA0001D072417350711F09A01F7CF81E02617B7
:10FEB000370709F080E008958F929F92AF92BF922A
:10FEC000CF92DF92EF92FF921F93CF93DF93C82FD1
:10FED00087ED9BE09093B3098093B2091092F30BE6
:10FEE00082E090E0A0E0B0E08093DC0B9093DD0B2B
:10FEF000A093DE0BB093DF0B1092B1091092AD0905
:10FF00001092AE091092AF091092B0098FEF9FEFD7
:10FF1000DC018093A9099093AA09A093AB09B0933F
:10FF2000AC09CC2379F1C53008F0F8C040E060E0BE
:10FF300070E0CB010E94CED1882309F4EFC020E10C
:10FF4000C29FC00111248756984FFC01E254FE4F16
:10FF500020812F7709F0E2C03C9640815181628177
:10FF60007381443651056105710508F4D7C0349793
:10FF7000C080D180E280F380C114D104E104F10497
:10FF800021F4CCC0C12CD12C760140E0C701B601D0
:10FF90000E94CED1182F882309F4C0C08091B407E5
:10FFA0009091B5078115924009F0B8C0A091B907AA
:10FFB000AA2309F4B3C06091B7077091B80761151F
:10FFC000710509F4ABC02091B607222309F4A6C03D
:10FFD000A093EE0B2093E00B80E030E041E050E096
:10FFE000C82FFA01082E02C0EE0FFF1F0A94E2F795
:10FFF0002E173F0739F08F5FC83091F789E0809363
:020000021000EC
:10000000E90B8CC08093E90B2091BF073091C007AA
:100010002115310519F040E050E008C02091CD07CE
:100020003091CE074091CF075091D0072093E10B3C
:100030003093E20B4093E30B5093E40B46015701DE
:10004000860E971EA11CB11C8092EF0B9092F00BB4
:10005000A092F10BB092F20BE091BA07F091BB07BE
:10006000F093F50BE093F40BB0E00E9496EA860E55
:10007000971EA81EB91E8092F60B9092F70BA092C5
:10008000F80BB092F90B85E0EE0FFF1F8A95E1F7B0
:10009000E150FE4FEF2FFF27E6958E0E9F1EA11C0D
:1000A000B11C8092EA0B9092EB0BA092EC0BB092F9
:1000B000ED0B2091BC073091BD072115310521F0D2
:1000C000A90160E070E008C04091C9075091CA07DB
:1000D0006091CB077091CC07D701C60188199909A7
:1000E000AA09BB09840F951FA61FB71F04C0B695A8
:1000F000A79597958795CA95D2F78093E50B90932E
:10010000E60BA093E70BB093E80B853F2FE0920737
:10011000A105B10528F48CE08093F30B10E01AC020
:10012000853F9F4FA105B10510F480E111C080917A
:10013000D5079091D607A091D707B091D8078093A3
:10014000F60B9093F70BA093F80BB093F90B80E2AA
:100150008093F30B812FDF91CF911F91FF90EF9050
:10016000DF90CF90BF90AF909F908F900895682FB1
:100170008EE99FE00C94E44ACF92DF92EF92FF92D7
:100180001F93CF93DF931092360A8091690A8823D8
:1001900021F086E69AE00E94E0981092DB0B109224
:1001A000D80B85E38093D70B0E940259EB01A895E9
:1001B00061E08091D70B0E9471BD87ED9BE00E94AA
:1001C000419A2398229A219A209A289A85E080932E
:1001D000D90B82E58CBD1DBC1AE08FEF0E94469AB8
:1001E0001150D9F720E030E0A90160E087ED9BE0F5
:1001F0000E944B9A182F8093DA0B813049F00E94AD
:1002000002596C1B7D0B613D774060F381E054C067
:100210002AEA31E040E050E068E087ED9BE00E9490
:100220004B9A82FF03C01093DB0B0EC014E00E94B8
:10023000599F8093DA0B1150D1F78A3A11F082E07E
:100240003BC082E08093DB0B8091DB0B823021F09E
:10025000C12CD12C760105C0C12CD12CE12C80E41D
:10026000F82E20E030E0A90167E387ED9BE00E94D3
:100270004B9AA701960169E287ED9BE00E944B9A99
:100280008093DA0B882349F00E9402596C1B7D0B86
:10029000613D774030F38AE00FC08091DB0B823004
:1002A00011F520E030E0A9016AE387ED9BE00E94B0
:1002B0004B9A882351F088E08093D80B87ED9BE020
:1002C0000E94419AE2EFFDE119C00E94599F807C93
:1002D000803C19F483E08093DB0B0E94599F0E94BD
:1002E000599F0E94599F87ED9BE00E94419A10926E
:1002F000D90B81E0E1DD811131C015C08491EF019E
:100300002196882321F00E94CD89FE01F7CFE4EEEB
:10031000FDE18491EF012196882309F454C00E94E5
:10032000CD89FE01F6CF80E0C7DD811117C0EDED6C
:10033000FDE18491EF012196882321F00E94CD896F
:10034000FE01F7CFE9ECFDE18491EF0121968823CE
:1003500009F439C00E94CD89FE01F6CF6CED7BE037
:1003600086E69AE00E948D98811116C0EDEDFDE1C0
:100370008491EF012196882321F00E94CD89FE010E
:10038000F7CFE8EBFDE18491EF0121968823D9F0C6
:100390000E94CD89FE01F7CF81E08093360AE2EF1B
:1003A000FDE18491EF012196882319F0F6D7FE0133
:1003B000F8CFECEAFDE18491EF012196882319F052
:1003C000ECD7FE01F8CF8BE1E6E6FAE0A5E8BAE06B
:1003D00001900D928A95E1F78091640A9091650AE7
:1003E0009093840A8093830ADF91CF911F91FF90AD
:1003F000EF90DF90CF9008958091430E823039F4D2
:1004000087E99DE19093A8078093A707F2D70E9400
:1004100002596093470E7093480E8093490E909353
:100420004A0E8091360A882319F081E08093350ABC
:1004300081E08093430E0895CF93DF931092350AA5
:1004400083E08093430E8091900E8823B1F0EFE813
:10045000FDE18491EF01882341F0082E000C990BF7
:1004600086DE2196FE018491F6CF8DE090E07FDE5E
:100470008AE090E0DF91CF917ACEE3E9FDE18491CB
:10048000EF01882391F3082E000C990B70DE219662
:10049000FE018491F6CF8F929F92AF92BF92CF923E
:1004A000DF92EF92FF920F931F93CF93DF9300D0D1
:1004B0001F92CDB7DEB7FC018381813079F5818150
:1004C00081FF2CC081899289A389B489892B8A2BC9
:1004D0008B2B09F448C07F0140E050E0BA01CF0106
:1004E0000E94F6978823D1F0F70185889688A7881F
:1004F000B08CC18CD28C82E090E0A0E0B0E0F6013C
:1005000080839183A283B3839E012F5F3F4FB50108
:10051000A401C6010E9497D2811102C080E03CC0B4
:1005200000E010E09801B501A401C6010E9406D2C6
:100530008823A1F389809A80AB80BC80F6018789EB
:10054000803141F4F8EF8F16FFEF9F06A104B1044C
:1005500060F4DACF88EF88168FEF9806A8068FE050
:10056000B80618F4D1CF81E017C0F701158A168AB2
:10057000178A108E118A128A138A148A81818068E0
:100580008183C7010E94E5D3882341F240E050E017
:10059000BA01C7010E94F6970F900F900F900F902D
:1005A000DF91CF911F910F91FF90EF90DF90CF904F
:1005B000BF90AF909F908F9008951092380A10923C
:1005C000350A8091010C882321F08EEF9BE00C947A
:1005D000E09808952F923F924F925F926F927F9290
:1005E0008F929F92AF92BF92CF92DF92EF92FF9243
:1005F0000F931F93CF93DF93CDB7DEB7C257D109C7
:100600000FB6F894DEBF0FBECDBF8C013B014A018F
:100610004DB75EB7E1965FAF4EAFE197AD961FAEB7
:10062000AD971B0154E0250E311C7E018FE5E80ECD
:10063000F11C9DEE492E92E0592EE0E4F0E0EC0F23
:10064000FD1F3496E396FFAFEEAFE397F30187818A
:10065000823008F45AC184859585A685B7858F7147
:100660009927AA27BB27892B8A2B8B2B09F04DC1F1
:100670001092460A46E45AE0BE016F5F7F4FC10107
:100680000E947DD318160CF040C18C85982F98716C
:10069000903129F42091B30C2150223078F4298133
:1006A000222309F432C1253E89F22E3279F22091BB
:1006B000460A2E3259F28A7049F6B4C04DB75EB779
:1006C000AF965FAF4EAFAF97BE016F5F7F4FC70171
:1006D0000E9478D10115110521F0F8018081811166
:1006E00097C021E081E090E0F70101900020E9F758
:1006F0003197EE19FF098E0F9F1F02964DB75EB717
:10070000481B590B0FB6F8945EBF0FBE4DBF8DB797
:100710009EB701965C01211102C0B80102C062E2DD
:1007200073E0C5010E941AEEB701C5010E94FBEDFE
:1007300062E273E0C5010E94FBED25961FAE25978E
:1007400028961FAE289724961FAE1EAE2497229699
:100750005FAE4EAE229721E0A701B101E3968EADC8
:100760009FADE3970E946C9E811126C08091B30CCF
:10077000811122C0E2EFFDE184916F019FEFC91A60
:10078000D90A882319F009D6F601F6CFEBE7FDE187
:1007900084916F012FEFC21AD20A882319F0FDD578
:1007A000F601F6CF6701F60181916F01882311F000
:1007B000F4D5F9CF8AE0F1D58BE1FE01EC5BFF4F78
:1007C000DE01959601900D928A95E1F724968EAD03
:1007D0009FAD24979CA38BA35AA249A240E050E06E
:1007E000BE016F5D7F4FC501F5DECE0181960E948F
:1007F00099A0CE01805C9F4F0E9499A0AF964EAD0C
:100800005FADAF970FB6F8945EBF0FBE4DBF1ECF62
:10081000F80101900020E9F73197CF01801B910B7F
:1008200020E062CF81E0903109F080E08093370AC8
:10083000903141F08985873409F008CF8A858E3759
:1008400009F404CF8091B30C813029F08230B9F1E2
:100850008111FCCE0AC08091B40C9091B50C019628
:100860009093B50C8093B40CF1CEBE016F5F7F4FB7
:1008700089E39AE00E9478D10115110529F489E3F2
:10088000C82E8AE0D82E08C06801F60181916F0158
:100890008823A9F382D5F9CFF60181916F018823CE
:1008A00011F07BD5F9CF80E278D56D8D7E8D8F8D5F
:1008B00098A14AE00E94F08C8AE06FD5C7CEBE01B5
:1008C0006F5F7F4F89E39AE00E9478D18114910491
:1008D00041F069E37AE0C4010E94E8ED892B69F4F4
:1008E00014C0AD96FFADAD978F2F90E02091C00F53
:1008F0003091C10F8217930741F0AD962FADAD97A0
:100900002F5FAD962FAFAD97A1CEE1968EAD9FAD87
:10091000E1970FB6F8949EBF0FBE8DBFCE58DF4F44
:100920000FB6F894DEBF0FBECDBFDF91CF911F9100
:100930000F91FF90EF90DF90CF90BF90AF909F907E
:100940008F907F906F905F904F903F902F90089581
:100950000F931F93CF93DF93CDB7DEB76F970FB68B
:10096000F894DEBF0FBECDBF8B0122E02093B30C05
:100970009093C10F8093C00F85E89AE00E943D9A42
:100980008BE1E5E8FAE0DE01159601900D928A957B
:10099000E1F78091830A9091840A9C838B838DEE8A
:1009A00092E09A838983A801BE016F5F7F4F80E048
:1009B00090E010DECE0101960E9499A06F960FB6CE
:1009C000F894DEBF0FBECDBFDF91CF911F910F9185
:1009D00008952F923F924F925F926F927F928F92E3
:1009E0009F92AF92BF92CF92DF92EF92FF920F93BE
:1009F0001F93CF93DF93CDB7DEB76F970FB6F89401
:100A0000DEBF0FBECDBF6C012DB63EB61D8218866F
:100A10001C821B828DEE92E09A838983FB01808188
:100A20009E012F5F3F4F39018F3241F081E89AE0FC
:100A3000F60191838083F62E172F62C082E69AE03A
:100A4000F601918380838B010F5F1F4F0115110504
:100A500009F454C04DB65EB66FE270E0C8010E9462
:100A600006EE4C010817190708F046C07C01E01A91
:100A7000F10AFF24C70101962DB73EB7281B390B99
:100A80000FB6F8943EBF0FBE2DBF8DB79EB701962F
:100A90005C01A701B8010E942FEEF501EE0DFF1DCC
:100AA0001082F601608171816115710511F06C5F32
:100AB0007F4F21E0A501CE0105960E946C9E811119
:100AC0000FC0B50187E69DE10E949AC58EE265D40C
:100AD0008AE063D40FB6F8945EBE0FBE4DBE0EC062
:100AE000F6017182608284010F5F1F4F0FB6F89488
:100AF0005EBE0FBE4DBEAACFF02E02C0F12C10E09C
:100B0000C3010E9499A08F2D912F0FB6F8943EBE7D
:100B10000FBE2DBE6F960FB6F894DEBF0FBECDBFD1
:100B2000DF91CF911F910F91FF90EF90DF90CF90C9
:100B3000BF90AF909F908F907F906F905F904F90FD
:100B40003F902F90089590913911E92FF0E0E85BE4
:100B5000FA4F80839F5F943018F49093391102C04C
:100B60001092391180913A118F5F80933A11089554
:100B7000CF93FC0120812B33A1F020913A11243036
:100B800080F4C62FBC0180913911F0E68F9FC0011F
:100B90001124835B9A4F0E941AEE8C2FD4DF81E0E0
:100BA00001C080E0CF9108952F923F924F925F92C3
:100BB0006F927F928F929F92AF92BF92CF92DF926D
:100BC000EF92FF920F931F93CF93DF9300D000D04B
:100BD000CDB7DEB79A8389830E940259E981FA81F1
:100BE000C680D780E084F184C114D104E104F1040B
:100BF00009F0ACC22485222309F469C3328521504F
:100C0000248721E0230F22874585241301C0128603
:100C1000E981FA8124E0329FE00DF11D1124C684A0
:100C2000D784E088F188E981FA81C282D382E482A4
:100C3000F582DC01CB018C0D9D1DA11DB11D8683AC
:100C40009783A087B18784819581892B09F43FC35D
:100C5000FFB7FD83F894E981FA8122803380210176
:100C6000612C712C04811581809119028F3121F042
:100C70008F3F09F068C205C0E5E5F8E124912E83B5
:100C8000DAC08FE180931902E5E5F8E184918E8363
:100C90008F3F09F458C2823009F469C030F58823C7
:100CA00009F44CC0813009F0C6C010928000109247
:100CB0008100809181008860809381008091810013
:100CC000816080938100E6E8F6E2E491F0E0EE0FC7
:100CD000FF1FED5CF94D85919491ECECF6E2E49107
:100CE000E093C50FE1E0EE8330C19E81943009F4BA
:100CF00082C008F460C0953009F09DC010922001B8
:100D000010922101809121018860809321018091BE
:100D10002101816080932101E6E8F6E2E491F0E0B0
:100D2000EE0FFF1FED5CF94D85919491ECECF6E22E
:100D3000E491E093C20F95E09E8307C114BC15BCFB
:100D400084B5826084BD85B5816085BDE6E8F6E244
:100D5000E491F0E0EE0FFF1FED5CF94D8591949169
:100D6000ECECF6E2E491E093C60F1E82ABC2109267
:100D7000B0001092B1008091B00082608093B0000A
:100D80008091B10081608093B100E6E8F6E2E491E1
:100D9000F0E0EE0FFF1FED5CF94D8591949190937B
:100DA0002D0580932C05ECECF6E2E491E0932E0502
:100DB000F2E0FE8387C21092900010929100809121
:100DC0009100886080939100809191008160809370
:100DD0009100E6E8F6E2E491F0E0EE0FFF1FED5C33
:100DE000F94D85919491ECECF6E2E491E093C40F17
:100DF00023E02E83AAC01092A0001092A10080913F
:100E0000A10088608093A1008091A10081608093FF
:100E1000A100E6E8F6E2E491F0E0EE0FFF1FED5CE2
:100E2000F94D85919491ECECF6E2E491E093C30FD7
:100E300084E08E838AC0EE81E7FD85C161E08FE1A9
:100E40000E9471BD8E818D7F09F083C04801A12C65
:100E5000B12C60E072E18AE790E0A50194010E9464
:100E60007AEA29833A834B835C8369017A01F1E052
:100E7000CF1AD108E108F1082FEFC216D104E1041E
:100E8000F10409F008F44EC060E472E48FE090E0F1
:100E9000A50194010E947AEA69017A0181E0C81AE9
:100EA000D108E108F1089E81923009F5EFEFCE16E6
:100EB000D104E104F10409F008F4CBC160E970ED5C
:100EC00083E090E0A50194010E947AEA69017A0129
:100ED000F1E0CF1AD108E108F1082FEFC216D104D2
:100EE000E104F10411F008F041C183E027C08FEF65
:100EF000C816D104E104F104B9F0B0F068E478EE6A
:100F000081E090E0A50194010E947AEA69017A01EA
:100F100091E0C91AD108E108F108EE81EE2309F445
:100F20009AC163C181E001C082E09E81911106C037
:100F300095B5987F892B85BD7AC085E09091B100E9
:100F4000987F892B8093B10072C061E08FE10E948D
:100F500071BD4801A12CB12C60E072E18AE790E0FC
:100F6000A50194010E947AEA69017A01E1E0CE1AB2
:100F7000D108E108F108C114D104F1E0EF06F10451
:100F800088F068E478EE81E090E0A50194010E9489
:100F90007AEA69017A0181E0C81AD108E108F1080A
:100FA00083E001C081E09E81913071F490918100D5
:100FB000987F892B80938100452846284728D9F5BA
:100FC0002FEF3FEFA90168C0EE81E33071F49091FB
:100FD0009100987F892B80939100452846284728C7
:100FE00051F52FEF3FEFA90179C0FE81F43071F484
:100FF0009091A100987F892B8093A10045284628D5
:101000004728C9F42FEF3FEFA9017AC02E81253080
:1010100071F490912101987F892B809321014528BB
:101020004628472841F42FEF3FEFA9017BC0452810
:101030004628472869F0D801AA0FBB1F91010E94DA
:10104000A6EA28EE33E040E050E00E9458EA03C0F0
:101050002FEF3FEFA9018E81823081F12CF488239C
:1010600061F08130C9F06FC09E81943009F448C0AE
:10107000ACF1953009F456C066C0C7BC2093D70FB9
:101080003093D80F4093D90F5093DA0F80916E00B0
:10109000826080936E0057C0D0928900C092880011
:1010A0002093D30F3093D40F4093D50F5093D60F86
:1010B00080916F00826080936F0045C0C092B30042
:1010C00020932F053093300540933105509332051E
:1010D0008091700082608093700035C0D09299003A
:1010E000C09298002093CF0F3093D00F4093D10F30
:1010F0005093D20F8091710082608093710023C061
:10110000D092A900C092A8002093CB0F3093CC0FAF
:101110004093CD0F5093CE0F8091720082608093E8
:10112000720011C0D0922901C09228012093C70FEC
:101130003093C80F4093C90F5093CA0F809173002A
:10114000826080937300ED81EFBFC1C0DC01CB01F1
:101150008C199D09AE09BF09B7FDB9C04698E98150
:10116000FA811682178210861186B1C068E478EE83
:1011700081E090E0A50194010E947AEA69017A0178
:10118000F1E0CF1AD108E108F1082FEFC216D1041F
:10119000E104F10441F138F164E274EF80E090E0A1
:1011A000A50194010E947AEA69017A01F1E0CF1A5F
:1011B000D108E108F1082FEFC216D104E104F104CF
:1011C00009F008F4BACE62E17AE780E090E0A50188
:1011D00094010E947AEA69017A0181E0C81AD10873
:1011E000E108F10819C084E0A9CE2FEFC216D1049E
:1011F000E104F10409F008F463C062E17AE780E0F9
:1012000090E0A50194010E947AEA69017A01F1E077
:10121000CF1AD108E108F1082FEFC216D104E1047A
:10122000F104A9F0A0F089819A81AB81BC812AE008
:10123000B595A795979587952A95D1F76C017D016E
:10124000F1E0CF1AD108E108F10887E077CE86E017
:1012500075CE82E073CEEFEFCE16D104E104F10437
:1012600069F160F162E17AE780E090E0A501940124
:101270000E947AEA69017A0181E0C81AD108E1087E
:10128000F1089FEFC916D104E104F104A9F0A0F020
:1012900089819A81AB81BC813AE0B595A7959795F4
:1012A00087953A95D1F76C017D01E1E0CE1AD1081E
:1012B000E108F10885E03CCE84E03ACE83E038CE08
:1012C00084E033CE61E08FE10E9471BDBFCD2696F0
:1012D0000FB6F894DEBF0FBECDBFDF91CF911F9147
:1012E0000F91FF90EF90DF90CF90BF90AF909F90C5
:1012F0008F907F906F905F904F903F902F900895C8
:101300000F931F93CF93DF93CDB7DEB72C970FB614
:10131000F894DEBF0FBECDBFE6E3F4E08085918593
:10132000A285B385448155816681778100811181D1
:101330002281338109831A832B833C834D835E830F
:101340006F83788789879A87AB87BC87AE01475FB1
:101350005F4FBE016B5F7F4FCE0101960E943BB68F
:1013600022E434E0AE01475F5F4FBE016B5F7F4F09
:10137000CE0101960E944FC82C960FB6F894DEBF9E
:101380000FBECDBFDF91CF911F910F910895FC014A
:10139000238121110C94E09808959091C00095FF4D
:1013A000FCCF8093C6000895EF92FF921F93CF93D6
:1013B000DF937C0160E0DCDB182F882399F0E2EFFB
:1013C000FDE18491EF012196882319F0E6DFFE010B
:1013D000F8CFB70188EF9DE10E949AC582E2DDDF78
:1013E0008AE0DBDF812FDF91CF911F91FF90EF909B
:1013F0000895DF92EF92FF920F931F93CF93DF93A5
:10140000CDB7DEB76E970FB6F894DEBF0FBECDBF77
:101410006091A7077091A8076115710541F14DE131
:1014200050E0CE0101967C010E9413E61E8EF7016A
:101430008F010E191F09D190DD2019F09AE0D91201
:10144000F7CFF701E00FF11F1082C701ADDF88234E
:1014500071F0DD20A9F00F5F1F4F8091A7079091D9
:10146000A807080F191F1093A8070093A70781E08A
:101470002091A7073091A807232B29F480E003C00F
:1014800000E010E0F0CF6E960FB6F894DEBF0FBE0E
:10149000CDBFDF91CF911F910F91FF90EF90DF9023
:1014A00008953F924F925F926F927F928F929F9298
:1014B000AF92BF92CF92DF92EF92FF920F931F9362
:1014C000CF93DF931F92CDB7DEB793DF811175C243
:1014D00080913A11843008F048C00E94AD4BAC01B5
:1014E00097FF7CC142C08E3409F0D9C101151105A6
:1014F00009F4D5C16BE27FE1C8010E9422E67C01BC
:10150000892B09F48EC16EE470E0C80104960E9434
:1015100006EE009709F485C14AE050E060E070E013
:1015200001960E94BEE36093DB0F7093DC0F809303
:10153000DD0F9093DE0F8090C7189090C818A09090
:10154000C918B090CA182FEF821A920AA20AB20ADA
:10155000681579058A059B0509F465C1EF2809F02E
:1015600062C188EF9EE10E9458D78091350A882396
:1015700009F423C280913A11811102C010924110E6
:10158000EE24E3944091AF0C5091B00C6091B10CFB
:101590007091B20C8091AB0C9091AC0CA091AD0C01
:1015A000B091AE0C481759076A077B0708F4E12C85
:1015B00000E010E09924939480E6882E90E3A92E11
:1015C0009FE1B92E2DE8322E80913A11843008F037
:1015D000F4C1E110F2C1809141108111EEC18091FE
:1015E000060C9091070CA091080CB091090C809307
:1015F000AF0C9093B00CA093B10CB093B20C41E03F
:1016000050E0BE016F5F7F4F8EEF9BE00E94609BBA
:10161000019719F4898190E002C08FEF9FEFF82EB7
:101620004090AF0C5090B00C6090B10C7090B20C28
:101630004091AB0C5091AC0C6091AD0C7091AE0C24
:10164000EE24E394441655066606770608F4E12C6A
:101650004416550666067706B0F4019609F46AC08A
:101660008AE0F81609F489C09DE0F91609F485C0EE
:1016700023E2F21619F08AE3F81296C08091401026
:10168000811192C06FC00E94226A8EEF9BE00E947F
:10169000E0988091190C882359F181508093190C9E
:1016A000389EC001112441E061E0825E934F0E94A8
:1016B000B8D5E091190C94E0E99FF0011124E65EA1
:1016C000F34F40815181628173814093AF0C5093FD
:1016D000B00C6093B10C7093B20C8EEF9BE00E9443
:1016E000F6978091360A8823A9F09092350A12C0A5
:1016F0001092350A0E941DB10E94FE780E947878EF
:101700006D3371058105910528F0B092A807A0926C
:10171000A7076FDE8091350A811128C0E3E4FFE15D
:1017200084916F012FEFC21AD20A8823D9F035DED7
:10173000F601F6CFEDEDFDE184916F019FEFC91A3F
:10174000D90A882319F029DEF601F6CFE4E3FFE198
:1017500084916F012FEFC21AD20A882319F01DDE7F
:10176000F601F6CF83E2F81208C005C023E2F212B8
:1017700021C100E010E0909241101092401001153C
:10178000110519F40E94D07B0CC080913911889EFC
:10179000000D111D1124F801E35BFA4F108280E067
:1017A000D2D900E010E010CF0F35110508F00CCFB2
:1017B0009BE3F91202C09092401080914010811179
:1017C00003CF80913911F801889EE00DF11D11249D
:1017D000E35BFA4FF0820F5F1F4FF6CE982F2091F8
:1017E000C5183091C6188A3019F09D3009F0B0C084
:1017F00010923F102115310519F40E94D07B68CE5C
:10180000F901E152F04F10821092C6181092C518DB
:101810000FED1FE0F8018191803209F064CE8F0155
:10182000F9CFC80179CE6AE270E0C8010E943EEEAD
:101830009C01009701F1982F901BF12C992339F00E
:101840009150F801E90FF11D8081F826F7CF4AE0A9
:1018500050E060E070E0C90101960E94BEE3CF2C29
:10186000D12CE12CF12C6C157D058E059F0531F0F6
:1018700089ED9EE178CE8FEA9EE175CE8091DB0FF7
:101880009091DC0FA091DD0FB091DE0F8093C7180F
:101890009093C818A093C918B093CA180EC080912D
:1018A000330A882351F065EF73E0C8010E9411EEFE
:1018B000892B19F085E89EE156CE8091270281118F
:1018C00026C067E470E0C8010E9406EE0097F9F0B8
:1018D0004AE050E060E070E001960E94BEE397FDB0
:1018E00016C064307105810591052CF065307105D5
:1018F0008105910561F4EEE0FEE184917F019FEFA7
:10190000E91AF90A882319F048DDF701F6CF69EFE3
:1019100073E0C8010E9411EE892B11F4109220028D
:101920006EEF73E0C8010E9411EE892B21F485E06F
:101930009EE10E94BCA063E074E0C8010E9411EE29
:10194000892B09F42AD261E08FED9FE011D9C0CD37
:101950002F3531050CF0BCCD9C35C1F40E94AD4B48
:1019600097FDB6CD20913F102111B2CD2091C51821
:101970003091C618A9014F5F5F4F5093C61840932E
:10198000C518F901E152F04F8083A2CD9B3319F4C1
:1019900081E080933F1080913F10811199CDC90162
:1019A00001969093C6188093C518F901E152F04F43
:1019B00040838ECD10924010E5CE0F90DF91CF91F5
:1019C0001F910F91FF90EF90DF90CF90BF90AF905D
:1019D0009F908F907F906F905F904F903F90089571
:1019E0008F929F92AF92BF92EF92FF920F931F93AD
:1019F000CF93DF93CDB7DEB7A0970FB6F894DEBFD5
:101A00000FBECDBF611571058105910589F100E01B
:101A1000842E912CA12CB12C102FEE24E394F12CC8
:101A2000EC0EFD1EE00EF11C07FDFA94A5019401D9
:101A30000E9458EAF7016083B901CA010F5F61157E
:101A400071058105910541F71F3F21F1E1E0F0E0CB
:101A5000EC0FFD1FE10FF11D17FDFA9580818A3013
:101A600010F097E301C090E3890F97DC1150ECCFA1
:101A700080E3A0960FB6F894DEBF0FBECDBFDF9116
:101A8000CF911F910F91FF90EF90BF90AF909F90DB
:101A90008F9083CCA0960FB6F894DEBF0FBECDBF5B
:101AA000DF91CF911F910F91FF90EF90BF90AF907A
:101AB0009F908F900895CF92DF92EF92FF926B01EB
:101AC0007C0197FF0AC08DE268DCF094E094D0942A
:101AD000C094C11CD11CE11CF11C4AE0C701B60135
:101AE000FF90EF90DF90CF907BCF8F929F92AF923D
:101AF000BF92CF92DF92EF92FF92CF936B017C0166
:101B0000B42E20E030E0A9010E946AE687FF06C0FB
:101B10008DE243DCF7FAF094F7F8F094C0E060E06F
:101B200070E080E09FE3CB1541F02DEC3CEC4CECF9
:101B30005DE30E94CFE6CF5FF6CF9B01AC01C7010A
:101B4000B6010E94B6EA6B017C010E94FFEB4B01DB
:101B50005C014AE045DFCC2379F1C501B4010E9464
:101B60006EE69B01AC01C701B6010E94B5EA6B01AC
:101B70007C018EE212DC20E030E040E251E4C7015B
:101B8000B6010E94CFE64B015C010E94FAEB6B01AB
:101B9000770FEE08FF08C701B6018DDFC701B60158
:101BA0000E9470E69B01AC01C501B4010E94B5EA38
:101BB0006B017C01C150F9F6CF91FF90EF90DF905F
:101BC000CF90BF90AF909F908F900895CF92DF926B
:101BD000EF92FF920F931F93CF93DF9388E50E94BC
:101BE000524CD82E89E40E94524CC82E882319F0FA
:101BF0000E94EB4B1CC0DD20C1F00E941B4C20E07A
:101C000030E040E251E40E94B5EA20E030E048ECE8
